MPLINK 5.00, LINKER
Linker Map File - Created Mon May 31 14:26:03 2021

                                 Section Info
                  Section       Type    Address   Location Size(Bytes)
                ---------  ---------  ---------  ---------  ---------
               _entry_scn       code   0x000000    program   0x000006
               HighVector       code   0x000018    program   0x000006
                   .cinit    romdata   0x000200    program   0x000002
           .code_Trames.o       code   0x000202    program   0x00c4c0
.code_CMSModifV1Nettoye.o       code   0x00c6c2    program   0x0089de
         .code_InToChar.o       code   0x0150a0    program   0x000eea
          .code_HORLOGE.o       code   0x015f8a    program   0x000ce2
          .code_Tension.o       code   0x016c6c    program   0x000876
          .code_Memoire.o       code   0x0174e2    program   0x000766
                     PROG       code   0x017c48    program   0x000626
           .code_Eeprom.o       code   0x01826e    program   0x000564
              .code_CRC.o       code   0x0187d2    program   0x000384
            .code_RS485.o       code   0x018b56    program   0x0002b2
            .code_Tempo.o       code   0x018e08    program   0x00013c
         .code_i2c1writ.o       code   0x018f44    program   0x000080
         .code_i2c1gets.o       code   0x018fc4    program   0x000076
              .code_SPI.o       code   0x01903a    program   0x000040
         .code_i2c1open.o       code   0x01907a    program   0x000036
               .code_IO.o       code   0x0190b0    program   0x000032
         .code_fxd1616u.o       code   0x0190e2    program   0x00002c
                    .code       code   0x01910e    program   0x000020
         .code_fxd0808u.o       code   0x01912e    program   0x00001c
         .code_i2c1read.o       code   0x01914a    program   0x00001a
             _startup_scn       code   0x019164    program   0x000018
              .code_I2C.o       code   0x01917c    program   0x000012
           .code___init.o       code   0x01918e    program   0x000002
           .romdata_CRC.o    romdata   0x019190    program   0x000000
           .idata_CRC.o_i    romdata   0x019190    program   0x000000
      .idata_fxd0808u.o_i    romdata   0x019190    program   0x000000
      .romdata_fxd0808u.o    romdata   0x019190    program   0x000000
        .romdata_Trames.o    romdata   0x019190    program   0x000000
      .idata_fxd1616u.o_i    romdata   0x019190    program   0x000000
      .romdata_fxd1616u.o    romdata   0x019190    program   0x000000
        .idata_Trames.o_i    romdata   0x019190    program   0x000000
      .idata_i2c1open.o_i    romdata   0x019190    program   0x000000
      .romdata_i2c1open.o    romdata   0x019190    program   0x000000
         .romdata_Tempo.o    romdata   0x019190    program   0x000000
      .idata_i2c1read.o_i    romdata   0x019190    program   0x000000
      .romdata_i2c1read.o    romdata   0x019190    program   0x000000
         .idata_Tempo.o_i    romdata   0x019190    program   0x000000
      .idata_i2c1writ.o_i    romdata   0x019190    program   0x000000
      .romdata_i2c1writ.o    romdata   0x019190    program   0x000000
             .code_c018.o       code   0x019190    program   0x000000
        .idata___init.o_i    romdata   0x019190    program   0x000000
        .romdata___init.o    romdata   0x019190    program   0x000000
      .idata_i2c1gets.o_i    romdata   0x019190    program   0x000000
      .romdata_i2c1gets.o    romdata   0x019190    program   0x000000
          .romdata_c018.o    romdata   0x019190    program   0x000000
          .idata_c018.o_i    romdata   0x019190    program   0x000000
       .romdata_HORLOGE.o    romdata   0x019190    program   0x000000
       .idata_Memoire.o_i    romdata   0x019190    program   0x000000
       .romdata_Memoire.o    romdata   0x019190    program   0x000000
       .idata_HORLOGE.o_i    romdata   0x019190    program   0x000000
       .idata_Tension.o_i    romdata   0x019190    program   0x000000
       .romdata_Tension.o    romdata   0x019190    program   0x000000
         .romdata_RS485.o    romdata   0x019190    program   0x000000
            .idata_IO.o_i    romdata   0x019190    program   0x000000
            .romdata_IO.o    romdata   0x019190    program   0x000000
         .idata_RS485.o_i    romdata   0x019190    program   0x000000
      .idata_InToChar.o_i    romdata   0x019190    program   0x000000
      .romdata_InToChar.o    romdata   0x019190    program   0x000000
        .romdata_Eeprom.o    romdata   0x019190    program   0x000000
           .idata_I2C.o_i    romdata   0x019190    program   0x000000
           .romdata_I2C.o    romdata   0x019190    program   0x000000
        .idata_Eeprom.o_i    romdata   0x019190    program   0x000000
.idata_CMSModifV1Nettoye.o_i    romdata   0x019190    program   0x000000
.romdata_CMSModifV1Nettoye.o    romdata   0x019190    program   0x000000
           .romdata_SPI.o    romdata   0x019190    program   0x000000
           .idata_SPI.o_i    romdata   0x019190    program   0x000000
.config_300001_CMSModifV1Nettoye.o    romdata   0x300001    program   0x000001
.config_300002_CMSModifV1Nettoye.o    romdata   0x300002    program   0x000001
.config_300003_CMSModifV1Nettoye.o    romdata   0x300003    program   0x000001
.config_300004_CMSModifV1Nettoye.o    romdata   0x300004    program   0x000001
.config_300005_CMSModifV1Nettoye.o    romdata   0x300005    program   0x000001
.config_300006_CMSModifV1Nettoye.o    romdata   0x300006    program   0x000001
.config_300008_CMSModifV1Nettoye.o    romdata   0x300008    program   0x000001
.config_300009_CMSModifV1Nettoye.o    romdata   0x300009    program   0x000001
.config_30000a_CMSModifV1Nettoye.o    romdata   0x30000a    program   0x000001
.config_30000b_CMSModifV1Nettoye.o    romdata   0x30000b    program   0x000001
.config_30000c_CMSModifV1Nettoye.o    romdata   0x30000c    program   0x000001
.config_30000d_CMSModifV1Nettoye.o    romdata   0x30000d    program   0x000001
                MATH_DATA      udata   0x000000       data   0x000014
                 .tmpdata      udata   0x000014       data   0x00000c
                   udata1      udata   0x000100       data   0x0000fa
        .udata_InToChar.o      udata   0x0001fa       data   0x000000
        .idata_InToChar.o      idata   0x0001fa       data   0x000000
             .udata_I2C.o      udata   0x0001fa       data   0x000000
             .idata_I2C.o      idata   0x0001fa       data   0x000000
.udata_CMSModifV1Nettoye.o      udata   0x0001fa       data   0x000000
.idata_CMSModifV1Nettoye.o      idata   0x0001fa       data   0x000000
        .udata_fxd0808u.o      udata   0x0001fa       data   0x000000
        .idata_fxd0808u.o      idata   0x0001fa       data   0x000000
        .udata_fxd1616u.o      udata   0x0001fa       data   0x000000
        .idata_fxd1616u.o      idata   0x0001fa       data   0x000000
        .udata_i2c1open.o      udata   0x0001fa       data   0x000000
        .idata_i2c1open.o      idata   0x0001fa       data   0x000000
        .udata_i2c1read.o      udata   0x0001fa       data   0x000000
        .idata_i2c1read.o      idata   0x0001fa       data   0x000000
        .udata_i2c1writ.o      udata   0x0001fa       data   0x000000
        .idata_i2c1writ.o      idata   0x0001fa       data   0x000000
          .udata___init.o      udata   0x0001fa       data   0x000000
          .idata___init.o      idata   0x0001fa       data   0x000000
        .udata_i2c1gets.o      udata   0x0001fa       data   0x000000
        .idata_i2c1gets.o      idata   0x0001fa       data   0x000000
            .udata_c018.o      udata   0x0001fa       data   0x000000
            .idata_c018.o      idata   0x0001fa       data   0x000000
           .udata_Tempo.o      udata   0x0001fa       data   0x000000
           .idata_Tempo.o      idata   0x0001fa       data   0x000000
          .udata_Trames.o      udata   0x0001fa       data   0x000000
          .idata_Trames.o      idata   0x0001fa       data   0x000000
             .udata_CRC.o      udata   0x0001fa       data   0x000000
             .idata_CRC.o      idata   0x0001fa       data   0x000000
             .udata_SPI.o      udata   0x0001fa       data   0x000000
             .idata_SPI.o      idata   0x0001fa       data   0x000000
          .udata_Eeprom.o      udata   0x0001fa       data   0x000000
          .idata_Eeprom.o      idata   0x0001fa       data   0x000000
           .udata_RS485.o      udata   0x0001fa       data   0x000000
           .idata_RS485.o      idata   0x0001fa       data   0x000000
         .udata_HORLOGE.o      udata   0x0001fa       data   0x000000
         .idata_HORLOGE.o      idata   0x0001fa       data   0x000000
         .udata_Memoire.o      udata   0x0001fa       data   0x000000
         .idata_Memoire.o      idata   0x0001fa       data   0x000000
         .udata_Tension.o      udata   0x0001fa       data   0x000000
         .idata_Tension.o      idata   0x0001fa       data   0x000000
              .udata_IO.o      udata   0x0001fa       data   0x000000
              .idata_IO.o      idata   0x0001fa       data   0x000000
                   udata2      udata   0x000200       data   0x0000f2
                   udata3      udata   0x000300       data   0x0000f0
                   .stack      udata   0x000e00       data   0x0000e0
                   udata4      udata   0x000f00       data   0x000046
            SFR_UNBANKED0      udata   0x000f62       data   0x00009e



                              Program Memory Usage 
                               Start         End      
                           ---------   ---------      
                            0x000000    0x000005      
                            0x000018    0x00001d      
                            0x000200    0x01918f      
                            0x300001    0x300006      
                            0x300008    0x30000d      
            102312 out of 132120 program addresses used, program memory utilization is 77%



                              Symbols - Sorted by Name
                     Name    Address   Location    Storage File                     
                ---------  ---------  ---------  --------- ---------                
              AQUIENVOYER   0x007da6    program     extern C:\CMS2Luc\ProjetsNettoyesCMSGit\ProjetCarteMereFonctions\project\Trames.c
                  AVERAGE   0x01713c    program     extern C:\CMS2Luc\ProjetsNettoyesCMSGit\ProjetCarteMereFonctions\project\Tension.c
                      CAN   0x0173e0    program     extern C:\CMS2Luc\ProjetsNettoyesCMSGit\ProjetCarteMereFonctions\project\Tension.c
 CHERCHER_DONNNEES_CABLES   0x0085ba    program     extern C:\CMS2Luc\ProjetsNettoyesCMSGit\ProjetCarteMereFonctions\project\Trames.c
     CONTROLE_CHARGE_BATT   0x016c6c    program     extern C:\CMS2Luc\ProjetsNettoyesCMSGit\ProjetCarteMereFonctions\project\Tension.c
                    CRC16   0x018a5a    program     extern C:\CMS2Luc\ProjetsNettoyesCMSGit\ProjetCarteMereFonctions\project\CRC.c
                CRC_verif   0x01890a    program     extern C:\CMS2Luc\ProjetsNettoyesCMSGit\ProjetCarteMereFonctions\project\CRC.c
                   D0808S   0x017f58    program     static E:\3.46\pic18-lt\cxx-framework\src\traditional\math\fxd0808s.asm
                D0808SNEG   0x017f66    program     static E:\3.46\pic18-lt\cxx-framework\src\traditional\math\fxd0808s.asm
                 D0808SOK   0x017f62    program     static E:\3.46\pic18-lt\cxx-framework\src\traditional\math\fxd0808s.asm
                  D0808SX   0x017f6c    program     static E:\3.46\pic18-lt\cxx-framework\src\traditional\math\fxd0808s.asm
                   D1616S   0x017f98    program     static E:\3.46\pic18-lt\cxx-framework\src\traditional\math\fxd1616s.asm
                D1616SNEG   0x017fa6    program     static E:\3.46\pic18-lt\cxx-framework\src\traditional\math\fxd1616s.asm
                 D1616SOK   0x017fa2    program     static E:\3.46\pic18-lt\cxx-framework\src\traditional\math\fxd1616s.asm
                  D1616SX   0x017fb8    program     static E:\3.46\pic18-lt\cxx-framework\src\traditional\math\fxd1616s.asm
                  DA0808S   0x017f4e    program     static E:\3.46\pic18-lt\cxx-framework\src\traditional\math\fxd0808s.asm
                  DA1616S   0x017f88    program     static E:\3.46\pic18-lt\cxx-framework\src\traditional\math\fxd1616s.asm
        ECRIRE_EEPROMBYTE   0x0184ac    program     extern C:\CMS2Luc\ProjetsNettoyesCMSGit\ProjetCarteMereFonctions\project\Eeprom.c
           ECRIRE_HORLOGE   0x015f8a    program     extern C:\CMS2Luc\ProjetsNettoyesCMSGit\ProjetCarteMereFonctions\project\HORLOGE.c
               EFFACEMENT   0x007900    program     extern C:\CMS2Luc\ProjetsNettoyesCMSGit\ProjetCarteMereFonctions\project\Trames.c
   EFFACER_CAPTEUR_SUR_CM   0x007f0a    program     extern C:\CMS2Luc\ProjetsNettoyesCMSGit\ProjetCarteMereFonctions\project\Trames.c
        ENVOIE_DES_TRAMES   0x00dff6    program     extern C:\CMS2Luc\ProjetsNettoyesCMSGit\ProjetCarteMereFonctions\project\CMSModifV1Nettoye.c
                 FLO0832S   0x017c4c    program     extern E:\3.46\pic18-lt\cxx-framework\src\traditional\math\cast08FP.asm
                 FLO0832U   0x017c48    program     extern E:\3.46\pic18-lt\cxx-framework\src\traditional\math\cast08FP.asm
                 FLO1632S   0x017c6e    program     extern E:\3.46\pic18-lt\cxx-framework\src\traditional\math\cast16FP.asm
                 FLO1632U   0x017c6a    program     extern E:\3.46\pic18-lt\cxx-framework\src\traditional\math\cast16FP.asm
                    FPA32   0x017c96    program     extern E:\3.46\pic18-lt\cxx-framework\src\traditional\math\addFP.asm
                    FPD32   0x017dc2    program     extern E:\3.46\pic18-lt\cxx-framework\src\traditional\math\divFP.asm
                    FPM32   0x017e68    program     extern E:\3.46\pic18-lt\cxx-framework\src\traditional\math\mulFP.asm
                    FPS32   0x017c94    program     extern E:\3.46\pic18-lt\cxx-framework\src\traditional\math\addFP.asm
                 FXD0808S   0x017f42    program     extern E:\3.46\pic18-lt\cxx-framework\src\traditional\math\fxd0808s.asm
                 FXD0808U   0x01912e    program     extern E:\3.46\pic18-lt\cxx-framework\src\traditional\math\fxd0808u.c
                 FXD1616S   0x017f76    program     extern E:\3.46\pic18-lt\cxx-framework\src\traditional\math\fxd1616s.asm
                 FXD1616U   0x0190e2    program     extern E:\3.46\pic18-lt\cxx-framework\src\traditional\math\fxd1616u.c
                 FXM1616S   0x017fc2    program     extern E:\3.46\pic18-lt\cxx-framework\src\traditional\math\fxm1616s.asm
                 FXM1616U   0x01801c    program     extern E:\3.46\pic18-lt\cxx-framework\src\traditional\math\fxm1616u.asm
        GROUPE_EN_MEMOIRE   0x0174e2    program     extern C:\CMS2Luc\ProjetsNettoyesCMSGit\ProjetCarteMereFonctions\project\Memoire.c
               HighVector   0x000018    program     extern C:\CMS2Luc\ProjetsNettoyesCMSGit\ProjetCarteMereFonctions\project\CMSModifV1Nettoye.c
       IDENTIF_TYPE_CARTE   0x00975e    program     extern C:\CMS2Luc\ProjetsNettoyesCMSGit\ProjetCarteMereFonctions\project\Trames.c
                  INT3208   0x018058    program     extern E:\3.46\pic18-lt\cxx-framework\src\traditional\math\castFP08.asm
INTERROGER_TOUT_LES_CAPTEURS   0x003d88    program     extern C:\CMS2Luc\ProjetsNettoyesCMSGit\ProjetCarteMereFonctions\project\Trames.c
                 Init_I2C   0x01917c    program     extern C:\CMS2Luc\ProjetsNettoyesCMSGit\ProjetCarteMereFonctions\project\I2C.c
               Init_RS485   0x018b56    program     extern C:\CMS2Luc\ProjetsNettoyesCMSGit\ProjetCarteMereFonctions\project\RS485.c
                IntToChar   0x0150a0    program     extern C:\CMS2Luc\ProjetsNettoyesCMSGit\ProjetCarteMereFonctions\project\InToChar.c
               IntToChar5   0x0156d6    program     extern C:\CMS2Luc\ProjetsNettoyesCMSGit\ProjetCarteMereFonctions\project\InToChar.c
              LIRE_EEPROM   0x01826e    program     extern C:\CMS2Luc\ProjetsNettoyesCMSGit\ProjetCarteMereFonctions\project\Eeprom.c
             LIRE_HORLOGE   0x0160ac    program     extern C:\CMS2Luc\ProjetsNettoyesCMSGit\ProjetCarteMereFonctions\project\HORLOGE.c
      MESURE_DES_TENSIONS   0x016d36    program     extern C:\CMS2Luc\ProjetsNettoyesCMSGit\ProjetCarteMereFonctions\project\Tension.c
  METTRE_EN_MEMOIRE_LISTE   0x01758a    program     extern C:\CMS2Luc\ProjetsNettoyesCMSGit\ProjetCarteMereFonctions\project\Memoire.c
MODIFICATION_TABLE_DEXISTENCE   0x008164    program     extern C:\CMS2Luc\ProjetsNettoyesCMSGit\ProjetCarteMereFonctions\project\Trames.c
                 OpenI2C1   0x01907a    program     extern E:\3.46\pic18-lt\cxx-framework\src\pmc_common\i2c\i2c1open.c
    PREPARATION_PAGE_AUTO   0x0048a4    program     extern C:\CMS2Luc\ProjetsNettoyesCMSGit\ProjetCarteMereFonctions\project\Trames.c
           RECEVOIR_RS485   0x018bb6    program     extern C:\CMS2Luc\ProjetsNettoyesCMSGit\ProjetCarteMereFonctions\project\RS485.c
 RECHERCHE_DONNEES_GROUPE   0x004838    program     extern C:\CMS2Luc\ProjetsNettoyesCMSGit\ProjetCarteMereFonctions\project\Trames.c
  RECUPERATION_DES_TRAMES   0x01068a    program     extern C:\CMS2Luc\ProjetsNettoyesCMSGit\ProjetCarteMereFonctions\project\CMSModifV1Nettoye.c
     REMISE_EN_FORME_PAGE   0x00a1bc    program     extern C:\CMS2Luc\ProjetsNettoyesCMSGit\ProjetCarteMereFonctions\project\Trames.c
         REPOSAQUIENVOYER   0x007c6a    program     extern C:\CMS2Luc\ProjetsNettoyesCMSGit\ProjetCarteMereFonctions\project\Trames.c
                    RS485   0x018cb8    program     extern C:\CMS2Luc\ProjetsNettoyesCMSGit\ProjetCarteMereFonctions\project\RS485.c
                 ReadI2C1   0x01914a    program     extern E:\3.46\pic18-lt\cxx-framework\src\pmc_common\i2c\i2c1read.c
            SAV_EXISTENCE   0x0041c4    program     extern C:\CMS2Luc\ProjetsNettoyesCMSGit\ProjetCarteMereFonctions\project\Trames.c
                      SDR   0x005374    program     extern C:\CMS2Luc\ProjetsNettoyesCMSGit\ProjetCarteMereFonctions\project\Trames.c
                    SDRBN   0x009ea8    program     extern C:\CMS2Luc\ProjetsNettoyesCMSGit\ProjetCarteMereFonctions\project\Trames.c
                      SDW   0x008b0c    program     extern C:\CMS2Luc\ProjetsNettoyesCMSGit\ProjetCarteMereFonctions\project\Trames.c
                    SDWBN   0x009d42    program     extern C:\CMS2Luc\ProjetsNettoyesCMSGit\ProjetCarteMereFonctions\project\Trames.c
            SERIALISATION   0x008a02    program     extern C:\CMS2Luc\ProjetsNettoyesCMSGit\ProjetCarteMereFonctions\project\Trames.c
            SPI_WriteByte   0x01903a    program     extern C:\CMS2Luc\ProjetsNettoyesCMSGit\ProjetCarteMereFonctions\project\SPI.c
                  TAGTB32   0x0180a6    program     extern E:\3.46\pic18-lt\cxx-framework\src\traditional\math\gtFP.asm
                    TEMPO   0x018ec0    program     extern C:\CMS2Luc\ProjetsNettoyesCMSGit\ProjetCarteMereFonctions\project\Tempo.c
   TRAMEENVOIRS485DONNEES   0x018d8a    program     extern C:\CMS2Luc\ProjetsNettoyesCMSGit\ProjetCarteMereFonctions\project\RS485.c
TRAMERECEPTIONRS485DONNEES   0x018ce0    program     extern C:\CMS2Luc\ProjetsNettoyesCMSGit\ProjetCarteMereFonctions\project\RS485.c
TRANSFORMER_TRAME_MEM_EN_COM   0x005ee6    program     extern C:\CMS2Luc\ProjetsNettoyesCMSGit\ProjetCarteMereFonctions\project\Trames.c
          TROUVER_ROBINET   0x00c396    program     extern C:\CMS2Luc\ProjetsNettoyesCMSGit\ProjetCarteMereFonctions\project\Trames.c
               TSIGN1616A   0x01800e    program     static E:\3.46\pic18-lt\cxx-framework\src\traditional\math\fxm1616s.asm
       VALIDER_CAPTEUR_CM   0x00448c    program     extern C:\CMS2Luc\ProjetsNettoyesCMSGit\ProjetCarteMereFonctions\project\Trames.c
                WriteI2C1   0x018f44    program     extern E:\3.46\pic18-lt\cxx-framework\src\pmc_common\i2c\i2c1writ.c
              __FpCompare   0x0180b8    program     extern E:\3.46\pic18-lt\cxx-framework\src\traditional\math\compFP.asm
                 __FpExit   0x01816e    program     extern E:\3.46\pic18-lt\cxx-framework\src\traditional\math\packFP.asm
                 __FpPack   0x01819a    program     extern E:\3.46\pic18-lt\cxx-framework\src\traditional\math\packFP.asm
            __FpReturnNaN   0x018162    program     extern E:\3.46\pic18-lt\cxx-framework\src\traditional\math\packFP.asm
         __FpReturnNegInf   0x018174    program     extern E:\3.46\pic18-lt\cxx-framework\src\traditional\math\packFP.asm
        __FpReturnNegZero   0x01818c    program     extern E:\3.46\pic18-lt\cxx-framework\src\traditional\math\packFP.asm
         __FpReturnPosInf   0x01817a    program     extern E:\3.46\pic18-lt\cxx-framework\src\traditional\math\packFP.asm
        __FpReturnPosZero   0x018194    program     extern E:\3.46\pic18-lt\cxx-framework\src\traditional\math\packFP.asm
        __FpReturnSignInf   0x018170    program     extern E:\3.46\pic18-lt\cxx-framework\src\traditional\math\packFP.asm
       __FpReturnSignZero   0x018188    program     extern E:\3.46\pic18-lt\cxx-framework\src\traditional\math\packFP.asm
              __FpReturnW   0x0181f2    program     extern E:\3.46\pic18-lt\cxx-framework\src\traditional\math\packFP.asm
              __FpUnPackA   0x018212    program     extern E:\3.46\pic18-lt\cxx-framework\src\traditional\math\UnpackFP.asm
              __FpUnPackB   0x018242    program     extern E:\3.46\pic18-lt\cxx-framework\src\traditional\math\UnpackFP.asm
       ___return_lbl00000   0x01910c    program     static                          
       ___return_lbl00000   0x00001c    program     static                          
       ___return_lbl00000   0x019148    program     static                          
       ___return_lbl00000   0x000004    program     static                          
       ___return_lbl00001   0x01917a    program     static                          
       ___return_lbl00071   0x0186e8    program     static                          
        ___while_lbl00072   0x0186e0    program     static                          
        ___while_lbl00073   0x0186e4    program     static                          
               __config_0   0x300001    program     static C:\CMS2Luc\ProjetsNettoyesCMSGit\ProjetCarteMereFonctions\project\CMSModifV1Nettoye.c
               __config_1   0x300002    program     static C:\CMS2Luc\ProjetsNettoyesCMSGit\ProjetCarteMereFonctions\project\CMSModifV1Nettoye.c
              __config_10   0x30000c    program     static C:\CMS2Luc\ProjetsNettoyesCMSGit\ProjetCarteMereFonctions\project\CMSModifV1Nettoye.c
              __config_11   0x30000d    program     static C:\CMS2Luc\ProjetsNettoyesCMSGit\ProjetCarteMereFonctions\project\CMSModifV1Nettoye.c
               __config_2   0x300003    program     static C:\CMS2Luc\ProjetsNettoyesCMSGit\ProjetCarteMereFonctions\project\CMSModifV1Nettoye.c
               __config_3   0x300004    program     static C:\CMS2Luc\ProjetsNettoyesCMSGit\ProjetCarteMereFonctions\project\CMSModifV1Nettoye.c
               __config_4   0x300005    program     static C:\CMS2Luc\ProjetsNettoyesCMSGit\ProjetCarteMereFonctions\project\CMSModifV1Nettoye.c
               __config_5   0x300006    program     static C:\CMS2Luc\ProjetsNettoyesCMSGit\ProjetCarteMereFonctions\project\CMSModifV1Nettoye.c
               __config_6   0x300008    program     static C:\CMS2Luc\ProjetsNettoyesCMSGit\ProjetCarteMereFonctions\project\CMSModifV1Nettoye.c
               __config_7   0x300009    program     static C:\CMS2Luc\ProjetsNettoyesCMSGit\ProjetCarteMereFonctions\project\CMSModifV1Nettoye.c
               __config_8   0x30000a    program     static C:\CMS2Luc\ProjetsNettoyesCMSGit\ProjetCarteMereFonctions\project\CMSModifV1Nettoye.c
               __config_9   0x30000b    program     static C:\CMS2Luc\ProjetsNettoyesCMSGit\ProjetCarteMereFonctions\project\CMSModifV1Nettoye.c
                   __init   0x01918e    program     extern E:\3.46\pic18-lt\cxx-framework\src\traditional\stdclib\__init.c
             __tmplbl_252   0x005600    program     static                          
             __tmplbl_261   0x009714    program     static                          
             __tmplbl_269   0x008c22    program     static                          
             __tmplbl_270   0x008c22    program     static                          
             __tmplbl_314   0x00b968    program     static                          
             __tmplbl_315   0x00b968    program     static                          
             __tmplbl_316   0x00b968    program     static                          
             __tmplbl_317   0x00b968    program     static                          
             __tmplbl_318   0x00b968    program     static                          
             __tmplbl_319   0x00b968    program     static                          
             __tmplbl_320   0x00b968    program     static                          
             __tmplbl_447   0x00dade    program     static                          
             __tmplbl_496   0x00cd6c    program     static                          
             __tmplbl_497   0x0100fa    program     static                          
             __tmplbl_498   0x00ff86    program     static                          
             __tmplbl_499   0x00fdb0    program     static                          
               __tmplbl_5   0x015f2e    program     static                          
             __tmplbl_500   0x00fc00    program     static                          
             __tmplbl_501   0x00f8ce    program     static                          
             __tmplbl_502   0x00f54a    program     static                          
             __tmplbl_503   0x00f3da    program     static                          
             __tmplbl_504   0x00f26c    program     static                          
             __tmplbl_509   0x010676    program     static                          
             __tmplbl_510   0x010676    program     static                          
             __tmplbl_511   0x010676    program     static                          
             __tmplbl_512   0x010676    program     static                          
             __tmplbl_513   0x010676    program     static                          
             __tmplbl_514   0x010676    program     static                          
             __tmplbl_515   0x010676    program     static                          
             __tmplbl_517   0x010676    program     static                          
             __tmplbl_528   0x010676    program     static                          
             __tmplbl_529   0x010676    program     static                          
             __tmplbl_530   0x010676    program     static                          
             __tmplbl_532   0x010676    program     static                          
             __tmplbl_533   0x010676    program     static                          
             __tmplbl_534   0x010676    program     static                          
             __tmplbl_536   0x010676    program     static                          
             __tmplbl_537   0x010676    program     static                          
             __tmplbl_540   0x010676    program     static                          
             __tmplbl_554   0x014348    program     static                          
             __tmplbl_555   0x0141ee    program     static                          
             __tmplbl_556   0x013f08    program     static                          
             __tmplbl_557   0x013eea    program     static                          
             __tmplbl_558   0x013ea0    program     static                          
             __tmplbl_559   0x013d32    program     static                          
             __tmplbl_560   0x013d2a    program     static                          
             __tmplbl_561   0x013c46    program     static                          
             __tmplbl_562   0x01381a    program     static                          
             __tmplbl_563   0x014b38    program     static                          
             __tmplbl_564   0x0137fa    program     static                          
             __tmplbl_565   0x0134ec    program     static                          
             __tmplbl_566   0x012f80    program     static                          
             __tmplbl_567   0x012c9c    program     static                          
             __tmplbl_568   0x012ac6    program     static                          
             __tmplbl_569   0x01289c    program     static                          
             __tmplbl_570   0x012572    program     static                          
             __tmplbl_571   0x011a8e    program     static                          
             __tmplbl_572   0x01195a    program     static                          
             __tmplbl_573   0x01168a    program     static                          
             __tmplbl_574   0x0111ba    program     static                          
             __tmplbl_582   0x014b2e    program     static                          
             __tmplbl_583   0x014b2e    program     static                          
             __tmplbl_584   0x014b0a    program     static                          
             __tmplbl_585   0x014b38    program     static                          
             __tmplbl_586   0x014b38    program     static                          
             __tmplbl_587   0x014b38    program     static                          
             __tmplbl_588   0x014b26    program     static                          
             __tmplbl_589   0x014b0a    program     static                          
             __tmplbl_590   0x013812    program     static                          
             __tmplbl_591   0x01256c    program     static                          
             __tmplbl_593   0x014b2a    program     static                          
             __tmplbl_594   0x0137f4    program     static                          
             __tmplbl_596   0x013812    program     static                          
             __tmplbl_597   0x013ee2    program     static                          
             __tmplbl_598   0x014b2a    program     static                          
             __tmplbl_599   0x012f7c    program     static                          
             __tmplbl_600   0x012f5c    program     static                          
             __tmplbl_601   0x012f6e    program     static                          
             __tmplbl_604   0x012f7c    program     static                          
             __tmplbl_605   0x012f7c    program     static                          
             __tmplbl_632   0x011d16    program     static                          
             __tmplbl_634   0x011d16    program     static                          
             __tmplbl_635   0x011cbe    program     static                          
             __tmplbl_636   0x014b2a    program     static                          
             __tmplbl_637   0x0134e6    program     static                          
             __tmplbl_638   0x0134e6    program     static                          
             __tmplbl_641   0x014b2a    program     static                          
             __tmplbl_653   0x014b2a    program     static                          
             __tmplbl_658   0x014b2a    program     static                          
             __tmplbl_659   0x014b38    program     static                          
             __tmplbl_662   0x014b38    program     static                          
             __tmplbl_663   0x014b36    program     static                          
             __tmplbl_664   0x014b0a    program     static                          
             __tmplbl_665   0x014b1c    program     static                          
             __tmplbl_666   0x014b38    program     static                          
            __zero_memory   0x01910e    program     extern E:\3.46\pic18-lt\cxx-framework\src\traditional\proc\p18f8723.asm
                   _entry   0x000000    program     extern E:\3.46\pic18-lt\cxx-framework\src\traditional\startup\c018.c
                 _startup   0x019164    program     extern E:\3.46\pic18-lt\cxx-framework\src\traditional\startup\c018.c
               calcul_CRC   0x0187d2    program     extern C:\CMS2Luc\ProjetsNettoyesCMSGit\ProjetCarteMereFonctions\project\CRC.c
        calcul_addmemoire   0x0176b8    program     extern C:\CMS2Luc\ProjetsNettoyesCMSGit\ProjetCarteMereFonctions\project\Memoire.c
            choix_memoire   0x017a7a    program     extern C:\CMS2Luc\ProjetsNettoyesCMSGit\ProjetCarteMereFonctions\project\Memoire.c
                compare_l   0x019124    program     static E:\3.46\pic18-lt\cxx-framework\src\traditional\proc\p18f8723.asm
 construire_trame_memoire   0x002348    program     extern C:\CMS2Luc\ProjetsNettoyesCMSGit\ProjetCarteMereFonctions\project\Trames.c
             controle_CRC   0x01888a    program     extern C:\CMS2Luc\ProjetsNettoyesCMSGit\ProjetCarteMereFonctions\project\CRC.c
      creer_trame_horloge   0x01617e    program     extern C:\CMS2Luc\ProjetsNettoyesCMSGit\ProjetCarteMereFonctions\project\HORLOGE.c
                 delay_ms   0x018e3c    program     extern C:\CMS2Luc\ProjetsNettoyesCMSGit\ProjetCarteMereFonctions\project\Tempo.c
                 delay_us   0x018e08    program     extern C:\CMS2Luc\ProjetsNettoyesCMSGit\ProjetCarteMereFonctions\project\Tempo.c
                  endloop   0x019108    program     static                          
                  endloop   0x019144    program     static                          
     entrer_trame_horloge   0x0165ae    program     extern C:\CMS2Luc\ProjetsNettoyesCMSGit\ProjetCarteMereFonctions\project\HORLOGE.c
       envoyerHORLOGE_i2c   0x016062    program     extern C:\CMS2Luc\ProjetsNettoyesCMSGit\ProjetCarteMereFonctions\project\HORLOGE.c
      envoyer_TRAME_PICSD   0x00b9a6    program     extern C:\CMS2Luc\ProjetsNettoyesCMSGit\ProjetCarteMereFonctions\project\Trames.c
                 getsI2C1   0x018fc4    program     extern E:\3.46\pic18-lt\cxx-framework\src\pmc_common\i2c\i2c1gets.c
      identificationINTER   0x014b4c    program     extern C:\CMS2Luc\ProjetsNettoyesCMSGit\ProjetCarteMereFonctions\project\CMSModifV1Nettoye.c
                 init_spi   0x019058    program     extern C:\CMS2Luc\ProjetsNettoyesCMSGit\ProjetCarteMereFonctions\project\SPI.c
                    inter   0x00c6c2    program     extern C:\CMS2Luc\ProjetsNettoyesCMSGit\ProjetCarteMereFonctions\project\CMSModifV1Nettoye.c
        intervertirOUT_IN   0x0047b8    program     extern C:\CMS2Luc\ProjetsNettoyesCMSGit\ProjetCarteMereFonctions\project\Trames.c
                 jANotInf   0x017e86    program     static E:\3.46\pic18-lt\cxx-framework\src\traditional\math\mulFP.asm
                 jANotInf   0x017cbe    program     static E:\3.46\pic18-lt\cxx-framework\src\traditional\math\addFP.asm
                 jANotInf   0x017de0    program     static E:\3.46\pic18-lt\cxx-framework\src\traditional\math\divFP.asm
                 jANotNeg   0x017d52    program     static E:\3.46\pic18-lt\cxx-framework\src\traditional\math\addFP.asm
                jANotZero   0x017df4    program     static E:\3.46\pic18-lt\cxx-framework\src\traditional\math\divFP.asm
              jAandWsetup   0x017d22    program     static E:\3.46\pic18-lt\cxx-framework\src\traditional\math\addFP.asm
                  jAisNeg   0x018134    program     static E:\3.46\pic18-lt\cxx-framework\src\traditional\math\compFP.asm
                 jAltBexp   0x017d10    program     static E:\3.46\pic18-lt\cxx-framework\src\traditional\math\addFP.asm
                jBANotInf   0x017cb4    program     static E:\3.46\pic18-lt\cxx-framework\src\traditional\math\addFP.asm
                 jBNotInf   0x017ccc    program     static E:\3.46\pic18-lt\cxx-framework\src\traditional\math\addFP.asm
              jBothFinite   0x017e94    program     static E:\3.46\pic18-lt\cxx-framework\src\traditional\math\mulFP.asm
             jBothNotZero   0x0180d6    program     static E:\3.46\pic18-lt\cxx-framework\src\traditional\math\compFP.asm
             jBothNotZero   0x017ea0    program     static E:\3.46\pic18-lt\cxx-framework\src\traditional\math\mulFP.asm
            jDifOrPosSign   0x017ce0    program     static E:\3.46\pic18-lt\cxx-framework\src\traditional\math\addFP.asm
                      jEQ   0x0180f2    program     static E:\3.46\pic18-lt\cxx-framework\src\traditional\math\compFP.asm
                    jExch   0x0180fe    program     static E:\3.46\pic18-lt\cxx-framework\src\traditional\math\compFP.asm
                    jExit   0x0180a4    program     static E:\3.46\pic18-lt\cxx-framework\src\traditional\math\castFP08.asm
                   jExpEQ   0x018144    program     static E:\3.46\pic18-lt\cxx-framework\src\traditional\math\compFP.asm
                   jFinal   0x018128    program     static E:\3.46\pic18-lt\cxx-framework\src\traditional\math\compFP.asm
               jFinalSign   0x017dba    program     static E:\3.46\pic18-lt\cxx-framework\src\traditional\math\addFP.asm
                jHaveZero   0x017e9c    program     static E:\3.46\pic18-lt\cxx-framework\src\traditional\math\mulFP.asm
                jI2F08Beg   0x017c56    program     static E:\3.46\pic18-lt\cxx-framework\src\traditional\math\cast08FP.asm
                jI2F16Beg   0x017c7e    program     static E:\3.46\pic18-lt\cxx-framework\src\traditional\math\cast16FP.asm
                    jLoop   0x01808c    program     static E:\3.46\pic18-lt\cxx-framework\src\traditional\math\castFP08.asm
                    jLoop   0x017e1c    program     static E:\3.46\pic18-lt\cxx-framework\src\traditional\math\divFP.asm
                jLoopExit   0x01809a    program     static E:\3.46\pic18-lt\cxx-framework\src\traditional\math\castFP08.asm
                     jMax   0x018068    program     static E:\3.46\pic18-lt\cxx-framework\src\traditional\math\castFP08.asm
                  jMaxNeg   0x018072    program     static E:\3.46\pic18-lt\cxx-framework\src\traditional\math\castFP08.asm
                  jMaxPos   0x01806c    program     static E:\3.46\pic18-lt\cxx-framework\src\traditional\math\castFP08.asm
                      jNE   0x0180f6    program     static E:\3.46\pic18-lt\cxx-framework\src\traditional\math\compFP.asm
                    jNext   0x017e42    program     static E:\3.46\pic18-lt\cxx-framework\src\traditional\math\divFP.asm
                jNoAdjust   0x017e40    program     static E:\3.46\pic18-lt\cxx-framework\src\traditional\math\divFP.asm
                  jNoExch   0x01811e    program     static E:\3.46\pic18-lt\cxx-framework\src\traditional\math\compFP.asm
             jNotBothZero   0x017ce4    program     static E:\3.46\pic18-lt\cxx-framework\src\traditional\math\addFP.asm
                  jNotInf   0x01807c    program     static E:\3.46\pic18-lt\cxx-framework\src\traditional\math\castFP08.asm
                  jPkLoop   0x0181a8    program     static E:\3.46\pic18-lt\cxx-framework\src\traditional\math\packFP.asm
             jPkRoundDone   0x0181f2    program     static E:\3.46\pic18-lt\cxx-framework\src\traditional\math\packFP.asm
               jPkRoundIt   0x0181da    program     static E:\3.46\pic18-lt\cxx-framework\src\traditional\math\packFP.asm
             jPkShiftDone   0x0181c4    program     static E:\3.46\pic18-lt\cxx-framework\src\traditional\math\packFP.asm
           jReturnPosInf0   0x01817e    program     static E:\3.46\pic18-lt\cxx-framework\src\traditional\math\packFP.asm
                  jRotate   0x018150    program     static E:\3.46\pic18-lt\cxx-framework\src\traditional\math\compFP.asm
                   jShift   0x01813a    program     static E:\3.46\pic18-lt\cxx-framework\src\traditional\math\compFP.asm
               jShiftDone   0x017d7a    program     static E:\3.46\pic18-lt\cxx-framework\src\traditional\math\addFP.asm
               jShiftLoop   0x017d6c    program     static E:\3.46\pic18-lt\cxx-framework\src\traditional\math\addFP.asm
                jSignDone   0x017daa    program     static E:\3.46\pic18-lt\cxx-framework\src\traditional\math\addFP.asm
              jSignedZero   0x017dea    program     static E:\3.46\pic18-lt\cxx-framework\src\traditional\math\divFP.asm
                 jSignsEQ   0x0180da    program     static E:\3.46\pic18-lt\cxx-framework\src\traditional\math\compFP.asm
                  jUnpkA1   0x01821c    program     static E:\3.46\pic18-lt\cxx-framework\src\traditional\math\UnpackFP.asm
                  jUnpkA2   0x018234    program     static E:\3.46\pic18-lt\cxx-framework\src\traditional\math\UnpackFP.asm
                 jUnpkANZ   0x01822a    program     static E:\3.46\pic18-lt\cxx-framework\src\traditional\math\UnpackFP.asm
                  jUnpkB1   0x01824c    program     static E:\3.46\pic18-lt\cxx-framework\src\traditional\math\UnpackFP.asm
                  jUnpkB2   0x018264    program     static E:\3.46\pic18-lt\cxx-framework\src\traditional\math\UnpackFP.asm
                 jUnpkBNZ   0x01825a    program     static E:\3.46\pic18-lt\cxx-framework\src\traditional\math\UnpackFP.asm
                 jUnpkNaN   0x01823e    program     static E:\3.46\pic18-lt\cxx-framework\src\traditional\math\UnpackFP.asm
                 jWNotNeg   0x017d66    program     static E:\3.46\pic18-lt\cxx-framework\src\traditional\math\addFP.asm
                    jZero   0x018078    program     static E:\3.46\pic18-lt\cxx-framework\src\traditional\math\castFP08.asm
               jZero1and2   0x018182    program     static E:\3.46\pic18-lt\cxx-framework\src\traditional\math\packFP.asm
             lire_horloge   0x0167fa    program     extern C:\CMS2Luc\ProjetsNettoyesCMSGit\ProjetCarteMereFonctions\project\HORLOGE.c
           litHORLOGE_i2c   0x01612a    program     extern C:\CMS2Luc\ProjetsNettoyesCMSGit\ProjetCarteMereFonctions\project\HORLOGE.c
                     loop   0x019136    program     static                          
                     loop   0x0190ec    program     static                          
                     loop   0x019170    program     static                          
                   loop_h   0x01911c    program     static E:\3.46\pic18-lt\cxx-framework\src\traditional\proc\p18f8723.asm
                   loop_l   0x019126    program     static E:\3.46\pic18-lt\cxx-framework\src\traditional\proc\p18f8723.asm
                     main   0x00c784    program     extern C:\CMS2Luc\ProjetsNettoyesCMSGit\ProjetCarteMereFonctions\project\CMSModifV1Nettoye.c
          pic_eeprom_read   0x0186f0    program     extern C:\CMS2Luc\ProjetsNettoyesCMSGit\ProjetCarteMereFonctions\project\Eeprom.c
         pic_eeprom_write   0x0186bc    program     extern C:\CMS2Luc\ProjetsNettoyesCMSGit\ProjetCarteMereFonctions\project\Eeprom.c
             putstringI2C   0x018712    program     extern C:\CMS2Luc\ProjetsNettoyesCMSGit\ProjetCarteMereFonctions\project\Eeprom.c
  recuperer_trame_memoire   0x000264    program     extern C:\CMS2Luc\ProjetsNettoyesCMSGit\ProjetCarteMereFonctions\project\Trames.c
      reglerhorlogeautres   0x01694e    program     extern C:\CMS2Luc\ProjetsNettoyesCMSGit\ProjetCarteMereFonctions\project\HORLOGE.c
                  resetTO   0x000202    program     extern C:\CMS2Luc\ProjetsNettoyesCMSGit\ProjetCarteMereFonctions\project\Trames.c
                  spi_low   0x019074    program     extern C:\CMS2Luc\ProjetsNettoyesCMSGit\ProjetCarteMereFonctions\project\SPI.c
                   stopIO   0x0190b0    program     extern C:\CMS2Luc\ProjetsNettoyesCMSGit\ProjetCarteMereFonctions\project\IO.c
trouver_carte_suivantvoie   0x007acc    program     extern C:\CMS2Luc\ProjetsNettoyesCMSGit\ProjetCarteMereFonctions\project\Trames.c
               zero_block   0x01911c    program     static E:\3.46\pic18-lt\cxx-framework\src\traditional\proc\p18f8723.asm
                   ADCON0   0x000fc2       data     extern E:\3.46\pic18-lt\cxx-framework\src\traditional\proc\p18f8723.asm
               ADCON0bits   0x000fc2       data     extern E:\3.46\pic18-lt\cxx-framework\src\traditional\proc\p18f8723.asm
                   ADCON1   0x000fc1       data     extern E:\3.46\pic18-lt\cxx-framework\src\traditional\proc\p18f8723.asm
               ADCON1bits   0x000fc1       data     extern E:\3.46\pic18-lt\cxx-framework\src\traditional\proc\p18f8723.asm
                   ADCON2   0x000fc0       data     extern E:\3.46\pic18-lt\cxx-framework\src\traditional\proc\p18f8723.asm
               ADCON2bits   0x000fc0       data     extern E:\3.46\pic18-lt\cxx-framework\src\traditional\proc\p18f8723.asm
                    ADRES   0x000fc3       data     extern E:\3.46\pic18-lt\cxx-framework\src\traditional\proc\p18f8723.asm
                   ADRESH   0x000fc4       data     extern E:\3.46\pic18-lt\cxx-framework\src\traditional\proc\p18f8723.asm
                   ADRESL   0x000fc3       data     extern E:\3.46\pic18-lt\cxx-framework\src\traditional\proc\p18f8723.asm
                    ANNEE   0x0002f0       data     extern C:\CMS2Luc\ProjetsNettoyesCMSGit\ProjetCarteMereFonctions\project\CMSModifV1Nettoye.c
                  BAUDCON   0x000f7e       data     extern E:\3.46\pic18-lt\cxx-framework\src\traditional\proc\p18f8723.asm
                 BAUDCON1   0x000f7e       data     extern E:\3.46\pic18-lt\cxx-framework\src\traditional\proc\p18f8723.asm
             BAUDCON1bits   0x000f7e       data     extern E:\3.46\pic18-lt\cxx-framework\src\traditional\proc\p18f8723.asm
                 BAUDCON2   0x000f7c       data     extern E:\3.46\pic18-lt\cxx-framework\src\traditional\proc\p18f8723.asm
             BAUDCON2bits   0x000f7c       data     extern E:\3.46\pic18-lt\cxx-framework\src\traditional\proc\p18f8723.asm
              BAUDCONbits   0x000f7e       data     extern E:\3.46\pic18-lt\cxx-framework\src\traditional\proc\p18f8723.asm
                      BSR   0x000fe0       data     extern E:\3.46\pic18-lt\cxx-framework\src\traditional\proc\p18f8723.asm
                    CABLE   0x000234       data     extern C:\CMS2Luc\ProjetsNettoyesCMSGit\ProjetCarteMereFonctions\project\CMSModifV1Nettoye.c
        CAPTEUR_A_EFFACER   0x00028e       data     extern C:\CMS2Luc\ProjetsNettoyesCMSGit\ProjetCarteMereFonctions\project\CMSModifV1Nettoye.c
                     CCON   0x00020b       data     extern C:\CMS2Luc\ProjetsNettoyesCMSGit\ProjetCarteMereFonctions\project\CMSModifV1Nettoye.c
                  CCP1CON   0x000fbd       data     extern E:\3.46\pic18-lt\cxx-framework\src\traditional\proc\p18f8723.asm
              CCP1CONbits   0x000fbd       data     extern E:\3.46\pic18-lt\cxx-framework\src\traditional\proc\p18f8723.asm
                  CCP2CON   0x000fba       data     extern E:\3.46\pic18-lt\cxx-framework\src\traditional\proc\p18f8723.asm
              CCP2CONbits   0x000fba       data     extern E:\3.46\pic18-lt\cxx-framework\src\traditional\proc\p18f8723.asm
                  CCP3CON   0x000fb7       data     extern E:\3.46\pic18-lt\cxx-framework\src\traditional\proc\p18f8723.asm
              CCP3CONbits   0x000fb7       data     extern E:\3.46\pic18-lt\cxx-framework\src\traditional\proc\p18f8723.asm
                  CCP4CON   0x000f73       data     extern E:\3.46\pic18-lt\cxx-framework\src\traditional\proc\p18f8723.asm
              CCP4CONbits   0x000f73       data     extern E:\3.46\pic18-lt\cxx-framework\src\traditional\proc\p18f8723.asm
                  CCP5CON   0x000f70       data     extern E:\3.46\pic18-lt\cxx-framework\src\traditional\proc\p18f8723.asm
              CCP5CONbits   0x000f70       data     extern E:\3.46\pic18-lt\cxx-framework\src\traditional\proc\p18f8723.asm
                    CCPR1   0x000fbe       data     extern E:\3.46\pic18-lt\cxx-framework\src\traditional\proc\p18f8723.asm
                   CCPR1H   0x000fbf       data     extern E:\3.46\pic18-lt\cxx-framework\src\traditional\proc\p18f8723.asm
                   CCPR1L   0x000fbe       data     extern E:\3.46\pic18-lt\cxx-framework\src\traditional\proc\p18f8723.asm
                    CCPR2   0x000fbb       data     extern E:\3.46\pic18-lt\cxx-framework\src\traditional\proc\p18f8723.asm
                   CCPR2H   0x000fbc       data     extern E:\3.46\pic18-lt\cxx-framework\src\traditional\proc\p18f8723.asm
                   CCPR2L   0x000fbb       data     extern E:\3.46\pic18-lt\cxx-framework\src\traditional\proc\p18f8723.asm
                    CCPR3   0x000fb8       data     extern E:\3.46\pic18-lt\cxx-framework\src\traditional\proc\p18f8723.asm
                   CCPR3H   0x000fb9       data     extern E:\3.46\pic18-lt\cxx-framework\src\traditional\proc\p18f8723.asm
                   CCPR3L   0x000fb8       data     extern E:\3.46\pic18-lt\cxx-framework\src\traditional\proc\p18f8723.asm
                    CCPR4   0x000f74       data     extern E:\3.46\pic18-lt\cxx-framework\src\traditional\proc\p18f8723.asm
                   CCPR4H   0x000f75       data     extern E:\3.46\pic18-lt\cxx-framework\src\traditional\proc\p18f8723.asm
                   CCPR4L   0x000f74       data     extern E:\3.46\pic18-lt\cxx-framework\src\traditional\proc\p18f8723.asm
                    CCPR5   0x000f71       data     extern E:\3.46\pic18-lt\cxx-framework\src\traditional\proc\p18f8723.asm
                   CCPR5H   0x000f72       data     extern E:\3.46\pic18-lt\cxx-framework\src\traditional\proc\p18f8723.asm
                   CCPR5L   0x000f71       data     extern E:\3.46\pic18-lt\cxx-framework\src\traditional\proc\p18f8723.asm
                    CMCON   0x000fb4       data     extern E:\3.46\pic18-lt\cxx-framework\src\traditional\proc\p18f8723.asm
                CMCONbits   0x000fb4       data     extern E:\3.46\pic18-lt\cxx-framework\src\traditional\proc\p18f8723.asm
                     CMOD   0x000207       data     extern C:\CMS2Luc\ProjetsNettoyesCMSGit\ProjetCarteMereFonctions\project\CMSModifV1Nettoye.c
                      COD   0x000240       data     extern C:\CMS2Luc\ProjetsNettoyesCMSGit\ProjetCarteMereFonctions\project\CMSModifV1Nettoye.c
              COMMENTAIRE   0x000220       data     extern C:\CMS2Luc\ProjetsNettoyesCMSGit\ProjetCarteMereFonctions\project\CMSModifV1Nettoye.c
             CONSTITUTION   0x000213       data     extern C:\CMS2Luc\ProjetsNettoyesCMSGit\ProjetCarteMereFonctions\project\CMSModifV1Nettoye.c
                      CRC   0x000264       data     extern C:\CMS2Luc\ProjetsNettoyesCMSGit\ProjetCarteMereFonctions\project\CMSModifV1Nettoye.c
                 CRC_ETAT   0x000f1e       data     extern C:\CMS2Luc\ProjetsNettoyesCMSGit\ProjetCarteMereFonctions\project\CMSModifV1Nettoye.c
                     CREP   0x00020f       data     extern C:\CMS2Luc\ProjetsNettoyesCMSGit\ProjetCarteMereFonctions\project\CMSModifV1Nettoye.c
                   CVRCON   0x000fb5       data     extern E:\3.46\pic18-lt\cxx-framework\src\traditional\proc\p18f8723.asm
               CVRCONbits   0x000fb5       data     extern E:\3.46\pic18-lt\cxx-framework\src\traditional\proc\p18f8723.asm
                  DATAFIX   0x0003e6       data     extern C:\CMS2Luc\ProjetsNettoyesCMSGit\ProjetCarteMereFonctions\project\CMSModifV1Nettoye.c
                     DATE   0x0002f1       data     extern C:\CMS2Luc\ProjetsNettoyesCMSGit\ProjetCarteMereFonctions\project\CMSModifV1Nettoye.c
                     DDRA   0x000f92       data     extern E:\3.46\pic18-lt\cxx-framework\src\traditional\proc\p18f8723.asm
                 DDRAbits   0x000f92       data     extern E:\3.46\pic18-lt\cxx-framework\src\traditional\proc\p18f8723.asm
                     DDRB   0x000f93       data     extern E:\3.46\pic18-lt\cxx-framework\src\traditional\proc\p18f8723.asm
                 DDRBbits   0x000f93       data     extern E:\3.46\pic18-lt\cxx-framework\src\traditional\proc\p18f8723.asm
                     DDRC   0x000f94       data     extern E:\3.46\pic18-lt\cxx-framework\src\traditional\proc\p18f8723.asm
                 DDRCbits   0x000f94       data     extern E:\3.46\pic18-lt\cxx-framework\src\traditional\proc\p18f8723.asm
                     DDRD   0x000f95       data     extern E:\3.46\pic18-lt\cxx-framework\src\traditional\proc\p18f8723.asm
                 DDRDbits   0x000f95       data     extern E:\3.46\pic18-lt\cxx-framework\src\traditional\proc\p18f8723.asm
                     DDRE   0x000f96       data     extern E:\3.46\pic18-lt\cxx-framework\src\traditional\proc\p18f8723.asm
                 DDREbits   0x000f96       data     extern E:\3.46\pic18-lt\cxx-framework\src\traditional\proc\p18f8723.asm
                     DDRF   0x000f97       data     extern E:\3.46\pic18-lt\cxx-framework\src\traditional\proc\p18f8723.asm
                 DDRFbits   0x000f97       data     extern E:\3.46\pic18-lt\cxx-framework\src\traditional\proc\p18f8723.asm
                     DDRG   0x000f98       data     extern E:\3.46\pic18-lt\cxx-framework\src\traditional\proc\p18f8723.asm
                 DDRGbits   0x000f98       data     extern E:\3.46\pic18-lt\cxx-framework\src\traditional\proc\p18f8723.asm
                     DDRH   0x000f99       data     extern E:\3.46\pic18-lt\cxx-framework\src\traditional\proc\p18f8723.asm
                 DDRHbits   0x000f99       data     extern E:\3.46\pic18-lt\cxx-framework\src\traditional\proc\p18f8723.asm
                     DDRJ   0x000f9a       data     extern E:\3.46\pic18-lt\cxx-framework\src\traditional\proc\p18f8723.asm
                 DDRJbits   0x000f9a       data     extern E:\3.46\pic18-lt\cxx-framework\src\traditional\proc\p18f8723.asm
             DEBIT_GLOBAL   0x0003b5       data     extern C:\CMS2Luc\ProjetsNettoyesCMSGit\ProjetCarteMereFonctions\project\CMSModifV1Nettoye.c
             DEMANDEZIGIO   0x000f3c       data     extern C:\CMS2Luc\ProjetsNettoyesCMSGit\ProjetCarteMereFonctions\project\CMSModifV1Nettoye.c
             DEMANDEZPLIO   0x000f41       data     extern C:\CMS2Luc\ProjetsNettoyesCMSGit\ProjetCarteMereFonctions\project\CMSModifV1Nettoye.c
   DEMANDE_INFOS_CAPTEURS   0x000293       data     extern C:\CMS2Luc\ProjetsNettoyesCMSGit\ProjetCarteMereFonctions\project\CMSModifV1Nettoye.c
                 DISTANCE   0x000248       data     extern C:\CMS2Luc\ProjetsNettoyesCMSGit\ProjetCarteMereFonctions\project\CMSModifV1Nettoye.c
                  ECCP1AS   0x000fb6       data     extern E:\3.46\pic18-lt\cxx-framework\src\traditional\proc\p18f8723.asm
              ECCP1ASbits   0x000fb6       data     extern E:\3.46\pic18-lt\cxx-framework\src\traditional\proc\p18f8723.asm
                 ECCP1CON   0x000fbd       data     extern E:\3.46\pic18-lt\cxx-framework\src\traditional\proc\p18f8723.asm
             ECCP1CONbits   0x000fbd       data     extern E:\3.46\pic18-lt\cxx-framework\src\traditional\proc\p18f8723.asm
                 ECCP1DEL   0x000f79       data     extern E:\3.46\pic18-lt\cxx-framework\src\traditional\proc\p18f8723.asm
             ECCP1DELbits   0x000f79       data     extern E:\3.46\pic18-lt\cxx-framework\src\traditional\proc\p18f8723.asm
                  ECCP2AS   0x000f68       data     extern E:\3.46\pic18-lt\cxx-framework\src\traditional\proc\p18f8723.asm
              ECCP2ASbits   0x000f68       data     extern E:\3.46\pic18-lt\cxx-framework\src\traditional\proc\p18f8723.asm
                 ECCP2CON   0x000fba       data     extern E:\3.46\pic18-lt\cxx-framework\src\traditional\proc\p18f8723.asm
             ECCP2CONbits   0x000fba       data     extern E:\3.46\pic18-lt\cxx-framework\src\traditional\proc\p18f8723.asm
                 ECCP2DEL   0x000f67       data     extern E:\3.46\pic18-lt\cxx-framework\src\traditional\proc\p18f8723.asm
             ECCP2DELbits   0x000f67       data     extern E:\3.46\pic18-lt\cxx-framework\src\traditional\proc\p18f8723.asm
                  ECCP3AS   0x000f6a       data     extern E:\3.46\pic18-lt\cxx-framework\src\traditional\proc\p18f8723.asm
              ECCP3ASbits   0x000f6a       data     extern E:\3.46\pic18-lt\cxx-framework\src\traditional\proc\p18f8723.asm
                 ECCP3CON   0x000fb7       data     extern E:\3.46\pic18-lt\cxx-framework\src\traditional\proc\p18f8723.asm
             ECCP3CONbits   0x000fb7       data     extern E:\3.46\pic18-lt\cxx-framework\src\traditional\proc\p18f8723.asm
                 ECCP3DEL   0x000f69       data     extern E:\3.46\pic18-lt\cxx-framework\src\traditional\proc\p18f8723.asm
             ECCP3DELbits   0x000f69       data     extern E:\3.46\pic18-lt\cxx-framework\src\traditional\proc\p18f8723.asm
                    EEADR   0x000fa9       data     extern E:\3.46\pic18-lt\cxx-framework\src\traditional\proc\p18f8723.asm
                   EEADRH   0x000faa       data     extern E:\3.46\pic18-lt\cxx-framework\src\traditional\proc\p18f8723.asm
                   EECON1   0x000fa6       data     extern E:\3.46\pic18-lt\cxx-framework\src\traditional\proc\p18f8723.asm
               EECON1bits   0x000fa6       data     extern E:\3.46\pic18-lt\cxx-framework\src\traditional\proc\p18f8723.asm
                   EECON2   0x000fa7       data     extern E:\3.46\pic18-lt\cxx-framework\src\traditional\proc\p18f8723.asm
                   EEDATA   0x000fa8       data     extern E:\3.46\pic18-lt\cxx-framework\src\traditional\proc\p18f8723.asm
                 ENTREES1   0x0002e9       data     extern C:\CMS2Luc\ProjetsNettoyesCMSGit\ProjetCarteMereFonctions\project\CMSModifV1Nettoye.c
                 ENTREES2   0x0002ea       data     extern C:\CMS2Luc\ProjetsNettoyesCMSGit\ProjetCarteMereFonctions\project\CMSModifV1Nettoye.c
                    ERRMM   0x000f42       data     extern C:\CMS2Luc\ProjetsNettoyesCMSGit\ProjetCarteMereFonctions\project\CMSModifV1Nettoye.c
                     ETAT   0x00024d       data     extern C:\CMS2Luc\ProjetsNettoyesCMSGit\ProjetCarteMereFonctions\project\CMSModifV1Nettoye.c
   ETATZIZCRATIONAUTOMATE   0x000f3a       data     extern C:\CMS2Luc\ProjetsNettoyesCMSGit\ProjetCarteMereFonctions\project\CMSModifV1Nettoye.c
                  ETAT_IO   0x000f1f       data     extern C:\CMS2Luc\ProjetsNettoyesCMSGit\ProjetCarteMereFonctions\project\CMSModifV1Nettoye.c
                   FCYCLE   0x000f44       data     extern C:\CMS2Luc\ProjetsNettoyesCMSGit\ProjetCarteMereFonctions\project\CMSModifV1Nettoye.c
              FIRST_DEMAR   0x000f20       data     extern C:\CMS2Luc\ProjetsNettoyesCMSGit\ProjetCarteMereFonctions\project\CMSModifV1Nettoye.c
                 FONCTION   0x000261       data     extern C:\CMS2Luc\ProjetsNettoyesCMSGit\ProjetCarteMereFonctions\project\CMSModifV1Nettoye.c
 FONCTION_ACTIVATION_AUTO   0x000f1b       data     extern C:\CMS2Luc\ProjetsNettoyesCMSGit\ProjetCarteMereFonctions\project\CMSModifV1Nettoye.c
                     FSR0   0x000fe9       data     extern E:\3.46\pic18-lt\cxx-framework\src\traditional\proc\p18f8723.asm
                    FSR0H   0x000fea       data     extern E:\3.46\pic18-lt\cxx-framework\src\traditional\proc\p18f8723.asm
                    FSR0L   0x000fe9       data     extern E:\3.46\pic18-lt\cxx-framework\src\traditional\proc\p18f8723.asm
                     FSR1   0x000fe1       data     extern E:\3.46\pic18-lt\cxx-framework\src\traditional\proc\p18f8723.asm
                    FSR1H   0x000fe2       data     extern E:\3.46\pic18-lt\cxx-framework\src\traditional\proc\p18f8723.asm
                    FSR1L   0x000fe1       data     extern E:\3.46\pic18-lt\cxx-framework\src\traditional\proc\p18f8723.asm
                     FSR2   0x000fd9       data     extern E:\3.46\pic18-lt\cxx-framework\src\traditional\proc\p18f8723.asm
                    FSR2H   0x000fda       data     extern E:\3.46\pic18-lt\cxx-framework\src\traditional\proc\p18f8723.asm
                    FSR2L   0x000fd9       data     extern E:\3.46\pic18-lt\cxx-framework\src\traditional\proc\p18f8723.asm
                    HEURE   0x0002eb       data     extern C:\CMS2Luc\ProjetsNettoyesCMSGit\ProjetCarteMereFonctions\project\CMSModifV1Nettoye.c
                       HH   0x00023b       data     extern C:\CMS2Luc\ProjetsNettoyesCMSGit\ProjetCarteMereFonctions\project\CMSModifV1Nettoye.c
                  HLVDCON   0x000fd2       data     extern E:\3.46\pic18-lt\cxx-framework\src\traditional\proc\p18f8723.asm
              HLVDCONbits   0x000fd2       data     extern E:\3.46\pic18-lt\cxx-framework\src\traditional\proc\p18f8723.asm
                  HORLOGE   0x000282       data     extern C:\CMS2Luc\ProjetsNettoyesCMSGit\ProjetCarteMereFonctions\project\CMSModifV1Nettoye.c
                      ID1   0x00025d       data     extern C:\CMS2Luc\ProjetsNettoyesCMSGit\ProjetCarteMereFonctions\project\CMSModifV1Nettoye.c
                      ID2   0x00025f       data     extern C:\CMS2Luc\ProjetsNettoyesCMSGit\ProjetCarteMereFonctions\project\CMSModifV1Nettoye.c
                    INDF0   0x000fef       data     extern E:\3.46\pic18-lt\cxx-framework\src\traditional\proc\p18f8723.asm
                    INDF1   0x000fe7       data     extern E:\3.46\pic18-lt\cxx-framework\src\traditional\proc\p18f8723.asm
                    INDF2   0x000fdf       data     extern E:\3.46\pic18-lt\cxx-framework\src\traditional\proc\p18f8723.asm
       INFORMATION_ERREUR   0x00026c       data     extern C:\CMS2Luc\ProjetsNettoyesCMSGit\ProjetCarteMereFonctions\project\CMSModifV1Nettoye.c
              INSTRUCTION   0x0002a8       data     extern C:\CMS2Luc\ProjetsNettoyesCMSGit\ProjetCarteMereFonctions\project\CMSModifV1Nettoye.c
                   INTCON   0x000ff2       data     extern E:\3.46\pic18-lt\cxx-framework\src\traditional\proc\p18f8723.asm
                  INTCON2   0x000ff1       data     extern E:\3.46\pic18-lt\cxx-framework\src\traditional\proc\p18f8723.asm
              INTCON2bits   0x000ff1       data     extern E:\3.46\pic18-lt\cxx-framework\src\traditional\proc\p18f8723.asm
                  INTCON3   0x000ff0       data     extern E:\3.46\pic18-lt\cxx-framework\src\traditional\proc\p18f8723.asm
              INTCON3bits   0x000ff0       data     extern E:\3.46\pic18-lt\cxx-framework\src\traditional\proc\p18f8723.asm
               INTCONbits   0x000ff2       data     extern E:\3.46\pic18-lt\cxx-framework\src\traditional\proc\p18f8723.asm
                IOTRAVAIL   0x000f24       data     extern C:\CMS2Luc\ProjetsNettoyesCMSGit\ProjetCarteMereFonctions\project\CMSModifV1Nettoye.c
                     IPR1   0x000f9f       data     extern E:\3.46\pic18-lt\cxx-framework\src\traditional\proc\p18f8723.asm
                 IPR1bits   0x000f9f       data     extern E:\3.46\pic18-lt\cxx-framework\src\traditional\proc\p18f8723.asm
                     IPR2   0x000fa2       data     extern E:\3.46\pic18-lt\cxx-framework\src\traditional\proc\p18f8723.asm
                 IPR2bits   0x000fa2       data     extern E:\3.46\pic18-lt\cxx-framework\src\traditional\proc\p18f8723.asm
                     IPR3   0x000fa5       data     extern E:\3.46\pic18-lt\cxx-framework\src\traditional\proc\p18f8723.asm
                 IPR3bits   0x000fa5       data     extern E:\3.46\pic18-lt\cxx-framework\src\traditional\proc\p18f8723.asm
                       JJ   0x000237       data     extern C:\CMS2Luc\ProjetsNettoyesCMSGit\ProjetCarteMereFonctions\project\CMSModifV1Nettoye.c
                     JOUR   0x0002ef       data     extern C:\CMS2Luc\ProjetsNettoyesCMSGit\ProjetCarteMereFonctions\project\CMSModifV1Nettoye.c
                     LATA   0x000f89       data     extern E:\3.46\pic18-lt\cxx-framework\src\traditional\proc\p18f8723.asm
                 LATAbits   0x000f89       data     extern E:\3.46\pic18-lt\cxx-framework\src\traditional\proc\p18f8723.asm
                     LATB   0x000f8a       data     extern E:\3.46\pic18-lt\cxx-framework\src\traditional\proc\p18f8723.asm
                 LATBbits   0x000f8a       data     extern E:\3.46\pic18-lt\cxx-framework\src\traditional\proc\p18f8723.asm
                     LATC   0x000f8b       data     extern E:\3.46\pic18-lt\cxx-framework\src\traditional\proc\p18f8723.asm
                 LATCbits   0x000f8b       data     extern E:\3.46\pic18-lt\cxx-framework\src\traditional\proc\p18f8723.asm
                     LATD   0x000f8c       data     extern E:\3.46\pic18-lt\cxx-framework\src\traditional\proc\p18f8723.asm
                 LATDbits   0x000f8c       data     extern E:\3.46\pic18-lt\cxx-framework\src\traditional\proc\p18f8723.asm
                     LATE   0x000f8d       data     extern E:\3.46\pic18-lt\cxx-framework\src\traditional\proc\p18f8723.asm
                 LATEbits   0x000f8d       data     extern E:\3.46\pic18-lt\cxx-framework\src\traditional\proc\p18f8723.asm
                     LATF   0x000f8e       data     extern E:\3.46\pic18-lt\cxx-framework\src\traditional\proc\p18f8723.asm
                 LATFbits   0x000f8e       data     extern E:\3.46\pic18-lt\cxx-framework\src\traditional\proc\p18f8723.asm
                     LATG   0x000f8f       data     extern E:\3.46\pic18-lt\cxx-framework\src\traditional\proc\p18f8723.asm
                 LATGbits   0x000f8f       data     extern E:\3.46\pic18-lt\cxx-framework\src\traditional\proc\p18f8723.asm
                     LATH   0x000f90       data     extern E:\3.46\pic18-lt\cxx-framework\src\traditional\proc\p18f8723.asm
                 LATHbits   0x000f90       data     extern E:\3.46\pic18-lt\cxx-framework\src\traditional\proc\p18f8723.asm
                     LATJ   0x000f91       data     extern E:\3.46\pic18-lt\cxx-framework\src\traditional\proc\p18f8723.asm
                 LATJbits   0x000f91       data     extern E:\3.46\pic18-lt\cxx-framework\src\traditional\proc\p18f8723.asm
                   LVDCON   0x000fd2       data     extern E:\3.46\pic18-lt\cxx-framework\src\traditional\proc\p18f8723.asm
               LVDCONbits   0x000fd2       data     extern E:\3.46\pic18-lt\cxx-framework\src\traditional\proc\p18f8723.asm
                  MAJBLOC   0x000f40       data     extern C:\CMS2Luc\ProjetsNettoyesCMSGit\ProjetCarteMereFonctions\project\CMSModifV1Nettoye.c
                  MAXBITE   0x000f3f       data     extern C:\CMS2Luc\ProjetsNettoyesCMSGit\ProjetCarteMereFonctions\project\CMSModifV1Nettoye.c
                   MEMCON   0x000f9c       data     extern E:\3.46\pic18-lt\cxx-framework\src\traditional\proc\p18f8723.asm
               MEMCONbits   0x000f9c       data     extern E:\3.46\pic18-lt\cxx-framework\src\traditional\proc\p18f8723.asm
              MINIRESETRI   0x000f35       data     extern C:\CMS2Luc\ProjetsNettoyesCMSGit\ProjetCarteMereFonctions\project\CMSModifV1Nettoye.c
                   MINUTE   0x0002ec       data     extern C:\CMS2Luc\ProjetsNettoyesCMSGit\ProjetCarteMereFonctions\project\CMSModifV1Nettoye.c
                       MM   0x000239       data     extern C:\CMS2Luc\ProjetsNettoyesCMSGit\ProjetCarteMereFonctions\project\CMSModifV1Nettoye.c
                MODERAPID   0x000f21       data     extern C:\CMS2Luc\ProjetsNettoyesCMSGit\ProjetCarteMereFonctions\project\CMSModifV1Nettoye.c
                     MOIS   0x0002ee       data     extern C:\CMS2Luc\ProjetsNettoyesCMSGit\ProjetCarteMereFonctions\project\CMSModifV1Nettoye.c
                     NBMM   0x000f43       data     extern C:\CMS2Luc\ProjetsNettoyesCMSGit\ProjetCarteMereFonctions\project\CMSModifV1Nettoye.c
       NBRECAPTEURS_CABLE   0x000280       data     extern C:\CMS2Luc\ProjetsNettoyesCMSGit\ProjetCarteMereFonctions\project\CMSModifV1Nettoye.c
            NBREDEMANDEIO   0x000f29       data     extern C:\CMS2Luc\ProjetsNettoyesCMSGit\ProjetCarteMereFonctions\project\CMSModifV1Nettoye.c
              NORECEPTION   0x0002e2       data     extern C:\CMS2Luc\ProjetsNettoyesCMSGit\ProjetCarteMereFonctions\project\CMSModifV1Nettoye.c
              NUMEROCARTE   0x000f28       data     extern C:\CMS2Luc\ProjetsNettoyesCMSGit\ProjetCarteMereFonctions\project\CMSModifV1Nettoye.c
             OEIL_CAPTEUR   0x00029d       data     extern C:\CMS2Luc\ProjetsNettoyesCMSGit\ProjetCarteMereFonctions\project\CMSModifV1Nettoye.c
                   OSCCON   0x000fd3       data     extern E:\3.46\pic18-lt\cxx-framework\src\traditional\proc\p18f8723.asm
               OSCCONbits   0x000fd3       data     extern E:\3.46\pic18-lt\cxx-framework\src\traditional\proc\p18f8723.asm
                  OSCTUNE   0x000f9b       data     extern E:\3.46\pic18-lt\cxx-framework\src\traditional\proc\p18f8723.asm
              OSCTUNEbits   0x000f9b       data     extern E:\3.46\pic18-lt\cxx-framework\src\traditional\proc\p18f8723.asm
                     PAGE   0x0002a2       data     extern C:\CMS2Luc\ProjetsNettoyesCMSGit\ProjetCarteMereFonctions\project\CMSModifV1Nettoye.c
                  PASDE_S   0x000f25       data     extern C:\CMS2Luc\ProjetsNettoyesCMSGit\ProjetCarteMereFonctions\project\CMSModifV1Nettoye.c
                       PC   0x000ff9       data     extern E:\3.46\pic18-lt\cxx-framework\src\traditional\proc\p18f8723.asm
                      PCL   0x000ff9       data     extern E:\3.46\pic18-lt\cxx-framework\src\traditional\proc\p18f8723.asm
                   PCLATH   0x000ffa       data     extern E:\3.46\pic18-lt\cxx-framework\src\traditional\proc\p18f8723.asm
                   PCLATU   0x000ffb       data     extern E:\3.46\pic18-lt\cxx-framework\src\traditional\proc\p18f8723.asm
                     PIE1   0x000f9d       data     extern E:\3.46\pic18-lt\cxx-framework\src\traditional\proc\p18f8723.asm
                 PIE1bits   0x000f9d       data     extern E:\3.46\pic18-lt\cxx-framework\src\traditional\proc\p18f8723.asm
                     PIE2   0x000fa0       data     extern E:\3.46\pic18-lt\cxx-framework\src\traditional\proc\p18f8723.asm
                 PIE2bits   0x000fa0       data     extern E:\3.46\pic18-lt\cxx-framework\src\traditional\proc\p18f8723.asm
                     PIE3   0x000fa3       data     extern E:\3.46\pic18-lt\cxx-framework\src\traditional\proc\p18f8723.asm
                 PIE3bits   0x000fa3       data     extern E:\3.46\pic18-lt\cxx-framework\src\traditional\proc\p18f8723.asm
                     PIR1   0x000f9e       data     extern E:\3.46\pic18-lt\cxx-framework\src\traditional\proc\p18f8723.asm
                 PIR1bits   0x000f9e       data     extern E:\3.46\pic18-lt\cxx-framework\src\traditional\proc\p18f8723.asm
                     PIR2   0x000fa1       data     extern E:\3.46\pic18-lt\cxx-framework\src\traditional\proc\p18f8723.asm
                 PIR2bits   0x000fa1       data     extern E:\3.46\pic18-lt\cxx-framework\src\traditional\proc\p18f8723.asm
                     PIR3   0x000fa4       data     extern E:\3.46\pic18-lt\cxx-framework\src\traditional\proc\p18f8723.asm
                 PIR3bits   0x000fa4       data     extern E:\3.46\pic18-lt\cxx-framework\src\traditional\proc\p18f8723.asm
                   PLUSW0   0x000feb       data     extern E:\3.46\pic18-lt\cxx-framework\src\traditional\proc\p18f8723.asm
                   PLUSW1   0x000fe3       data     extern E:\3.46\pic18-lt\cxx-framework\src\traditional\proc\p18f8723.asm
                   PLUSW2   0x000fdb       data     extern E:\3.46\pic18-lt\cxx-framework\src\traditional\proc\p18f8723.asm
              POINT_ROSEE   0x0003aa       data     extern C:\CMS2Luc\ProjetsNettoyesCMSGit\ProjetCarteMereFonctions\project\CMSModifV1Nettoye.c
                    PORTA   0x000f80       data     extern E:\3.46\pic18-lt\cxx-framework\src\traditional\proc\p18f8723.asm
                PORTAbits   0x000f80       data     extern E:\3.46\pic18-lt\cxx-framework\src\traditional\proc\p18f8723.asm
                    PORTB   0x000f81       data     extern E:\3.46\pic18-lt\cxx-framework\src\traditional\proc\p18f8723.asm
                PORTBbits   0x000f81       data     extern E:\3.46\pic18-lt\cxx-framework\src\traditional\proc\p18f8723.asm
                    PORTC   0x000f82       data     extern E:\3.46\pic18-lt\cxx-framework\src\traditional\proc\p18f8723.asm
                PORTCbits   0x000f82       data     extern E:\3.46\pic18-lt\cxx-framework\src\traditional\proc\p18f8723.asm
                    PORTD   0x000f83       data     extern E:\3.46\pic18-lt\cxx-framework\src\traditional\proc\p18f8723.asm
                PORTDbits   0x000f83       data     extern E:\3.46\pic18-lt\cxx-framework\src\traditional\proc\p18f8723.asm
                    PORTE   0x000f84       data     extern E:\3.46\pic18-lt\cxx-framework\src\traditional\proc\p18f8723.asm
                PORTEbits   0x000f84       data     extern E:\3.46\pic18-lt\cxx-framework\src\traditional\proc\p18f8723.asm
                    PORTF   0x000f85       data     extern E:\3.46\pic18-lt\cxx-framework\src\traditional\proc\p18f8723.asm
                PORTFbits   0x000f85       data     extern E:\3.46\pic18-lt\cxx-framework\src\traditional\proc\p18f8723.asm
                    PORTG   0x000f86       data     extern E:\3.46\pic18-lt\cxx-framework\src\traditional\proc\p18f8723.asm
                PORTGbits   0x000f86       data     extern E:\3.46\pic18-lt\cxx-framework\src\traditional\proc\p18f8723.asm
                    PORTH   0x000f87       data     extern E:\3.46\pic18-lt\cxx-framework\src\traditional\proc\p18f8723.asm
                PORTHbits   0x000f87       data     extern E:\3.46\pic18-lt\cxx-framework\src\traditional\proc\p18f8723.asm
                    PORTJ   0x000f88       data     extern E:\3.46\pic18-lt\cxx-framework\src\traditional\proc\p18f8723.asm
                PORTJbits   0x000f88       data     extern E:\3.46\pic18-lt\cxx-framework\src\traditional\proc\p18f8723.asm
                      POS   0x000242       data     extern C:\CMS2Luc\ProjetsNettoyesCMSGit\ProjetCarteMereFonctions\project\CMSModifV1Nettoye.c
                 POSTDEC0   0x000fed       data     extern E:\3.46\pic18-lt\cxx-framework\src\traditional\proc\p18f8723.asm
                 POSTDEC1   0x000fe5       data     extern E:\3.46\pic18-lt\cxx-framework\src\traditional\proc\p18f8723.asm
                 POSTDEC2   0x000fdd       data     extern E:\3.46\pic18-lt\cxx-framework\src\traditional\proc\p18f8723.asm
                 POSTINC0   0x000fee       data     extern E:\3.46\pic18-lt\cxx-framework\src\traditional\proc\p18f8723.asm
                 POSTINC1   0x000fe6       data     extern E:\3.46\pic18-lt\cxx-framework\src\traditional\proc\p18f8723.asm
                 POSTINC2   0x000fde       data     extern E:\3.46\pic18-lt\cxx-framework\src\traditional\proc\p18f8723.asm
                      PR2   0x000fcb       data     extern E:\3.46\pic18-lt\cxx-framework\src\traditional\proc\p18f8723.asm
                      PR4   0x000f77       data     extern E:\3.46\pic18-lt\cxx-framework\src\traditional\proc\p18f8723.asm
                  PREINC0   0x000fec       data     extern E:\3.46\pic18-lt\cxx-framework\src\traditional\proc\p18f8723.asm
                  PREINC1   0x000fe4       data     extern E:\3.46\pic18-lt\cxx-framework\src\traditional\proc\p18f8723.asm
                  PREINC2   0x000fdc       data     extern E:\3.46\pic18-lt\cxx-framework\src\traditional\proc\p18f8723.asm
          PRESENCEDEBITSD   0x000f2a       data     extern C:\CMS2Luc\ProjetsNettoyesCMSGit\ProjetCarteMereFonctions\project\CMSModifV1Nettoye.c
            PRESENCE_220V   0x0003da       data     extern C:\CMS2Luc\ProjetsNettoyesCMSGit\ProjetCarteMereFonctions\project\CMSModifV1Nettoye.c
             PRESENCE_48V   0x0003e0       data     extern C:\CMS2Luc\ProjetsNettoyesCMSGit\ProjetCarteMereFonctions\project\CMSModifV1Nettoye.c
             PRIO_AUTO_IO   0x000281       data     extern C:\CMS2Luc\ProjetsNettoyesCMSGit\ProjetCarteMereFonctions\project\CMSModifV1Nettoye.c
                     PROD   0x000ff3       data     extern E:\3.46\pic18-lt\cxx-framework\src\traditional\proc\p18f8723.asm
                    PRODH   0x000ff4       data     extern E:\3.46\pic18-lt\cxx-framework\src\traditional\proc\p18f8723.asm
                    PRODL   0x000ff3       data     extern E:\3.46\pic18-lt\cxx-framework\src\traditional\proc\p18f8723.asm
                   PSPCON   0x000fb0       data     extern E:\3.46\pic18-lt\cxx-framework\src\traditional\proc\p18f8723.asm
               PSPCONbits   0x000fb0       data     extern E:\3.46\pic18-lt\cxx-framework\src\traditional\proc\p18f8723.asm
              P_RESERVOIR   0x00037d       data     extern C:\CMS2Luc\ProjetsNettoyesCMSGit\ProjetCarteMereFonctions\project\CMSModifV1Nettoye.c
                P_SECOURS   0x00039b       data     extern C:\CMS2Luc\ProjetsNettoyesCMSGit\ProjetCarteMereFonctions\project\CMSModifV1Nettoye.c
                 P_SORTIE   0x00038c       data     extern C:\CMS2Luc\ProjetsNettoyesCMSGit\ProjetCarteMereFonctions\project\CMSModifV1Nettoye.c
                  R1NOREP   0x000f2b       data     extern C:\CMS2Luc\ProjetsNettoyesCMSGit\ProjetCarteMereFonctions\project\CMSModifV1Nettoye.c
                  R2NOREP   0x000f2c       data     extern C:\CMS2Luc\ProjetsNettoyesCMSGit\ProjetCarteMereFonctions\project\CMSModifV1Nettoye.c
                  R3NOREP   0x000f2d       data     extern C:\CMS2Luc\ProjetsNettoyesCMSGit\ProjetCarteMereFonctions\project\CMSModifV1Nettoye.c
                  R4NOREP   0x000f2e       data     extern C:\CMS2Luc\ProjetsNettoyesCMSGit\ProjetCarteMereFonctions\project\CMSModifV1Nettoye.c
                  R5NOREP   0x000f2f       data     extern C:\CMS2Luc\ProjetsNettoyesCMSGit\ProjetCarteMereFonctions\project\CMSModifV1Nettoye.c
                     RCON   0x000fd0       data     extern E:\3.46\pic18-lt\cxx-framework\src\traditional\proc\p18f8723.asm
                 RCONbits   0x000fd0       data     extern E:\3.46\pic18-lt\cxx-framework\src\traditional\proc\p18f8723.asm
                    RCREG   0x000fae       data     extern E:\3.46\pic18-lt\cxx-framework\src\traditional\proc\p18f8723.asm
                   RCREG1   0x000fae       data     extern E:\3.46\pic18-lt\cxx-framework\src\traditional\proc\p18f8723.asm
                   RCREG2   0x000f6e       data     extern E:\3.46\pic18-lt\cxx-framework\src\traditional\proc\p18f8723.asm
                    RCSTA   0x000fab       data     extern E:\3.46\pic18-lt\cxx-framework\src\traditional\proc\p18f8723.asm
                   RCSTA1   0x000fab       data     extern E:\3.46\pic18-lt\cxx-framework\src\traditional\proc\p18f8723.asm
               RCSTA1bits   0x000fab       data     extern E:\3.46\pic18-lt\cxx-framework\src\traditional\proc\p18f8723.asm
                   RCSTA2   0x000f6b       data     extern E:\3.46\pic18-lt\cxx-framework\src\traditional\proc\p18f8723.asm
               RCSTA2bits   0x000f6b       data     extern E:\3.46\pic18-lt\cxx-framework\src\traditional\proc\p18f8723.asm
                RCSTAbits   0x000fab       data     extern E:\3.46\pic18-lt\cxx-framework\src\traditional\proc\p18f8723.asm
             RESCRUTATION   0x000f27       data     extern C:\CMS2Luc\ProjetsNettoyesCMSGit\ProjetCarteMereFonctions\project\CMSModifV1Nettoye.c
             SAVAUTOCYCLE   0x000f3e       data     extern C:\CMS2Luc\ProjetsNettoyesCMSGit\ProjetCarteMereFonctions\project\CMSModifV1Nettoye.c
                   SAVTAB   0x000f00       data     extern C:\CMS2Luc\ProjetsNettoyesCMSGit\ProjetCarteMereFonctions\project\CMSModifV1Nettoye.c
                  SECONDE   0x0002ed       data     extern C:\CMS2Luc\ProjetsNettoyesCMSGit\ProjetCarteMereFonctions\project\CMSModifV1Nettoye.c
                    SEUIL   0x000253       data     extern C:\CMS2Luc\ProjetsNettoyesCMSGit\ProjetCarteMereFonctions\project\CMSModifV1Nettoye.c
                     SIGN   0x000000       data     extern E:\3.46\pic18-lt\cxx-framework\src\traditional\math\cmath18.asm
                    SPBRG   0x000faf       data     extern E:\3.46\pic18-lt\cxx-framework\src\traditional\proc\p18f8723.asm
                   SPBRG1   0x000faf       data     extern E:\3.46\pic18-lt\cxx-framework\src\traditional\proc\p18f8723.asm
                   SPBRG2   0x000f6f       data     extern E:\3.46\pic18-lt\cxx-framework\src\traditional\proc\p18f8723.asm
                   SPBRGH   0x000f7f       data     extern E:\3.46\pic18-lt\cxx-framework\src\traditional\proc\p18f8723.asm
                  SPBRGH1   0x000f7f       data     extern E:\3.46\pic18-lt\cxx-framework\src\traditional\proc\p18f8723.asm
                  SPBRGH2   0x000f7d       data     extern E:\3.46\pic18-lt\cxx-framework\src\traditional\proc\p18f8723.asm
                  SSP1ADD   0x000fc8       data     extern E:\3.46\pic18-lt\cxx-framework\src\traditional\proc\p18f8723.asm
                  SSP1BUF   0x000fc9       data     extern E:\3.46\pic18-lt\cxx-framework\src\traditional\proc\p18f8723.asm
                 SSP1CON1   0x000fc6       data     extern E:\3.46\pic18-lt\cxx-framework\src\traditional\proc\p18f8723.asm
             SSP1CON1bits   0x000fc6       data     extern E:\3.46\pic18-lt\cxx-framework\src\traditional\proc\p18f8723.asm
                 SSP1CON2   0x000fc5       data     extern E:\3.46\pic18-lt\cxx-framework\src\traditional\proc\p18f8723.asm
             SSP1CON2bits   0x000fc5       data     extern E:\3.46\pic18-lt\cxx-framework\src\traditional\proc\p18f8723.asm
                 SSP1STAT   0x000fc7       data     extern E:\3.46\pic18-lt\cxx-framework\src\traditional\proc\p18f8723.asm
             SSP1STATbits   0x000fc7       data     extern E:\3.46\pic18-lt\cxx-framework\src\traditional\proc\p18f8723.asm
                  SSP2ADD   0x000f65       data     extern E:\3.46\pic18-lt\cxx-framework\src\traditional\proc\p18f8723.asm
                  SSP2BUF   0x000f66       data     extern E:\3.46\pic18-lt\cxx-framework\src\traditional\proc\p18f8723.asm
                 SSP2CON1   0x000f63       data     extern E:\3.46\pic18-lt\cxx-framework\src\traditional\proc\p18f8723.asm
             SSP2CON1bits   0x000f63       data     extern E:\3.46\pic18-lt\cxx-framework\src\traditional\proc\p18f8723.asm
                 SSP2CON2   0x000f62       data     extern E:\3.46\pic18-lt\cxx-framework\src\traditional\proc\p18f8723.asm
             SSP2CON2bits   0x000f62       data     extern E:\3.46\pic18-lt\cxx-framework\src\traditional\proc\p18f8723.asm
                 SSP2STAT   0x000f64       data     extern E:\3.46\pic18-lt\cxx-framework\src\traditional\proc\p18f8723.asm
             SSP2STATbits   0x000f64       data     extern E:\3.46\pic18-lt\cxx-framework\src\traditional\proc\p18f8723.asm
                   SSPADD   0x000fc8       data     extern E:\3.46\pic18-lt\cxx-framework\src\traditional\proc\p18f8723.asm
                   SSPBUF   0x000fc9       data     extern E:\3.46\pic18-lt\cxx-framework\src\traditional\proc\p18f8723.asm
                  SSPCON1   0x000fc6       data     extern E:\3.46\pic18-lt\cxx-framework\src\traditional\proc\p18f8723.asm
              SSPCON1bits   0x000fc6       data     extern E:\3.46\pic18-lt\cxx-framework\src\traditional\proc\p18f8723.asm
                  SSPCON2   0x000fc5       data     extern E:\3.46\pic18-lt\cxx-framework\src\traditional\proc\p18f8723.asm
              SSPCON2bits   0x000fc5       data     extern E:\3.46\pic18-lt\cxx-framework\src\traditional\proc\p18f8723.asm
                  SSPSTAT   0x000fc7       data     extern E:\3.46\pic18-lt\cxx-framework\src\traditional\proc\p18f8723.asm
              SSPSTATbits   0x000fc7       data     extern E:\3.46\pic18-lt\cxx-framework\src\traditional\proc\p18f8723.asm
                   STATUS   0x000fd8       data     extern E:\3.46\pic18-lt\cxx-framework\src\traditional\proc\p18f8723.asm
               STATUSbits   0x000fd8       data     extern E:\3.46\pic18-lt\cxx-framework\src\traditional\proc\p18f8723.asm
                   STKPTR   0x000ffc       data     extern E:\3.46\pic18-lt\cxx-framework\src\traditional\proc\p18f8723.asm
               STKPTRbits   0x000ffc       data     extern E:\3.46\pic18-lt\cxx-framework\src\traditional\proc\p18f8723.asm
                    T0CON   0x000fd5       data     extern E:\3.46\pic18-lt\cxx-framework\src\traditional\proc\p18f8723.asm
                T0CONbits   0x000fd5       data     extern E:\3.46\pic18-lt\cxx-framework\src\traditional\proc\p18f8723.asm
                    T1CON   0x000fcd       data     extern E:\3.46\pic18-lt\cxx-framework\src\traditional\proc\p18f8723.asm
                T1CONbits   0x000fcd       data     extern E:\3.46\pic18-lt\cxx-framework\src\traditional\proc\p18f8723.asm
                    T2CON   0x000fca       data     extern E:\3.46\pic18-lt\cxx-framework\src\traditional\proc\p18f8723.asm
                T2CONbits   0x000fca       data     extern E:\3.46\pic18-lt\cxx-framework\src\traditional\proc\p18f8723.asm
                    T3CON   0x000fb1       data     extern E:\3.46\pic18-lt\cxx-framework\src\traditional\proc\p18f8723.asm
                T3CONbits   0x000fb1       data     extern E:\3.46\pic18-lt\cxx-framework\src\traditional\proc\p18f8723.asm
                    T4CON   0x000f76       data     extern E:\3.46\pic18-lt\cxx-framework\src\traditional\proc\p18f8723.asm
                T4CONbits   0x000f76       data     extern E:\3.46\pic18-lt\cxx-framework\src\traditional\proc\p18f8723.asm
                   TABLAT   0x000ff5       data     extern E:\3.46\pic18-lt\cxx-framework\src\traditional\proc\p18f8723.asm
                   TBLPTR   0x000ff6       data     extern E:\3.46\pic18-lt\cxx-framework\src\traditional\proc\p18f8723.asm
                  TBLPTRH   0x000ff7       data     extern E:\3.46\pic18-lt\cxx-framework\src\traditional\proc\p18f8723.asm
                  TBLPTRL   0x000ff6       data     extern E:\3.46\pic18-lt\cxx-framework\src\traditional\proc\p18f8723.asm
                  TBLPTRU   0x000ff8       data     extern E:\3.46\pic18-lt\cxx-framework\src\traditional\proc\p18f8723.asm
       TEMPS_CYCLE_MOTEUR   0x0003c0       data     extern C:\CMS2Luc\ProjetsNettoyesCMSGit\ProjetCarteMereFonctions\project\CMSModifV1Nettoye.c
             TEMPS_MOTEUR   0x0003cb       data     extern C:\CMS2Luc\ProjetsNettoyesCMSGit\ProjetCarteMereFonctions\project\CMSModifV1Nettoye.c
                TESTCYCLE   0x000f45       data     extern C:\CMS2Luc\ProjetsNettoyesCMSGit\ProjetCarteMereFonctions\project\CMSModifV1Nettoye.c
             TIMEOUTCYCLE   0x000f37       data     extern C:\CMS2Luc\ProjetsNettoyesCMSGit\ProjetCarteMereFonctions\project\CMSModifV1Nettoye.c
                      TMP   0x000300       data     extern C:\CMS2Luc\ProjetsNettoyesCMSGit\ProjetCarteMereFonctions\project\CMSModifV1Nettoye.c
                     TMPI   0x0002e7       data     extern C:\CMS2Luc\ProjetsNettoyesCMSGit\ProjetCarteMereFonctions\project\CMSModifV1Nettoye.c
                    TMR0H   0x000fd7       data     extern E:\3.46\pic18-lt\cxx-framework\src\traditional\proc\p18f8723.asm
                    TMR0L   0x000fd6       data     extern E:\3.46\pic18-lt\cxx-framework\src\traditional\proc\p18f8723.asm
                    TMR1H   0x000fcf       data     extern E:\3.46\pic18-lt\cxx-framework\src\traditional\proc\p18f8723.asm
                    TMR1L   0x000fce       data     extern E:\3.46\pic18-lt\cxx-framework\src\traditional\proc\p18f8723.asm
                     TMR2   0x000fcc       data     extern E:\3.46\pic18-lt\cxx-framework\src\traditional\proc\p18f8723.asm
                    TMR3H   0x000fb3       data     extern E:\3.46\pic18-lt\cxx-framework\src\traditional\proc\p18f8723.asm
                    TMR3L   0x000fb2       data     extern E:\3.46\pic18-lt\cxx-framework\src\traditional\proc\p18f8723.asm
                     TMR4   0x000f78       data     extern E:\3.46\pic18-lt\cxx-framework\src\traditional\proc\p18f8723.asm
                      TOS   0x000ffd       data     extern E:\3.46\pic18-lt\cxx-framework\src\traditional\proc\p18f8723.asm
                     TOSH   0x000ffe       data     extern E:\3.46\pic18-lt\cxx-framework\src\traditional\proc\p18f8723.asm
                     TOSL   0x000ffd       data     extern E:\3.46\pic18-lt\cxx-framework\src\traditional\proc\p18f8723.asm
                     TOSU   0x000fff       data     extern E:\3.46\pic18-lt\cxx-framework\src\traditional\proc\p18f8723.asm
                  TRAMEIN   0x00017d       data     extern C:\CMS2Luc\ProjetsNettoyesCMSGit\ProjetCarteMereFonctions\project\CMSModifV1Nettoye.c
                 TRAMEOUT   0x000100       data     extern C:\CMS2Luc\ProjetsNettoyesCMSGit\ProjetCarteMereFonctions\project\CMSModifV1Nettoye.c
                    TRISA   0x000f92       data     extern E:\3.46\pic18-lt\cxx-framework\src\traditional\proc\p18f8723.asm
                TRISAbits   0x000f92       data     extern E:\3.46\pic18-lt\cxx-framework\src\traditional\proc\p18f8723.asm
                    TRISB   0x000f93       data     extern E:\3.46\pic18-lt\cxx-framework\src\traditional\proc\p18f8723.asm
                TRISBbits   0x000f93       data     extern E:\3.46\pic18-lt\cxx-framework\src\traditional\proc\p18f8723.asm
                    TRISC   0x000f94       data     extern E:\3.46\pic18-lt\cxx-framework\src\traditional\proc\p18f8723.asm
                TRISCbits   0x000f94       data     extern E:\3.46\pic18-lt\cxx-framework\src\traditional\proc\p18f8723.asm
                    TRISD   0x000f95       data     extern E:\3.46\pic18-lt\cxx-framework\src\traditional\proc\p18f8723.asm
                TRISDbits   0x000f95       data     extern E:\3.46\pic18-lt\cxx-framework\src\traditional\proc\p18f8723.asm
                    TRISE   0x000f96       data     extern E:\3.46\pic18-lt\cxx-framework\src\traditional\proc\p18f8723.asm
                TRISEbits   0x000f96       data     extern E:\3.46\pic18-lt\cxx-framework\src\traditional\proc\p18f8723.asm
                    TRISF   0x000f97       data     extern E:\3.46\pic18-lt\cxx-framework\src\traditional\proc\p18f8723.asm
                TRISFbits   0x000f97       data     extern E:\3.46\pic18-lt\cxx-framework\src\traditional\proc\p18f8723.asm
                    TRISG   0x000f98       data     extern E:\3.46\pic18-lt\cxx-framework\src\traditional\proc\p18f8723.asm
                TRISGbits   0x000f98       data     extern E:\3.46\pic18-lt\cxx-framework\src\traditional\proc\p18f8723.asm
                    TRISH   0x000f99       data     extern E:\3.46\pic18-lt\cxx-framework\src\traditional\proc\p18f8723.asm
                TRISHbits   0x000f99       data     extern E:\3.46\pic18-lt\cxx-framework\src\traditional\proc\p18f8723.asm
                    TRISJ   0x000f9a       data     extern E:\3.46\pic18-lt\cxx-framework\src\traditional\proc\p18f8723.asm
                TRISJbits   0x000f9a       data     extern E:\3.46\pic18-lt\cxx-framework\src\traditional\proc\p18f8723.asm
         TROPDENONREPONSE   0x000f1d       data     extern C:\CMS2Luc\ProjetsNettoyesCMSGit\ProjetCarteMereFonctions\project\CMSModifV1Nettoye.c
                    TXREG   0x000fad       data     extern E:\3.46\pic18-lt\cxx-framework\src\traditional\proc\p18f8723.asm
                   TXREG1   0x000fad       data     extern E:\3.46\pic18-lt\cxx-framework\src\traditional\proc\p18f8723.asm
                   TXREG2   0x000f6d       data     extern E:\3.46\pic18-lt\cxx-framework\src\traditional\proc\p18f8723.asm
                    TXSTA   0x000fac       data     extern E:\3.46\pic18-lt\cxx-framework\src\traditional\proc\p18f8723.asm
                   TXSTA1   0x000fac       data     extern E:\3.46\pic18-lt\cxx-framework\src\traditional\proc\p18f8723.asm
               TXSTA1bits   0x000fac       data     extern E:\3.46\pic18-lt\cxx-framework\src\traditional\proc\p18f8723.asm
                   TXSTA2   0x000f6c       data     extern E:\3.46\pic18-lt\cxx-framework\src\traditional\proc\p18f8723.asm
               TXSTA2bits   0x000f6c       data     extern E:\3.46\pic18-lt\cxx-framework\src\traditional\proc\p18f8723.asm
                TXSTAbits   0x000fac       data     extern E:\3.46\pic18-lt\cxx-framework\src\traditional\proc\p18f8723.asm
                     TYPE   0x000206       data     extern C:\CMS2Luc\ProjetsNettoyesCMSGit\ProjetCarteMereFonctions\project\CMSModifV1Nettoye.c
                TYPECARTE   0x000257       data     extern C:\CMS2Luc\ProjetsNettoyesCMSGit\ProjetCarteMereFonctions\project\CMSModifV1Nettoye.c
             TYPECOMMANDE   0x000f22       data     extern C:\CMS2Luc\ProjetsNettoyesCMSGit\ProjetCarteMereFonctions\project\CMSModifV1Nettoye.c
          TYPEDECARTEOEIL   0x000f36       data     extern C:\CMS2Luc\ProjetsNettoyesCMSGit\ProjetCarteMereFonctions\project\CMSModifV1Nettoye.c
              TYPE_ERREUR   0x00026a       data     extern C:\CMS2Luc\ProjetsNettoyesCMSGit\ProjetCarteMereFonctions\project\CMSModifV1Nettoye.c
               UNRESETRI1   0x000f30       data     extern C:\CMS2Luc\ProjetsNettoyesCMSGit\ProjetCarteMereFonctions\project\CMSModifV1Nettoye.c
               UNRESETRI2   0x000f31       data     extern C:\CMS2Luc\ProjetsNettoyesCMSGit\ProjetCarteMereFonctions\project\CMSModifV1Nettoye.c
               UNRESETRI3   0x000f32       data     extern C:\CMS2Luc\ProjetsNettoyesCMSGit\ProjetCarteMereFonctions\project\CMSModifV1Nettoye.c
               UNRESETRI4   0x000f33       data     extern C:\CMS2Luc\ProjetsNettoyesCMSGit\ProjetCarteMereFonctions\project\CMSModifV1Nettoye.c
               UNRESETRI5   0x000f34       data     extern C:\CMS2Luc\ProjetsNettoyesCMSGit\ProjetCarteMereFonctions\project\CMSModifV1Nettoye.c
                   VALEUR   0x00024f       data     extern C:\CMS2Luc\ProjetsNettoyesCMSGit\ProjetCarteMereFonctions\project\CMSModifV1Nettoye.c
                     VBAT   0x0002de       data     extern C:\CMS2Luc\ProjetsNettoyesCMSGit\ProjetCarteMereFonctions\project\CMSModifV1Nettoye.c
                     VDD1   0x0002c2       data     extern C:\CMS2Luc\ProjetsNettoyesCMSGit\ProjetCarteMereFonctions\project\CMSModifV1Nettoye.c
                     VDD2   0x0002c6       data     extern C:\CMS2Luc\ProjetsNettoyesCMSGit\ProjetCarteMereFonctions\project\CMSModifV1Nettoye.c
                     VDD3   0x0002ca       data     extern C:\CMS2Luc\ProjetsNettoyesCMSGit\ProjetCarteMereFonctions\project\CMSModifV1Nettoye.c
                     VDD4   0x0002ce       data     extern C:\CMS2Luc\ProjetsNettoyesCMSGit\ProjetCarteMereFonctions\project\CMSModifV1Nettoye.c
                     VDD5   0x0002d2       data     extern C:\CMS2Luc\ProjetsNettoyesCMSGit\ProjetCarteMereFonctions\project\CMSModifV1Nettoye.c
                     VDD6   0x0002da       data     extern C:\CMS2Luc\ProjetsNettoyesCMSGit\ProjetCarteMereFonctions\project\CMSModifV1Nettoye.c
                  VOIECOD   0x000200       data     extern C:\CMS2Luc\ProjetsNettoyesCMSGit\ProjetCarteMereFonctions\project\CMSModifV1Nettoye.c
                    Vtemp   0x0002d6       data     extern C:\CMS2Luc\ProjetsNettoyesCMSGit\ProjetCarteMereFonctions\project\CMSModifV1Nettoye.c
                   WDTCON   0x000fd1       data     extern E:\3.46\pic18-lt\cxx-framework\src\traditional\proc\p18f8723.asm
               WDTCONbits   0x000fd1       data     extern E:\3.46\pic18-lt\cxx-framework\src\traditional\proc\p18f8723.asm
                     WREG   0x000fe8       data     extern E:\3.46\pic18-lt\cxx-framework\src\traditional\proc\p18f8723.asm
                 __AARGB0   0x000009       data     extern E:\3.46\pic18-lt\cxx-framework\src\traditional\math\aarg.asm
                 __AARGB1   0x000008       data     extern E:\3.46\pic18-lt\cxx-framework\src\traditional\math\aarg.asm
                 __AARGB2   0x000007       data     extern E:\3.46\pic18-lt\cxx-framework\src\traditional\math\aarg.asm
                 __AARGB3   0x000006       data     extern E:\3.46\pic18-lt\cxx-framework\src\traditional\math\aarg.asm
                 __AARGB4   0x000005       data     extern E:\3.46\pic18-lt\cxx-framework\src\traditional\math\aarg.asm
                 __AARGB5   0x000004       data     extern E:\3.46\pic18-lt\cxx-framework\src\traditional\math\aarg.asm
                 __AARGB6   0x000003       data     extern E:\3.46\pic18-lt\cxx-framework\src\traditional\math\aarg.asm
                 __AARGB7   0x000002       data     extern E:\3.46\pic18-lt\cxx-framework\src\traditional\math\aarg.asm
                   __AEXP   0x00000a       data     extern E:\3.46\pic18-lt\cxx-framework\src\traditional\math\aarg.asm
                 __BARGB0   0x00000e       data     extern E:\3.46\pic18-lt\cxx-framework\src\traditional\math\barg.asm
                 __BARGB1   0x00000d       data     extern E:\3.46\pic18-lt\cxx-framework\src\traditional\math\barg.asm
                 __BARGB2   0x00000c       data     extern E:\3.46\pic18-lt\cxx-framework\src\traditional\math\barg.asm
                 __BARGB3   0x00000b       data     extern E:\3.46\pic18-lt\cxx-framework\src\traditional\math\barg.asm
                   __BEXP   0x00000f       data     extern E:\3.46\pic18-lt\cxx-framework\src\traditional\math\barg.asm
                __FPFLAGS   0x000001       data     extern E:\3.46\pic18-lt\cxx-framework\src\traditional\math\cmath18.asm
            __FPFLAGSbits   0x000001       data     extern E:\3.46\pic18-lt\cxx-framework\src\traditional\math\cmath18.asm
                  __REMB0   0x000005       data     extern E:\3.46\pic18-lt\cxx-framework\src\traditional\math\aarg.asm
                  __REMB1   0x000004       data     extern E:\3.46\pic18-lt\cxx-framework\src\traditional\math\aarg.asm
                  __REMB2   0x000003       data     extern E:\3.46\pic18-lt\cxx-framework\src\traditional\math\aarg.asm
                  __REMB3   0x000002       data     extern E:\3.46\pic18-lt\cxx-framework\src\traditional\math\aarg.asm
                   __TEMP   0x000013       data     extern E:\3.46\pic18-lt\cxx-framework\src\traditional\math\temparg.asm
                 __TEMPB0   0x000013       data     extern E:\3.46\pic18-lt\cxx-framework\src\traditional\math\temparg.asm
                 __TEMPB1   0x000012       data     extern E:\3.46\pic18-lt\cxx-framework\src\traditional\math\temparg.asm
                 __TEMPB2   0x000011       data     extern E:\3.46\pic18-lt\cxx-framework\src\traditional\math\temparg.asm
                 __TEMPB3   0x000010       data     extern E:\3.46\pic18-lt\cxx-framework\src\traditional\math\temparg.asm
                  __tmp_0   0x000014       data     static C:\CMS2Luc\ProjetsNettoyesCMSGit\ProjetCarteMereFonctions\project\Tempo.c
                  __tmp_0   0x000014       data     static C:\CMS2Luc\ProjetsNettoyesCMSGit\ProjetCarteMereFonctions\project\Trames.c
                  __tmp_0   0x000014       data     static C:\CMS2Luc\ProjetsNettoyesCMSGit\ProjetCarteMereFonctions\project\CRC.c
                  __tmp_0   0x000014       data     static C:\CMS2Luc\ProjetsNettoyesCMSGit\ProjetCarteMereFonctions\project\Eeprom.c
                  __tmp_0   0x000014       data     static C:\CMS2Luc\ProjetsNettoyesCMSGit\ProjetCarteMereFonctions\project\RS485.c
                  __tmp_0   0x000014       data     static C:\CMS2Luc\ProjetsNettoyesCMSGit\ProjetCarteMereFonctions\project\HORLOGE.c
                  __tmp_0   0x000014       data     static C:\CMS2Luc\ProjetsNettoyesCMSGit\ProjetCarteMereFonctions\project\Memoire.c
                  __tmp_0   0x000014       data     static C:\CMS2Luc\ProjetsNettoyesCMSGit\ProjetCarteMereFonctions\project\Tension.c
                  __tmp_0   0x000014       data     static C:\CMS2Luc\ProjetsNettoyesCMSGit\ProjetCarteMereFonctions\project\InToChar.c
                  __tmp_0   0x000014       data     static C:\CMS2Luc\ProjetsNettoyesCMSGit\ProjetCarteMereFonctions\project\CMSModifV1Nettoye.c
                  __tmp_0   0x000014       data     static E:\3.46\pic18-lt\cxx-framework\src\pmc_common\i2c\i2c1writ.c
              cDebutTrame   0x00025c       data     extern C:\CMS2Luc\ProjetsNettoyesCMSGit\ProjetCarteMereFonctions\project\CMSModifV1Nettoye.c
                cFinTrame   0x000269       data     extern C:\CMS2Luc\ProjetsNettoyesCMSGit\ProjetCarteMereFonctions\project\CMSModifV1Nettoye.c
               calculBLOC   0x000f19       data     extern C:\CMS2Luc\ProjetsNettoyesCMSGit\ProjetCarteMereFonctions\project\CMSModifV1Nettoye.c
               capt_exist   0x0002c1       data     extern C:\CMS2Luc\ProjetsNettoyesCMSGit\ProjetCarteMereFonctions\project\CMSModifV1Nettoye.c
                   cycleN   0x000f26       data     extern C:\CMS2Luc\ProjetsNettoyesCMSGit\ProjetCarteMereFonctions\project\CMSModifV1Nettoye.c
                       ii   0x00023f       data     extern C:\CMS2Luc\ProjetsNettoyesCMSGit\ProjetCarteMereFonctions\project\CMSModifV1Nettoye.c
                     iiii   0x000244       data     extern C:\CMS2Luc\ProjetsNettoyesCMSGit\ProjetCarteMereFonctions\project\CMSModifV1Nettoye.c
                       mm   0x00023d       data     extern C:\CMS2Luc\ProjetsNettoyesCMSGit\ProjetCarteMereFonctions\project\CMSModifV1Nettoye.c
             mouchardINT0   0x000f3b       data     extern C:\CMS2Luc\ProjetsNettoyesCMSGit\ProjetCarteMereFonctions\project\CMSModifV1Nettoye.c
             numdecarteRI   0x000f1c       data     extern C:\CMS2Luc\ProjetsNettoyesCMSGit\ProjetCarteMereFonctions\project\CMSModifV1Nettoye.c
          pointeur_out_in   0x0002e3       data     extern C:\CMS2Luc\ProjetsNettoyesCMSGit\ProjetCarteMereFonctions\project\CMSModifV1Nettoye.c
           resetheurefixe   0x000f3d       data     extern C:\CMS2Luc\ProjetsNettoyesCMSGit\ProjetCarteMereFonctions\project\CMSModifV1Nettoye.c
        scrutationunevoie   0x000f39       data     extern C:\CMS2Luc\ProjetsNettoyesCMSGit\ProjetCarteMereFonctions\project\CMSModifV1Nettoye.c
         temoinfinvoieZIZ   0x000f23       data     extern C:\CMS2Luc\ProjetsNettoyesCMSGit\ProjetCarteMereFonctions\project\CMSModifV1Nettoye.c
                      tmp   0x0002e5       data     extern C:\CMS2Luc\ProjetsNettoyesCMSGit\ProjetCarteMereFonctions\project\CMSModifV1Nettoye.c
                     tmp2   0x0002e6       data     extern C:\CMS2Luc\ProjetsNettoyesCMSGit\ProjetCarteMereFonctions\project\CMSModifV1Nettoye.c



                              Symbols - Sorted by Address
                     Name    Address   Location    Storage File                     
                ---------  ---------  ---------  --------- ---------                
                   _entry   0x000000    program     extern E:\3.46\pic18-lt\cxx-framework\src\traditional\startup\c018.c
       ___return_lbl00000   0x000004    program     static                          
               HighVector   0x000018    program     extern C:\CMS2Luc\ProjetsNettoyesCMSGit\ProjetCarteMereFonctions\project\CMSModifV1Nettoye.c
       ___return_lbl00000   0x00001c    program     static                          
                  resetTO   0x000202    program     extern C:\CMS2Luc\ProjetsNettoyesCMSGit\ProjetCarteMereFonctions\project\Trames.c
  recuperer_trame_memoire   0x000264    program     extern C:\CMS2Luc\ProjetsNettoyesCMSGit\ProjetCarteMereFonctions\project\Trames.c
 construire_trame_memoire   0x002348    program     extern C:\CMS2Luc\ProjetsNettoyesCMSGit\ProjetCarteMereFonctions\project\Trames.c
INTERROGER_TOUT_LES_CAPTEURS   0x003d88    program     extern C:\CMS2Luc\ProjetsNettoyesCMSGit\ProjetCarteMereFonctions\project\Trames.c
            SAV_EXISTENCE   0x0041c4    program     extern C:\CMS2Luc\ProjetsNettoyesCMSGit\ProjetCarteMereFonctions\project\Trames.c
       VALIDER_CAPTEUR_CM   0x00448c    program     extern C:\CMS2Luc\ProjetsNettoyesCMSGit\ProjetCarteMereFonctions\project\Trames.c
        intervertirOUT_IN   0x0047b8    program     extern C:\CMS2Luc\ProjetsNettoyesCMSGit\ProjetCarteMereFonctions\project\Trames.c
 RECHERCHE_DONNEES_GROUPE   0x004838    program     extern C:\CMS2Luc\ProjetsNettoyesCMSGit\ProjetCarteMereFonctions\project\Trames.c
    PREPARATION_PAGE_AUTO   0x0048a4    program     extern C:\CMS2Luc\ProjetsNettoyesCMSGit\ProjetCarteMereFonctions\project\Trames.c
                      SDR   0x005374    program     extern C:\CMS2Luc\ProjetsNettoyesCMSGit\ProjetCarteMereFonctions\project\Trames.c
             __tmplbl_252   0x005600    program     static                          
TRANSFORMER_TRAME_MEM_EN_COM   0x005ee6    program     extern C:\CMS2Luc\ProjetsNettoyesCMSGit\ProjetCarteMereFonctions\project\Trames.c
               EFFACEMENT   0x007900    program     extern C:\CMS2Luc\ProjetsNettoyesCMSGit\ProjetCarteMereFonctions\project\Trames.c
trouver_carte_suivantvoie   0x007acc    program     extern C:\CMS2Luc\ProjetsNettoyesCMSGit\ProjetCarteMereFonctions\project\Trames.c
         REPOSAQUIENVOYER   0x007c6a    program     extern C:\CMS2Luc\ProjetsNettoyesCMSGit\ProjetCarteMereFonctions\project\Trames.c
              AQUIENVOYER   0x007da6    program     extern C:\CMS2Luc\ProjetsNettoyesCMSGit\ProjetCarteMereFonctions\project\Trames.c
   EFFACER_CAPTEUR_SUR_CM   0x007f0a    program     extern C:\CMS2Luc\ProjetsNettoyesCMSGit\ProjetCarteMereFonctions\project\Trames.c
MODIFICATION_TABLE_DEXISTENCE   0x008164    program     extern C:\CMS2Luc\ProjetsNettoyesCMSGit\ProjetCarteMereFonctions\project\Trames.c
 CHERCHER_DONNNEES_CABLES   0x0085ba    program     extern C:\CMS2Luc\ProjetsNettoyesCMSGit\ProjetCarteMereFonctions\project\Trames.c
            SERIALISATION   0x008a02    program     extern C:\CMS2Luc\ProjetsNettoyesCMSGit\ProjetCarteMereFonctions\project\Trames.c
                      SDW   0x008b0c    program     extern C:\CMS2Luc\ProjetsNettoyesCMSGit\ProjetCarteMereFonctions\project\Trames.c
             __tmplbl_269   0x008c22    program     static                          
             __tmplbl_270   0x008c22    program     static                          
             __tmplbl_261   0x009714    program     static                          
       IDENTIF_TYPE_CARTE   0x00975e    program     extern C:\CMS2Luc\ProjetsNettoyesCMSGit\ProjetCarteMereFonctions\project\Trames.c
                    SDWBN   0x009d42    program     extern C:\CMS2Luc\ProjetsNettoyesCMSGit\ProjetCarteMereFonctions\project\Trames.c
                    SDRBN   0x009ea8    program     extern C:\CMS2Luc\ProjetsNettoyesCMSGit\ProjetCarteMereFonctions\project\Trames.c
     REMISE_EN_FORME_PAGE   0x00a1bc    program     extern C:\CMS2Luc\ProjetsNettoyesCMSGit\ProjetCarteMereFonctions\project\Trames.c
             __tmplbl_317   0x00b968    program     static                          
             __tmplbl_316   0x00b968    program     static                          
             __tmplbl_315   0x00b968    program     static                          
             __tmplbl_314   0x00b968    program     static                          
             __tmplbl_318   0x00b968    program     static                          
             __tmplbl_319   0x00b968    program     static                          
             __tmplbl_320   0x00b968    program     static                          
      envoyer_TRAME_PICSD   0x00b9a6    program     extern C:\CMS2Luc\ProjetsNettoyesCMSGit\ProjetCarteMereFonctions\project\Trames.c
          TROUVER_ROBINET   0x00c396    program     extern C:\CMS2Luc\ProjetsNettoyesCMSGit\ProjetCarteMereFonctions\project\Trames.c
                    inter   0x00c6c2    program     extern C:\CMS2Luc\ProjetsNettoyesCMSGit\ProjetCarteMereFonctions\project\CMSModifV1Nettoye.c
                     main   0x00c784    program     extern C:\CMS2Luc\ProjetsNettoyesCMSGit\ProjetCarteMereFonctions\project\CMSModifV1Nettoye.c
             __tmplbl_496   0x00cd6c    program     static                          
             __tmplbl_447   0x00dade    program     static                          
        ENVOIE_DES_TRAMES   0x00dff6    program     extern C:\CMS2Luc\ProjetsNettoyesCMSGit\ProjetCarteMereFonctions\project\CMSModifV1Nettoye.c
             __tmplbl_504   0x00f26c    program     static                          
             __tmplbl_503   0x00f3da    program     static                          
             __tmplbl_502   0x00f54a    program     static                          
             __tmplbl_501   0x00f8ce    program     static                          
             __tmplbl_500   0x00fc00    program     static                          
             __tmplbl_499   0x00fdb0    program     static                          
             __tmplbl_498   0x00ff86    program     static                          
             __tmplbl_497   0x0100fa    program     static                          
             __tmplbl_509   0x010676    program     static                          
             __tmplbl_510   0x010676    program     static                          
             __tmplbl_511   0x010676    program     static                          
             __tmplbl_512   0x010676    program     static                          
             __tmplbl_513   0x010676    program     static                          
             __tmplbl_514   0x010676    program     static                          
             __tmplbl_515   0x010676    program     static                          
             __tmplbl_517   0x010676    program     static                          
             __tmplbl_528   0x010676    program     static                          
             __tmplbl_529   0x010676    program     static                          
             __tmplbl_530   0x010676    program     static                          
             __tmplbl_532   0x010676    program     static                          
             __tmplbl_533   0x010676    program     static                          
             __tmplbl_534   0x010676    program     static                          
             __tmplbl_540   0x010676    program     static                          
             __tmplbl_536   0x010676    program     static                          
             __tmplbl_537   0x010676    program     static                          
  RECUPERATION_DES_TRAMES   0x01068a    program     extern C:\CMS2Luc\ProjetsNettoyesCMSGit\ProjetCarteMereFonctions\project\CMSModifV1Nettoye.c
             __tmplbl_574   0x0111ba    program     static                          
             __tmplbl_573   0x01168a    program     static                          
             __tmplbl_572   0x01195a    program     static                          
             __tmplbl_571   0x011a8e    program     static                          
             __tmplbl_635   0x011cbe    program     static                          
             __tmplbl_634   0x011d16    program     static                          
             __tmplbl_632   0x011d16    program     static                          
             __tmplbl_591   0x01256c    program     static                          
             __tmplbl_570   0x012572    program     static                          
             __tmplbl_569   0x01289c    program     static                          
             __tmplbl_568   0x012ac6    program     static                          
             __tmplbl_567   0x012c9c    program     static                          
             __tmplbl_600   0x012f5c    program     static                          
             __tmplbl_601   0x012f6e    program     static                          
             __tmplbl_599   0x012f7c    program     static                          
             __tmplbl_604   0x012f7c    program     static                          
             __tmplbl_605   0x012f7c    program     static                          
             __tmplbl_566   0x012f80    program     static                          
             __tmplbl_638   0x0134e6    program     static                          
             __tmplbl_637   0x0134e6    program     static                          
             __tmplbl_565   0x0134ec    program     static                          
             __tmplbl_594   0x0137f4    program     static                          
             __tmplbl_564   0x0137fa    program     static                          
             __tmplbl_596   0x013812    program     static                          
             __tmplbl_590   0x013812    program     static                          
             __tmplbl_562   0x01381a    program     static                          
             __tmplbl_561   0x013c46    program     static                          
             __tmplbl_560   0x013d2a    program     static                          
             __tmplbl_559   0x013d32    program     static                          
             __tmplbl_558   0x013ea0    program     static                          
             __tmplbl_597   0x013ee2    program     static                          
             __tmplbl_557   0x013eea    program     static                          
             __tmplbl_556   0x013f08    program     static                          
             __tmplbl_555   0x0141ee    program     static                          
             __tmplbl_554   0x014348    program     static                          
             __tmplbl_584   0x014b0a    program     static                          
             __tmplbl_589   0x014b0a    program     static                          
             __tmplbl_664   0x014b0a    program     static                          
             __tmplbl_665   0x014b1c    program     static                          
             __tmplbl_588   0x014b26    program     static                          
             __tmplbl_593   0x014b2a    program     static                          
             __tmplbl_598   0x014b2a    program     static                          
             __tmplbl_636   0x014b2a    program     static                          
             __tmplbl_641   0x014b2a    program     static                          
             __tmplbl_653   0x014b2a    program     static                          
             __tmplbl_658   0x014b2a    program     static                          
             __tmplbl_582   0x014b2e    program     static                          
             __tmplbl_583   0x014b2e    program     static                          
             __tmplbl_663   0x014b36    program     static                          
             __tmplbl_563   0x014b38    program     static                          
             __tmplbl_585   0x014b38    program     static                          
             __tmplbl_586   0x014b38    program     static                          
             __tmplbl_587   0x014b38    program     static                          
             __tmplbl_666   0x014b38    program     static                          
             __tmplbl_659   0x014b38    program     static                          
             __tmplbl_662   0x014b38    program     static                          
      identificationINTER   0x014b4c    program     extern C:\CMS2Luc\ProjetsNettoyesCMSGit\ProjetCarteMereFonctions\project\CMSModifV1Nettoye.c
                IntToChar   0x0150a0    program     extern C:\CMS2Luc\ProjetsNettoyesCMSGit\ProjetCarteMereFonctions\project\InToChar.c
               IntToChar5   0x0156d6    program     extern C:\CMS2Luc\ProjetsNettoyesCMSGit\ProjetCarteMereFonctions\project\InToChar.c
               __tmplbl_5   0x015f2e    program     static                          
           ECRIRE_HORLOGE   0x015f8a    program     extern C:\CMS2Luc\ProjetsNettoyesCMSGit\ProjetCarteMereFonctions\project\HORLOGE.c
       envoyerHORLOGE_i2c   0x016062    program     extern C:\CMS2Luc\ProjetsNettoyesCMSGit\ProjetCarteMereFonctions\project\HORLOGE.c
             LIRE_HORLOGE   0x0160ac    program     extern C:\CMS2Luc\ProjetsNettoyesCMSGit\ProjetCarteMereFonctions\project\HORLOGE.c
           litHORLOGE_i2c   0x01612a    program     extern C:\CMS2Luc\ProjetsNettoyesCMSGit\ProjetCarteMereFonctions\project\HORLOGE.c
      creer_trame_horloge   0x01617e    program     extern C:\CMS2Luc\ProjetsNettoyesCMSGit\ProjetCarteMereFonctions\project\HORLOGE.c
     entrer_trame_horloge   0x0165ae    program     extern C:\CMS2Luc\ProjetsNettoyesCMSGit\ProjetCarteMereFonctions\project\HORLOGE.c
             lire_horloge   0x0167fa    program     extern C:\CMS2Luc\ProjetsNettoyesCMSGit\ProjetCarteMereFonctions\project\HORLOGE.c
      reglerhorlogeautres   0x01694e    program     extern C:\CMS2Luc\ProjetsNettoyesCMSGit\ProjetCarteMereFonctions\project\HORLOGE.c
     CONTROLE_CHARGE_BATT   0x016c6c    program     extern C:\CMS2Luc\ProjetsNettoyesCMSGit\ProjetCarteMereFonctions\project\Tension.c
      MESURE_DES_TENSIONS   0x016d36    program     extern C:\CMS2Luc\ProjetsNettoyesCMSGit\ProjetCarteMereFonctions\project\Tension.c
                  AVERAGE   0x01713c    program     extern C:\CMS2Luc\ProjetsNettoyesCMSGit\ProjetCarteMereFonctions\project\Tension.c
                      CAN   0x0173e0    program     extern C:\CMS2Luc\ProjetsNettoyesCMSGit\ProjetCarteMereFonctions\project\Tension.c
        GROUPE_EN_MEMOIRE   0x0174e2    program     extern C:\CMS2Luc\ProjetsNettoyesCMSGit\ProjetCarteMereFonctions\project\Memoire.c
  METTRE_EN_MEMOIRE_LISTE   0x01758a    program     extern C:\CMS2Luc\ProjetsNettoyesCMSGit\ProjetCarteMereFonctions\project\Memoire.c
        calcul_addmemoire   0x0176b8    program     extern C:\CMS2Luc\ProjetsNettoyesCMSGit\ProjetCarteMereFonctions\project\Memoire.c
            choix_memoire   0x017a7a    program     extern C:\CMS2Luc\ProjetsNettoyesCMSGit\ProjetCarteMereFonctions\project\Memoire.c
                 FLO0832U   0x017c48    program     extern E:\3.46\pic18-lt\cxx-framework\src\traditional\math\cast08FP.asm
                 FLO0832S   0x017c4c    program     extern E:\3.46\pic18-lt\cxx-framework\src\traditional\math\cast08FP.asm
                jI2F08Beg   0x017c56    program     static E:\3.46\pic18-lt\cxx-framework\src\traditional\math\cast08FP.asm
                 FLO1632U   0x017c6a    program     extern E:\3.46\pic18-lt\cxx-framework\src\traditional\math\cast16FP.asm
                 FLO1632S   0x017c6e    program     extern E:\3.46\pic18-lt\cxx-framework\src\traditional\math\cast16FP.asm
                jI2F16Beg   0x017c7e    program     static E:\3.46\pic18-lt\cxx-framework\src\traditional\math\cast16FP.asm
                    FPS32   0x017c94    program     extern E:\3.46\pic18-lt\cxx-framework\src\traditional\math\addFP.asm
                    FPA32   0x017c96    program     extern E:\3.46\pic18-lt\cxx-framework\src\traditional\math\addFP.asm
                jBANotInf   0x017cb4    program     static E:\3.46\pic18-lt\cxx-framework\src\traditional\math\addFP.asm
                 jANotInf   0x017cbe    program     static E:\3.46\pic18-lt\cxx-framework\src\traditional\math\addFP.asm
                 jBNotInf   0x017ccc    program     static E:\3.46\pic18-lt\cxx-framework\src\traditional\math\addFP.asm
            jDifOrPosSign   0x017ce0    program     static E:\3.46\pic18-lt\cxx-framework\src\traditional\math\addFP.asm
             jNotBothZero   0x017ce4    program     static E:\3.46\pic18-lt\cxx-framework\src\traditional\math\addFP.asm
                 jAltBexp   0x017d10    program     static E:\3.46\pic18-lt\cxx-framework\src\traditional\math\addFP.asm
              jAandWsetup   0x017d22    program     static E:\3.46\pic18-lt\cxx-framework\src\traditional\math\addFP.asm
                 jANotNeg   0x017d52    program     static E:\3.46\pic18-lt\cxx-framework\src\traditional\math\addFP.asm
                 jWNotNeg   0x017d66    program     static E:\3.46\pic18-lt\cxx-framework\src\traditional\math\addFP.asm
               jShiftLoop   0x017d6c    program     static E:\3.46\pic18-lt\cxx-framework\src\traditional\math\addFP.asm
               jShiftDone   0x017d7a    program     static E:\3.46\pic18-lt\cxx-framework\src\traditional\math\addFP.asm
                jSignDone   0x017daa    program     static E:\3.46\pic18-lt\cxx-framework\src\traditional\math\addFP.asm
               jFinalSign   0x017dba    program     static E:\3.46\pic18-lt\cxx-framework\src\traditional\math\addFP.asm
                    FPD32   0x017dc2    program     extern E:\3.46\pic18-lt\cxx-framework\src\traditional\math\divFP.asm
                 jANotInf   0x017de0    program     static E:\3.46\pic18-lt\cxx-framework\src\traditional\math\divFP.asm
              jSignedZero   0x017dea    program     static E:\3.46\pic18-lt\cxx-framework\src\traditional\math\divFP.asm
                jANotZero   0x017df4    program     static E:\3.46\pic18-lt\cxx-framework\src\traditional\math\divFP.asm
                    jLoop   0x017e1c    program     static E:\3.46\pic18-lt\cxx-framework\src\traditional\math\divFP.asm
                jNoAdjust   0x017e40    program     static E:\3.46\pic18-lt\cxx-framework\src\traditional\math\divFP.asm
                    jNext   0x017e42    program     static E:\3.46\pic18-lt\cxx-framework\src\traditional\math\divFP.asm
                    FPM32   0x017e68    program     extern E:\3.46\pic18-lt\cxx-framework\src\traditional\math\mulFP.asm
                 jANotInf   0x017e86    program     static E:\3.46\pic18-lt\cxx-framework\src\traditional\math\mulFP.asm
              jBothFinite   0x017e94    program     static E:\3.46\pic18-lt\cxx-framework\src\traditional\math\mulFP.asm
                jHaveZero   0x017e9c    program     static E:\3.46\pic18-lt\cxx-framework\src\traditional\math\mulFP.asm
             jBothNotZero   0x017ea0    program     static E:\3.46\pic18-lt\cxx-framework\src\traditional\math\mulFP.asm
                 FXD0808S   0x017f42    program     extern E:\3.46\pic18-lt\cxx-framework\src\traditional\math\fxd0808s.asm
                  DA0808S   0x017f4e    program     static E:\3.46\pic18-lt\cxx-framework\src\traditional\math\fxd0808s.asm
                   D0808S   0x017f58    program     static E:\3.46\pic18-lt\cxx-framework\src\traditional\math\fxd0808s.asm
                 D0808SOK   0x017f62    program     static E:\3.46\pic18-lt\cxx-framework\src\traditional\math\fxd0808s.asm
                D0808SNEG   0x017f66    program     static E:\3.46\pic18-lt\cxx-framework\src\traditional\math\fxd0808s.asm
                  D0808SX   0x017f6c    program     static E:\3.46\pic18-lt\cxx-framework\src\traditional\math\fxd0808s.asm
                 FXD1616S   0x017f76    program     extern E:\3.46\pic18-lt\cxx-framework\src\traditional\math\fxd1616s.asm
                  DA1616S   0x017f88    program     static E:\3.46\pic18-lt\cxx-framework\src\traditional\math\fxd1616s.asm
                   D1616S   0x017f98    program     static E:\3.46\pic18-lt\cxx-framework\src\traditional\math\fxd1616s.asm
                 D1616SOK   0x017fa2    program     static E:\3.46\pic18-lt\cxx-framework\src\traditional\math\fxd1616s.asm
                D1616SNEG   0x017fa6    program     static E:\3.46\pic18-lt\cxx-framework\src\traditional\math\fxd1616s.asm
                  D1616SX   0x017fb8    program     static E:\3.46\pic18-lt\cxx-framework\src\traditional\math\fxd1616s.asm
                 FXM1616S   0x017fc2    program     extern E:\3.46\pic18-lt\cxx-framework\src\traditional\math\fxm1616s.asm
               TSIGN1616A   0x01800e    program     static E:\3.46\pic18-lt\cxx-framework\src\traditional\math\fxm1616s.asm
                 FXM1616U   0x01801c    program     extern E:\3.46\pic18-lt\cxx-framework\src\traditional\math\fxm1616u.asm
                  INT3208   0x018058    program     extern E:\3.46\pic18-lt\cxx-framework\src\traditional\math\castFP08.asm
                     jMax   0x018068    program     static E:\3.46\pic18-lt\cxx-framework\src\traditional\math\castFP08.asm
                  jMaxPos   0x01806c    program     static E:\3.46\pic18-lt\cxx-framework\src\traditional\math\castFP08.asm
                  jMaxNeg   0x018072    program     static E:\3.46\pic18-lt\cxx-framework\src\traditional\math\castFP08.asm
                    jZero   0x018078    program     static E:\3.46\pic18-lt\cxx-framework\src\traditional\math\castFP08.asm
                  jNotInf   0x01807c    program     static E:\3.46\pic18-lt\cxx-framework\src\traditional\math\castFP08.asm
                    jLoop   0x01808c    program     static E:\3.46\pic18-lt\cxx-framework\src\traditional\math\castFP08.asm
                jLoopExit   0x01809a    program     static E:\3.46\pic18-lt\cxx-framework\src\traditional\math\castFP08.asm
                    jExit   0x0180a4    program     static E:\3.46\pic18-lt\cxx-framework\src\traditional\math\castFP08.asm
                  TAGTB32   0x0180a6    program     extern E:\3.46\pic18-lt\cxx-framework\src\traditional\math\gtFP.asm
              __FpCompare   0x0180b8    program     extern E:\3.46\pic18-lt\cxx-framework\src\traditional\math\compFP.asm
             jBothNotZero   0x0180d6    program     static E:\3.46\pic18-lt\cxx-framework\src\traditional\math\compFP.asm
                 jSignsEQ   0x0180da    program     static E:\3.46\pic18-lt\cxx-framework\src\traditional\math\compFP.asm
                      jEQ   0x0180f2    program     static E:\3.46\pic18-lt\cxx-framework\src\traditional\math\compFP.asm
                      jNE   0x0180f6    program     static E:\3.46\pic18-lt\cxx-framework\src\traditional\math\compFP.asm
                    jExch   0x0180fe    program     static E:\3.46\pic18-lt\cxx-framework\src\traditional\math\compFP.asm
                  jNoExch   0x01811e    program     static E:\3.46\pic18-lt\cxx-framework\src\traditional\math\compFP.asm
                   jFinal   0x018128    program     static E:\3.46\pic18-lt\cxx-framework\src\traditional\math\compFP.asm
                  jAisNeg   0x018134    program     static E:\3.46\pic18-lt\cxx-framework\src\traditional\math\compFP.asm
                   jShift   0x01813a    program     static E:\3.46\pic18-lt\cxx-framework\src\traditional\math\compFP.asm
                   jExpEQ   0x018144    program     static E:\3.46\pic18-lt\cxx-framework\src\traditional\math\compFP.asm
                  jRotate   0x018150    program     static E:\3.46\pic18-lt\cxx-framework\src\traditional\math\compFP.asm
            __FpReturnNaN   0x018162    program     extern E:\3.46\pic18-lt\cxx-framework\src\traditional\math\packFP.asm
                 __FpExit   0x01816e    program     extern E:\3.46\pic18-lt\cxx-framework\src\traditional\math\packFP.asm
        __FpReturnSignInf   0x018170    program     extern E:\3.46\pic18-lt\cxx-framework\src\traditional\math\packFP.asm
         __FpReturnNegInf   0x018174    program     extern E:\3.46\pic18-lt\cxx-framework\src\traditional\math\packFP.asm
         __FpReturnPosInf   0x01817a    program     extern E:\3.46\pic18-lt\cxx-framework\src\traditional\math\packFP.asm
           jReturnPosInf0   0x01817e    program     static E:\3.46\pic18-lt\cxx-framework\src\traditional\math\packFP.asm
               jZero1and2   0x018182    program     static E:\3.46\pic18-lt\cxx-framework\src\traditional\math\packFP.asm
       __FpReturnSignZero   0x018188    program     extern E:\3.46\pic18-lt\cxx-framework\src\traditional\math\packFP.asm
        __FpReturnNegZero   0x01818c    program     extern E:\3.46\pic18-lt\cxx-framework\src\traditional\math\packFP.asm
        __FpReturnPosZero   0x018194    program     extern E:\3.46\pic18-lt\cxx-framework\src\traditional\math\packFP.asm
                 __FpPack   0x01819a    program     extern E:\3.46\pic18-lt\cxx-framework\src\traditional\math\packFP.asm
                  jPkLoop   0x0181a8    program     static E:\3.46\pic18-lt\cxx-framework\src\traditional\math\packFP.asm
             jPkShiftDone   0x0181c4    program     static E:\3.46\pic18-lt\cxx-framework\src\traditional\math\packFP.asm
               jPkRoundIt   0x0181da    program     static E:\3.46\pic18-lt\cxx-framework\src\traditional\math\packFP.asm
              __FpReturnW   0x0181f2    program     extern E:\3.46\pic18-lt\cxx-framework\src\traditional\math\packFP.asm
             jPkRoundDone   0x0181f2    program     static E:\3.46\pic18-lt\cxx-framework\src\traditional\math\packFP.asm
              __FpUnPackA   0x018212    program     extern E:\3.46\pic18-lt\cxx-framework\src\traditional\math\UnpackFP.asm
                  jUnpkA1   0x01821c    program     static E:\3.46\pic18-lt\cxx-framework\src\traditional\math\UnpackFP.asm
                 jUnpkANZ   0x01822a    program     static E:\3.46\pic18-lt\cxx-framework\src\traditional\math\UnpackFP.asm
                  jUnpkA2   0x018234    program     static E:\3.46\pic18-lt\cxx-framework\src\traditional\math\UnpackFP.asm
                 jUnpkNaN   0x01823e    program     static E:\3.46\pic18-lt\cxx-framework\src\traditional\math\UnpackFP.asm
              __FpUnPackB   0x018242    program     extern E:\3.46\pic18-lt\cxx-framework\src\traditional\math\UnpackFP.asm
                  jUnpkB1   0x01824c    program     static E:\3.46\pic18-lt\cxx-framework\src\traditional\math\UnpackFP.asm
                 jUnpkBNZ   0x01825a    program     static E:\3.46\pic18-lt\cxx-framework\src\traditional\math\UnpackFP.asm
                  jUnpkB2   0x018264    program     static E:\3.46\pic18-lt\cxx-framework\src\traditional\math\UnpackFP.asm
              LIRE_EEPROM   0x01826e    program     extern C:\CMS2Luc\ProjetsNettoyesCMSGit\ProjetCarteMereFonctions\project\Eeprom.c
        ECRIRE_EEPROMBYTE   0x0184ac    program     extern C:\CMS2Luc\ProjetsNettoyesCMSGit\ProjetCarteMereFonctions\project\Eeprom.c
         pic_eeprom_write   0x0186bc    program     extern C:\CMS2Luc\ProjetsNettoyesCMSGit\ProjetCarteMereFonctions\project\Eeprom.c
        ___while_lbl00072   0x0186e0    program     static                          
        ___while_lbl00073   0x0186e4    program     static                          
       ___return_lbl00071   0x0186e8    program     static                          
          pic_eeprom_read   0x0186f0    program     extern C:\CMS2Luc\ProjetsNettoyesCMSGit\ProjetCarteMereFonctions\project\Eeprom.c
             putstringI2C   0x018712    program     extern C:\CMS2Luc\ProjetsNettoyesCMSGit\ProjetCarteMereFonctions\project\Eeprom.c
               calcul_CRC   0x0187d2    program     extern C:\CMS2Luc\ProjetsNettoyesCMSGit\ProjetCarteMereFonctions\project\CRC.c
             controle_CRC   0x01888a    program     extern C:\CMS2Luc\ProjetsNettoyesCMSGit\ProjetCarteMereFonctions\project\CRC.c
                CRC_verif   0x01890a    program     extern C:\CMS2Luc\ProjetsNettoyesCMSGit\ProjetCarteMereFonctions\project\CRC.c
                    CRC16   0x018a5a    program     extern C:\CMS2Luc\ProjetsNettoyesCMSGit\ProjetCarteMereFonctions\project\CRC.c
               Init_RS485   0x018b56    program     extern C:\CMS2Luc\ProjetsNettoyesCMSGit\ProjetCarteMereFonctions\project\RS485.c
           RECEVOIR_RS485   0x018bb6    program     extern C:\CMS2Luc\ProjetsNettoyesCMSGit\ProjetCarteMereFonctions\project\RS485.c
                    RS485   0x018cb8    program     extern C:\CMS2Luc\ProjetsNettoyesCMSGit\ProjetCarteMereFonctions\project\RS485.c
TRAMERECEPTIONRS485DONNEES   0x018ce0    program     extern C:\CMS2Luc\ProjetsNettoyesCMSGit\ProjetCarteMereFonctions\project\RS485.c
   TRAMEENVOIRS485DONNEES   0x018d8a    program     extern C:\CMS2Luc\ProjetsNettoyesCMSGit\ProjetCarteMereFonctions\project\RS485.c
                 delay_us   0x018e08    program     extern C:\CMS2Luc\ProjetsNettoyesCMSGit\ProjetCarteMereFonctions\project\Tempo.c
                 delay_ms   0x018e3c    program     extern C:\CMS2Luc\ProjetsNettoyesCMSGit\ProjetCarteMereFonctions\project\Tempo.c
                    TEMPO   0x018ec0    program     extern C:\CMS2Luc\ProjetsNettoyesCMSGit\ProjetCarteMereFonctions\project\Tempo.c
                WriteI2C1   0x018f44    program     extern E:\3.46\pic18-lt\cxx-framework\src\pmc_common\i2c\i2c1writ.c
                 getsI2C1   0x018fc4    program     extern E:\3.46\pic18-lt\cxx-framework\src\pmc_common\i2c\i2c1gets.c
            SPI_WriteByte   0x01903a    program     extern C:\CMS2Luc\ProjetsNettoyesCMSGit\ProjetCarteMereFonctions\project\SPI.c
                 init_spi   0x019058    program     extern C:\CMS2Luc\ProjetsNettoyesCMSGit\ProjetCarteMereFonctions\project\SPI.c
                  spi_low   0x019074    program     extern C:\CMS2Luc\ProjetsNettoyesCMSGit\ProjetCarteMereFonctions\project\SPI.c
                 OpenI2C1   0x01907a    program     extern E:\3.46\pic18-lt\cxx-framework\src\pmc_common\i2c\i2c1open.c
                   stopIO   0x0190b0    program     extern C:\CMS2Luc\ProjetsNettoyesCMSGit\ProjetCarteMereFonctions\project\IO.c
                 FXD1616U   0x0190e2    program     extern E:\3.46\pic18-lt\cxx-framework\src\traditional\math\fxd1616u.c
                     loop   0x0190ec    program     static                          
                  endloop   0x019108    program     static                          
       ___return_lbl00000   0x01910c    program     static                          
            __zero_memory   0x01910e    program     extern E:\3.46\pic18-lt\cxx-framework\src\traditional\proc\p18f8723.asm
                   loop_h   0x01911c    program     static E:\3.46\pic18-lt\cxx-framework\src\traditional\proc\p18f8723.asm
               zero_block   0x01911c    program     static E:\3.46\pic18-lt\cxx-framework\src\traditional\proc\p18f8723.asm
                compare_l   0x019124    program     static E:\3.46\pic18-lt\cxx-framework\src\traditional\proc\p18f8723.asm
                   loop_l   0x019126    program     static E:\3.46\pic18-lt\cxx-framework\src\traditional\proc\p18f8723.asm
                 FXD0808U   0x01912e    program     extern E:\3.46\pic18-lt\cxx-framework\src\traditional\math\fxd0808u.c
                     loop   0x019136    program     static                          
                  endloop   0x019144    program     static                          
       ___return_lbl00000   0x019148    program     static                          
                 ReadI2C1   0x01914a    program     extern E:\3.46\pic18-lt\cxx-framework\src\pmc_common\i2c\i2c1read.c
                 _startup   0x019164    program     extern E:\3.46\pic18-lt\cxx-framework\src\traditional\startup\c018.c
                     loop   0x019170    program     static                          
       ___return_lbl00001   0x01917a    program     static                          
                 Init_I2C   0x01917c    program     extern C:\CMS2Luc\ProjetsNettoyesCMSGit\ProjetCarteMereFonctions\project\I2C.c
                   __init   0x01918e    program     extern E:\3.46\pic18-lt\cxx-framework\src\traditional\stdclib\__init.c
               __config_0   0x300001    program     static C:\CMS2Luc\ProjetsNettoyesCMSGit\ProjetCarteMereFonctions\project\CMSModifV1Nettoye.c
               __config_1   0x300002    program     static C:\CMS2Luc\ProjetsNettoyesCMSGit\ProjetCarteMereFonctions\project\CMSModifV1Nettoye.c
               __config_2   0x300003    program     static C:\CMS2Luc\ProjetsNettoyesCMSGit\ProjetCarteMereFonctions\project\CMSModifV1Nettoye.c
               __config_3   0x300004    program     static C:\CMS2Luc\ProjetsNettoyesCMSGit\ProjetCarteMereFonctions\project\CMSModifV1Nettoye.c
               __config_4   0x300005    program     static C:\CMS2Luc\ProjetsNettoyesCMSGit\ProjetCarteMereFonctions\project\CMSModifV1Nettoye.c
               __config_5   0x300006    program     static C:\CMS2Luc\ProjetsNettoyesCMSGit\ProjetCarteMereFonctions\project\CMSModifV1Nettoye.c
               __config_6   0x300008    program     static C:\CMS2Luc\ProjetsNettoyesCMSGit\ProjetCarteMereFonctions\project\CMSModifV1Nettoye.c
               __config_7   0x300009    program     static C:\CMS2Luc\ProjetsNettoyesCMSGit\ProjetCarteMereFonctions\project\CMSModifV1Nettoye.c
               __config_8   0x30000a    program     static C:\CMS2Luc\ProjetsNettoyesCMSGit\ProjetCarteMereFonctions\project\CMSModifV1Nettoye.c
               __config_9   0x30000b    program     static C:\CMS2Luc\ProjetsNettoyesCMSGit\ProjetCarteMereFonctions\project\CMSModifV1Nettoye.c
              __config_10   0x30000c    program     static C:\CMS2Luc\ProjetsNettoyesCMSGit\ProjetCarteMereFonctions\project\CMSModifV1Nettoye.c
              __config_11   0x30000d    program     static C:\CMS2Luc\ProjetsNettoyesCMSGit\ProjetCarteMereFonctions\project\CMSModifV1Nettoye.c
                     SIGN   0x000000       data     extern E:\3.46\pic18-lt\cxx-framework\src\traditional\math\cmath18.asm
            __FPFLAGSbits   0x000001       data     extern E:\3.46\pic18-lt\cxx-framework\src\traditional\math\cmath18.asm
                __FPFLAGS   0x000001       data     extern E:\3.46\pic18-lt\cxx-framework\src\traditional\math\cmath18.asm
                  __REMB3   0x000002       data     extern E:\3.46\pic18-lt\cxx-framework\src\traditional\math\aarg.asm
                 __AARGB7   0x000002       data     extern E:\3.46\pic18-lt\cxx-framework\src\traditional\math\aarg.asm
                  __REMB2   0x000003       data     extern E:\3.46\pic18-lt\cxx-framework\src\traditional\math\aarg.asm
                 __AARGB6   0x000003       data     extern E:\3.46\pic18-lt\cxx-framework\src\traditional\math\aarg.asm
                 __AARGB5   0x000004       data     extern E:\3.46\pic18-lt\cxx-framework\src\traditional\math\aarg.asm
                  __REMB1   0x000004       data     extern E:\3.46\pic18-lt\cxx-framework\src\traditional\math\aarg.asm
                 __AARGB4   0x000005       data     extern E:\3.46\pic18-lt\cxx-framework\src\traditional\math\aarg.asm
                  __REMB0   0x000005       data     extern E:\3.46\pic18-lt\cxx-framework\src\traditional\math\aarg.asm
                 __AARGB3   0x000006       data     extern E:\3.46\pic18-lt\cxx-framework\src\traditional\math\aarg.asm
                 __AARGB2   0x000007       data     extern E:\3.46\pic18-lt\cxx-framework\src\traditional\math\aarg.asm
                 __AARGB1   0x000008       data     extern E:\3.46\pic18-lt\cxx-framework\src\traditional\math\aarg.asm
                 __AARGB0   0x000009       data     extern E:\3.46\pic18-lt\cxx-framework\src\traditional\math\aarg.asm
                   __AEXP   0x00000a       data     extern E:\3.46\pic18-lt\cxx-framework\src\traditional\math\aarg.asm
                 __BARGB3   0x00000b       data     extern E:\3.46\pic18-lt\cxx-framework\src\traditional\math\barg.asm
                 __BARGB2   0x00000c       data     extern E:\3.46\pic18-lt\cxx-framework\src\traditional\math\barg.asm
                 __BARGB1   0x00000d       data     extern E:\3.46\pic18-lt\cxx-framework\src\traditional\math\barg.asm
                 __BARGB0   0x00000e       data     extern E:\3.46\pic18-lt\cxx-framework\src\traditional\math\barg.asm
                   __BEXP   0x00000f       data     extern E:\3.46\pic18-lt\cxx-framework\src\traditional\math\barg.asm
                 __TEMPB3   0x000010       data     extern E:\3.46\pic18-lt\cxx-framework\src\traditional\math\temparg.asm
                 __TEMPB2   0x000011       data     extern E:\3.46\pic18-lt\cxx-framework\src\traditional\math\temparg.asm
                 __TEMPB1   0x000012       data     extern E:\3.46\pic18-lt\cxx-framework\src\traditional\math\temparg.asm
                   __TEMP   0x000013       data     extern E:\3.46\pic18-lt\cxx-framework\src\traditional\math\temparg.asm
                 __TEMPB0   0x000013       data     extern E:\3.46\pic18-lt\cxx-framework\src\traditional\math\temparg.asm
                  __tmp_0   0x000014       data     static C:\CMS2Luc\ProjetsNettoyesCMSGit\ProjetCarteMereFonctions\project\Trames.c
                  __tmp_0   0x000014       data     static C:\CMS2Luc\ProjetsNettoyesCMSGit\ProjetCarteMereFonctions\project\Tempo.c
                  __tmp_0   0x000014       data     static C:\CMS2Luc\ProjetsNettoyesCMSGit\ProjetCarteMereFonctions\project\CRC.c
                  __tmp_0   0x000014       data     static C:\CMS2Luc\ProjetsNettoyesCMSGit\ProjetCarteMereFonctions\project\Eeprom.c
                  __tmp_0   0x000014       data     static E:\3.46\pic18-lt\cxx-framework\src\pmc_common\i2c\i2c1writ.c
                  __tmp_0   0x000014       data     static C:\CMS2Luc\ProjetsNettoyesCMSGit\ProjetCarteMereFonctions\project\CMSModifV1Nettoye.c
                  __tmp_0   0x000014       data     static C:\CMS2Luc\ProjetsNettoyesCMSGit\ProjetCarteMereFonctions\project\InToChar.c
                  __tmp_0   0x000014       data     static C:\CMS2Luc\ProjetsNettoyesCMSGit\ProjetCarteMereFonctions\project\Tension.c
                  __tmp_0   0x000014       data     static C:\CMS2Luc\ProjetsNettoyesCMSGit\ProjetCarteMereFonctions\project\Memoire.c
                  __tmp_0   0x000014       data     static C:\CMS2Luc\ProjetsNettoyesCMSGit\ProjetCarteMereFonctions\project\HORLOGE.c
                  __tmp_0   0x000014       data     static C:\CMS2Luc\ProjetsNettoyesCMSGit\ProjetCarteMereFonctions\project\RS485.c
                 TRAMEOUT   0x000100       data     extern C:\CMS2Luc\ProjetsNettoyesCMSGit\ProjetCarteMereFonctions\project\CMSModifV1Nettoye.c
                  TRAMEIN   0x00017d       data     extern C:\CMS2Luc\ProjetsNettoyesCMSGit\ProjetCarteMereFonctions\project\CMSModifV1Nettoye.c
                  VOIECOD   0x000200       data     extern C:\CMS2Luc\ProjetsNettoyesCMSGit\ProjetCarteMereFonctions\project\CMSModifV1Nettoye.c
                     TYPE   0x000206       data     extern C:\CMS2Luc\ProjetsNettoyesCMSGit\ProjetCarteMereFonctions\project\CMSModifV1Nettoye.c
                     CMOD   0x000207       data     extern C:\CMS2Luc\ProjetsNettoyesCMSGit\ProjetCarteMereFonctions\project\CMSModifV1Nettoye.c
                     CCON   0x00020b       data     extern C:\CMS2Luc\ProjetsNettoyesCMSGit\ProjetCarteMereFonctions\project\CMSModifV1Nettoye.c
                     CREP   0x00020f       data     extern C:\CMS2Luc\ProjetsNettoyesCMSGit\ProjetCarteMereFonctions\project\CMSModifV1Nettoye.c
             CONSTITUTION   0x000213       data     extern C:\CMS2Luc\ProjetsNettoyesCMSGit\ProjetCarteMereFonctions\project\CMSModifV1Nettoye.c
              COMMENTAIRE   0x000220       data     extern C:\CMS2Luc\ProjetsNettoyesCMSGit\ProjetCarteMereFonctions\project\CMSModifV1Nettoye.c
                    CABLE   0x000234       data     extern C:\CMS2Luc\ProjetsNettoyesCMSGit\ProjetCarteMereFonctions\project\CMSModifV1Nettoye.c
                       JJ   0x000237       data     extern C:\CMS2Luc\ProjetsNettoyesCMSGit\ProjetCarteMereFonctions\project\CMSModifV1Nettoye.c
                       MM   0x000239       data     extern C:\CMS2Luc\ProjetsNettoyesCMSGit\ProjetCarteMereFonctions\project\CMSModifV1Nettoye.c
                       HH   0x00023b       data     extern C:\CMS2Luc\ProjetsNettoyesCMSGit\ProjetCarteMereFonctions\project\CMSModifV1Nettoye.c
                       mm   0x00023d       data     extern C:\CMS2Luc\ProjetsNettoyesCMSGit\ProjetCarteMereFonctions\project\CMSModifV1Nettoye.c
                       ii   0x00023f       data     extern C:\CMS2Luc\ProjetsNettoyesCMSGit\ProjetCarteMereFonctions\project\CMSModifV1Nettoye.c
                      COD   0x000240       data     extern C:\CMS2Luc\ProjetsNettoyesCMSGit\ProjetCarteMereFonctions\project\CMSModifV1Nettoye.c
                      POS   0x000242       data     extern C:\CMS2Luc\ProjetsNettoyesCMSGit\ProjetCarteMereFonctions\project\CMSModifV1Nettoye.c
                     iiii   0x000244       data     extern C:\CMS2Luc\ProjetsNettoyesCMSGit\ProjetCarteMereFonctions\project\CMSModifV1Nettoye.c
                 DISTANCE   0x000248       data     extern C:\CMS2Luc\ProjetsNettoyesCMSGit\ProjetCarteMereFonctions\project\CMSModifV1Nettoye.c
                     ETAT   0x00024d       data     extern C:\CMS2Luc\ProjetsNettoyesCMSGit\ProjetCarteMereFonctions\project\CMSModifV1Nettoye.c
                   VALEUR   0x00024f       data     extern C:\CMS2Luc\ProjetsNettoyesCMSGit\ProjetCarteMereFonctions\project\CMSModifV1Nettoye.c
                    SEUIL   0x000253       data     extern C:\CMS2Luc\ProjetsNettoyesCMSGit\ProjetCarteMereFonctions\project\CMSModifV1Nettoye.c
                TYPECARTE   0x000257       data     extern C:\CMS2Luc\ProjetsNettoyesCMSGit\ProjetCarteMereFonctions\project\CMSModifV1Nettoye.c
              cDebutTrame   0x00025c       data     extern C:\CMS2Luc\ProjetsNettoyesCMSGit\ProjetCarteMereFonctions\project\CMSModifV1Nettoye.c
                      ID1   0x00025d       data     extern C:\CMS2Luc\ProjetsNettoyesCMSGit\ProjetCarteMereFonctions\project\CMSModifV1Nettoye.c
                      ID2   0x00025f       data     extern C:\CMS2Luc\ProjetsNettoyesCMSGit\ProjetCarteMereFonctions\project\CMSModifV1Nettoye.c
                 FONCTION   0x000261       data     extern C:\CMS2Luc\ProjetsNettoyesCMSGit\ProjetCarteMereFonctions\project\CMSModifV1Nettoye.c
                      CRC   0x000264       data     extern C:\CMS2Luc\ProjetsNettoyesCMSGit\ProjetCarteMereFonctions\project\CMSModifV1Nettoye.c
                cFinTrame   0x000269       data     extern C:\CMS2Luc\ProjetsNettoyesCMSGit\ProjetCarteMereFonctions\project\CMSModifV1Nettoye.c
              TYPE_ERREUR   0x00026a       data     extern C:\CMS2Luc\ProjetsNettoyesCMSGit\ProjetCarteMereFonctions\project\CMSModifV1Nettoye.c
       INFORMATION_ERREUR   0x00026c       data     extern C:\CMS2Luc\ProjetsNettoyesCMSGit\ProjetCarteMereFonctions\project\CMSModifV1Nettoye.c
       NBRECAPTEURS_CABLE   0x000280       data     extern C:\CMS2Luc\ProjetsNettoyesCMSGit\ProjetCarteMereFonctions\project\CMSModifV1Nettoye.c
             PRIO_AUTO_IO   0x000281       data     extern C:\CMS2Luc\ProjetsNettoyesCMSGit\ProjetCarteMereFonctions\project\CMSModifV1Nettoye.c
                  HORLOGE   0x000282       data     extern C:\CMS2Luc\ProjetsNettoyesCMSGit\ProjetCarteMereFonctions\project\CMSModifV1Nettoye.c
        CAPTEUR_A_EFFACER   0x00028e       data     extern C:\CMS2Luc\ProjetsNettoyesCMSGit\ProjetCarteMereFonctions\project\CMSModifV1Nettoye.c
   DEMANDE_INFOS_CAPTEURS   0x000293       data     extern C:\CMS2Luc\ProjetsNettoyesCMSGit\ProjetCarteMereFonctions\project\CMSModifV1Nettoye.c
             OEIL_CAPTEUR   0x00029d       data     extern C:\CMS2Luc\ProjetsNettoyesCMSGit\ProjetCarteMereFonctions\project\CMSModifV1Nettoye.c
                     PAGE   0x0002a2       data     extern C:\CMS2Luc\ProjetsNettoyesCMSGit\ProjetCarteMereFonctions\project\CMSModifV1Nettoye.c
              INSTRUCTION   0x0002a8       data     extern C:\CMS2Luc\ProjetsNettoyesCMSGit\ProjetCarteMereFonctions\project\CMSModifV1Nettoye.c
               capt_exist   0x0002c1       data     extern C:\CMS2Luc\ProjetsNettoyesCMSGit\ProjetCarteMereFonctions\project\CMSModifV1Nettoye.c
                     VDD1   0x0002c2       data     extern C:\CMS2Luc\ProjetsNettoyesCMSGit\ProjetCarteMereFonctions\project\CMSModifV1Nettoye.c
                     VDD2   0x0002c6       data     extern C:\CMS2Luc\ProjetsNettoyesCMSGit\ProjetCarteMereFonctions\project\CMSModifV1Nettoye.c
                     VDD3   0x0002ca       data     extern C:\CMS2Luc\ProjetsNettoyesCMSGit\ProjetCarteMereFonctions\project\CMSModifV1Nettoye.c
                     VDD4   0x0002ce       data     extern C:\CMS2Luc\ProjetsNettoyesCMSGit\ProjetCarteMereFonctions\project\CMSModifV1Nettoye.c
                     VDD5   0x0002d2       data     extern C:\CMS2Luc\ProjetsNettoyesCMSGit\ProjetCarteMereFonctions\project\CMSModifV1Nettoye.c
                    Vtemp   0x0002d6       data     extern C:\CMS2Luc\ProjetsNettoyesCMSGit\ProjetCarteMereFonctions\project\CMSModifV1Nettoye.c
                     VDD6   0x0002da       data     extern C:\CMS2Luc\ProjetsNettoyesCMSGit\ProjetCarteMereFonctions\project\CMSModifV1Nettoye.c
                     VBAT   0x0002de       data     extern C:\CMS2Luc\ProjetsNettoyesCMSGit\ProjetCarteMereFonctions\project\CMSModifV1Nettoye.c
              NORECEPTION   0x0002e2       data     extern C:\CMS2Luc\ProjetsNettoyesCMSGit\ProjetCarteMereFonctions\project\CMSModifV1Nettoye.c
          pointeur_out_in   0x0002e3       data     extern C:\CMS2Luc\ProjetsNettoyesCMSGit\ProjetCarteMereFonctions\project\CMSModifV1Nettoye.c
                      tmp   0x0002e5       data     extern C:\CMS2Luc\ProjetsNettoyesCMSGit\ProjetCarteMereFonctions\project\CMSModifV1Nettoye.c
                     tmp2   0x0002e6       data     extern C:\CMS2Luc\ProjetsNettoyesCMSGit\ProjetCarteMereFonctions\project\CMSModifV1Nettoye.c
                     TMPI   0x0002e7       data     extern C:\CMS2Luc\ProjetsNettoyesCMSGit\ProjetCarteMereFonctions\project\CMSModifV1Nettoye.c
                 ENTREES1   0x0002e9       data     extern C:\CMS2Luc\ProjetsNettoyesCMSGit\ProjetCarteMereFonctions\project\CMSModifV1Nettoye.c
                 ENTREES2   0x0002ea       data     extern C:\CMS2Luc\ProjetsNettoyesCMSGit\ProjetCarteMereFonctions\project\CMSModifV1Nettoye.c
                    HEURE   0x0002eb       data     extern C:\CMS2Luc\ProjetsNettoyesCMSGit\ProjetCarteMereFonctions\project\CMSModifV1Nettoye.c
                   MINUTE   0x0002ec       data     extern C:\CMS2Luc\ProjetsNettoyesCMSGit\ProjetCarteMereFonctions\project\CMSModifV1Nettoye.c
                  SECONDE   0x0002ed       data     extern C:\CMS2Luc\ProjetsNettoyesCMSGit\ProjetCarteMereFonctions\project\CMSModifV1Nettoye.c
                     MOIS   0x0002ee       data     extern C:\CMS2Luc\ProjetsNettoyesCMSGit\ProjetCarteMereFonctions\project\CMSModifV1Nettoye.c
                     JOUR   0x0002ef       data     extern C:\CMS2Luc\ProjetsNettoyesCMSGit\ProjetCarteMereFonctions\project\CMSModifV1Nettoye.c
                    ANNEE   0x0002f0       data     extern C:\CMS2Luc\ProjetsNettoyesCMSGit\ProjetCarteMereFonctions\project\CMSModifV1Nettoye.c
                     DATE   0x0002f1       data     extern C:\CMS2Luc\ProjetsNettoyesCMSGit\ProjetCarteMereFonctions\project\CMSModifV1Nettoye.c
                      TMP   0x000300       data     extern C:\CMS2Luc\ProjetsNettoyesCMSGit\ProjetCarteMereFonctions\project\CMSModifV1Nettoye.c
              P_RESERVOIR   0x00037d       data     extern C:\CMS2Luc\ProjetsNettoyesCMSGit\ProjetCarteMereFonctions\project\CMSModifV1Nettoye.c
                 P_SORTIE   0x00038c       data     extern C:\CMS2Luc\ProjetsNettoyesCMSGit\ProjetCarteMereFonctions\project\CMSModifV1Nettoye.c
                P_SECOURS   0x00039b       data     extern C:\CMS2Luc\ProjetsNettoyesCMSGit\ProjetCarteMereFonctions\project\CMSModifV1Nettoye.c
              POINT_ROSEE   0x0003aa       data     extern C:\CMS2Luc\ProjetsNettoyesCMSGit\ProjetCarteMereFonctions\project\CMSModifV1Nettoye.c
             DEBIT_GLOBAL   0x0003b5       data     extern C:\CMS2Luc\ProjetsNettoyesCMSGit\ProjetCarteMereFonctions\project\CMSModifV1Nettoye.c
       TEMPS_CYCLE_MOTEUR   0x0003c0       data     extern C:\CMS2Luc\ProjetsNettoyesCMSGit\ProjetCarteMereFonctions\project\CMSModifV1Nettoye.c
             TEMPS_MOTEUR   0x0003cb       data     extern C:\CMS2Luc\ProjetsNettoyesCMSGit\ProjetCarteMereFonctions\project\CMSModifV1Nettoye.c
            PRESENCE_220V   0x0003da       data     extern C:\CMS2Luc\ProjetsNettoyesCMSGit\ProjetCarteMereFonctions\project\CMSModifV1Nettoye.c
             PRESENCE_48V   0x0003e0       data     extern C:\CMS2Luc\ProjetsNettoyesCMSGit\ProjetCarteMereFonctions\project\CMSModifV1Nettoye.c
                  DATAFIX   0x0003e6       data     extern C:\CMS2Luc\ProjetsNettoyesCMSGit\ProjetCarteMereFonctions\project\CMSModifV1Nettoye.c
                   SAVTAB   0x000f00       data     extern C:\CMS2Luc\ProjetsNettoyesCMSGit\ProjetCarteMereFonctions\project\CMSModifV1Nettoye.c
               calculBLOC   0x000f19       data     extern C:\CMS2Luc\ProjetsNettoyesCMSGit\ProjetCarteMereFonctions\project\CMSModifV1Nettoye.c
 FONCTION_ACTIVATION_AUTO   0x000f1b       data     extern C:\CMS2Luc\ProjetsNettoyesCMSGit\ProjetCarteMereFonctions\project\CMSModifV1Nettoye.c
             numdecarteRI   0x000f1c       data     extern C:\CMS2Luc\ProjetsNettoyesCMSGit\ProjetCarteMereFonctions\project\CMSModifV1Nettoye.c
         TROPDENONREPONSE   0x000f1d       data     extern C:\CMS2Luc\ProjetsNettoyesCMSGit\ProjetCarteMereFonctions\project\CMSModifV1Nettoye.c
                 CRC_ETAT   0x000f1e       data     extern C:\CMS2Luc\ProjetsNettoyesCMSGit\ProjetCarteMereFonctions\project\CMSModifV1Nettoye.c
                  ETAT_IO   0x000f1f       data     extern C:\CMS2Luc\ProjetsNettoyesCMSGit\ProjetCarteMereFonctions\project\CMSModifV1Nettoye.c
              FIRST_DEMAR   0x000f20       data     extern C:\CMS2Luc\ProjetsNettoyesCMSGit\ProjetCarteMereFonctions\project\CMSModifV1Nettoye.c
                MODERAPID   0x000f21       data     extern C:\CMS2Luc\ProjetsNettoyesCMSGit\ProjetCarteMereFonctions\project\CMSModifV1Nettoye.c
             TYPECOMMANDE   0x000f22       data     extern C:\CMS2Luc\ProjetsNettoyesCMSGit\ProjetCarteMereFonctions\project\CMSModifV1Nettoye.c
         temoinfinvoieZIZ   0x000f23       data     extern C:\CMS2Luc\ProjetsNettoyesCMSGit\ProjetCarteMereFonctions\project\CMSModifV1Nettoye.c
                IOTRAVAIL   0x000f24       data     extern C:\CMS2Luc\ProjetsNettoyesCMSGit\ProjetCarteMereFonctions\project\CMSModifV1Nettoye.c
                  PASDE_S   0x000f25       data     extern C:\CMS2Luc\ProjetsNettoyesCMSGit\ProjetCarteMereFonctions\project\CMSModifV1Nettoye.c
                   cycleN   0x000f26       data     extern C:\CMS2Luc\ProjetsNettoyesCMSGit\ProjetCarteMereFonctions\project\CMSModifV1Nettoye.c
             RESCRUTATION   0x000f27       data     extern C:\CMS2Luc\ProjetsNettoyesCMSGit\ProjetCarteMereFonctions\project\CMSModifV1Nettoye.c
              NUMEROCARTE   0x000f28       data     extern C:\CMS2Luc\ProjetsNettoyesCMSGit\ProjetCarteMereFonctions\project\CMSModifV1Nettoye.c
            NBREDEMANDEIO   0x000f29       data     extern C:\CMS2Luc\ProjetsNettoyesCMSGit\ProjetCarteMereFonctions\project\CMSModifV1Nettoye.c
          PRESENCEDEBITSD   0x000f2a       data     extern C:\CMS2Luc\ProjetsNettoyesCMSGit\ProjetCarteMereFonctions\project\CMSModifV1Nettoye.c
                  R1NOREP   0x000f2b       data     extern C:\CMS2Luc\ProjetsNettoyesCMSGit\ProjetCarteMereFonctions\project\CMSModifV1Nettoye.c
                  R2NOREP   0x000f2c       data     extern C:\CMS2Luc\ProjetsNettoyesCMSGit\ProjetCarteMereFonctions\project\CMSModifV1Nettoye.c
                  R3NOREP   0x000f2d       data     extern C:\CMS2Luc\ProjetsNettoyesCMSGit\ProjetCarteMereFonctions\project\CMSModifV1Nettoye.c
                  R4NOREP   0x000f2e       data     extern C:\CMS2Luc\ProjetsNettoyesCMSGit\ProjetCarteMereFonctions\project\CMSModifV1Nettoye.c
                  R5NOREP   0x000f2f       data     extern C:\CMS2Luc\ProjetsNettoyesCMSGit\ProjetCarteMereFonctions\project\CMSModifV1Nettoye.c
               UNRESETRI1   0x000f30       data     extern C:\CMS2Luc\ProjetsNettoyesCMSGit\ProjetCarteMereFonctions\project\CMSModifV1Nettoye.c
               UNRESETRI2   0x000f31       data     extern C:\CMS2Luc\ProjetsNettoyesCMSGit\ProjetCarteMereFonctions\project\CMSModifV1Nettoye.c
               UNRESETRI3   0x000f32       data     extern C:\CMS2Luc\ProjetsNettoyesCMSGit\ProjetCarteMereFonctions\project\CMSModifV1Nettoye.c
               UNRESETRI4   0x000f33       data     extern C:\CMS2Luc\ProjetsNettoyesCMSGit\ProjetCarteMereFonctions\project\CMSModifV1Nettoye.c
               UNRESETRI5   0x000f34       data     extern C:\CMS2Luc\ProjetsNettoyesCMSGit\ProjetCarteMereFonctions\project\CMSModifV1Nettoye.c
              MINIRESETRI   0x000f35       data     extern C:\CMS2Luc\ProjetsNettoyesCMSGit\ProjetCarteMereFonctions\project\CMSModifV1Nettoye.c
          TYPEDECARTEOEIL   0x000f36       data     extern C:\CMS2Luc\ProjetsNettoyesCMSGit\ProjetCarteMereFonctions\project\CMSModifV1Nettoye.c
             TIMEOUTCYCLE   0x000f37       data     extern C:\CMS2Luc\ProjetsNettoyesCMSGit\ProjetCarteMereFonctions\project\CMSModifV1Nettoye.c
        scrutationunevoie   0x000f39       data     extern C:\CMS2Luc\ProjetsNettoyesCMSGit\ProjetCarteMereFonctions\project\CMSModifV1Nettoye.c
   ETATZIZCRATIONAUTOMATE   0x000f3a       data     extern C:\CMS2Luc\ProjetsNettoyesCMSGit\ProjetCarteMereFonctions\project\CMSModifV1Nettoye.c
             mouchardINT0   0x000f3b       data     extern C:\CMS2Luc\ProjetsNettoyesCMSGit\ProjetCarteMereFonctions\project\CMSModifV1Nettoye.c
             DEMANDEZIGIO   0x000f3c       data     extern C:\CMS2Luc\ProjetsNettoyesCMSGit\ProjetCarteMereFonctions\project\CMSModifV1Nettoye.c
           resetheurefixe   0x000f3d       data     extern C:\CMS2Luc\ProjetsNettoyesCMSGit\ProjetCarteMereFonctions\project\CMSModifV1Nettoye.c
             SAVAUTOCYCLE   0x000f3e       data     extern C:\CMS2Luc\ProjetsNettoyesCMSGit\ProjetCarteMereFonctions\project\CMSModifV1Nettoye.c
                  MAXBITE   0x000f3f       data     extern C:\CMS2Luc\ProjetsNettoyesCMSGit\ProjetCarteMereFonctions\project\CMSModifV1Nettoye.c
                  MAJBLOC   0x000f40       data     extern C:\CMS2Luc\ProjetsNettoyesCMSGit\ProjetCarteMereFonctions\project\CMSModifV1Nettoye.c
             DEMANDEZPLIO   0x000f41       data     extern C:\CMS2Luc\ProjetsNettoyesCMSGit\ProjetCarteMereFonctions\project\CMSModifV1Nettoye.c
                    ERRMM   0x000f42       data     extern C:\CMS2Luc\ProjetsNettoyesCMSGit\ProjetCarteMereFonctions\project\CMSModifV1Nettoye.c
                     NBMM   0x000f43       data     extern C:\CMS2Luc\ProjetsNettoyesCMSGit\ProjetCarteMereFonctions\project\CMSModifV1Nettoye.c
                   FCYCLE   0x000f44       data     extern C:\CMS2Luc\ProjetsNettoyesCMSGit\ProjetCarteMereFonctions\project\CMSModifV1Nettoye.c
                TESTCYCLE   0x000f45       data     extern C:\CMS2Luc\ProjetsNettoyesCMSGit\ProjetCarteMereFonctions\project\CMSModifV1Nettoye.c
             SSP2CON2bits   0x000f62       data     extern E:\3.46\pic18-lt\cxx-framework\src\traditional\proc\p18f8723.asm
                 SSP2CON2   0x000f62       data     extern E:\3.46\pic18-lt\cxx-framework\src\traditional\proc\p18f8723.asm
             SSP2CON1bits   0x000f63       data     extern E:\3.46\pic18-lt\cxx-framework\src\traditional\proc\p18f8723.asm
                 SSP2CON1   0x000f63       data     extern E:\3.46\pic18-lt\cxx-framework\src\traditional\proc\p18f8723.asm
                 SSP2STAT   0x000f64       data     extern E:\3.46\pic18-lt\cxx-framework\src\traditional\proc\p18f8723.asm
             SSP2STATbits   0x000f64       data     extern E:\3.46\pic18-lt\cxx-framework\src\traditional\proc\p18f8723.asm
                  SSP2ADD   0x000f65       data     extern E:\3.46\pic18-lt\cxx-framework\src\traditional\proc\p18f8723.asm
                  SSP2BUF   0x000f66       data     extern E:\3.46\pic18-lt\cxx-framework\src\traditional\proc\p18f8723.asm
             ECCP2DELbits   0x000f67       data     extern E:\3.46\pic18-lt\cxx-framework\src\traditional\proc\p18f8723.asm
                 ECCP2DEL   0x000f67       data     extern E:\3.46\pic18-lt\cxx-framework\src\traditional\proc\p18f8723.asm
              ECCP2ASbits   0x000f68       data     extern E:\3.46\pic18-lt\cxx-framework\src\traditional\proc\p18f8723.asm
                  ECCP2AS   0x000f68       data     extern E:\3.46\pic18-lt\cxx-framework\src\traditional\proc\p18f8723.asm
                 ECCP3DEL   0x000f69       data     extern E:\3.46\pic18-lt\cxx-framework\src\traditional\proc\p18f8723.asm
             ECCP3DELbits   0x000f69       data     extern E:\3.46\pic18-lt\cxx-framework\src\traditional\proc\p18f8723.asm
                  ECCP3AS   0x000f6a       data     extern E:\3.46\pic18-lt\cxx-framework\src\traditional\proc\p18f8723.asm
              ECCP3ASbits   0x000f6a       data     extern E:\3.46\pic18-lt\cxx-framework\src\traditional\proc\p18f8723.asm
               RCSTA2bits   0x000f6b       data     extern E:\3.46\pic18-lt\cxx-framework\src\traditional\proc\p18f8723.asm
                   RCSTA2   0x000f6b       data     extern E:\3.46\pic18-lt\cxx-framework\src\traditional\proc\p18f8723.asm
               TXSTA2bits   0x000f6c       data     extern E:\3.46\pic18-lt\cxx-framework\src\traditional\proc\p18f8723.asm
                   TXSTA2   0x000f6c       data     extern E:\3.46\pic18-lt\cxx-framework\src\traditional\proc\p18f8723.asm
                   TXREG2   0x000f6d       data     extern E:\3.46\pic18-lt\cxx-framework\src\traditional\proc\p18f8723.asm
                   RCREG2   0x000f6e       data     extern E:\3.46\pic18-lt\cxx-framework\src\traditional\proc\p18f8723.asm
                   SPBRG2   0x000f6f       data     extern E:\3.46\pic18-lt\cxx-framework\src\traditional\proc\p18f8723.asm
                  CCP5CON   0x000f70       data     extern E:\3.46\pic18-lt\cxx-framework\src\traditional\proc\p18f8723.asm
              CCP5CONbits   0x000f70       data     extern E:\3.46\pic18-lt\cxx-framework\src\traditional\proc\p18f8723.asm
                   CCPR5L   0x000f71       data     extern E:\3.46\pic18-lt\cxx-framework\src\traditional\proc\p18f8723.asm
                    CCPR5   0x000f71       data     extern E:\3.46\pic18-lt\cxx-framework\src\traditional\proc\p18f8723.asm
                   CCPR5H   0x000f72       data     extern E:\3.46\pic18-lt\cxx-framework\src\traditional\proc\p18f8723.asm
                  CCP4CON   0x000f73       data     extern E:\3.46\pic18-lt\cxx-framework\src\traditional\proc\p18f8723.asm
              CCP4CONbits   0x000f73       data     extern E:\3.46\pic18-lt\cxx-framework\src\traditional\proc\p18f8723.asm
                   CCPR4L   0x000f74       data     extern E:\3.46\pic18-lt\cxx-framework\src\traditional\proc\p18f8723.asm
                    CCPR4   0x000f74       data     extern E:\3.46\pic18-lt\cxx-framework\src\traditional\proc\p18f8723.asm
                   CCPR4H   0x000f75       data     extern E:\3.46\pic18-lt\cxx-framework\src\traditional\proc\p18f8723.asm
                    T4CON   0x000f76       data     extern E:\3.46\pic18-lt\cxx-framework\src\traditional\proc\p18f8723.asm
                T4CONbits   0x000f76       data     extern E:\3.46\pic18-lt\cxx-framework\src\traditional\proc\p18f8723.asm
                      PR4   0x000f77       data     extern E:\3.46\pic18-lt\cxx-framework\src\traditional\proc\p18f8723.asm
                     TMR4   0x000f78       data     extern E:\3.46\pic18-lt\cxx-framework\src\traditional\proc\p18f8723.asm
             ECCP1DELbits   0x000f79       data     extern E:\3.46\pic18-lt\cxx-framework\src\traditional\proc\p18f8723.asm
                 ECCP1DEL   0x000f79       data     extern E:\3.46\pic18-lt\cxx-framework\src\traditional\proc\p18f8723.asm
             BAUDCON2bits   0x000f7c       data     extern E:\3.46\pic18-lt\cxx-framework\src\traditional\proc\p18f8723.asm
                 BAUDCON2   0x000f7c       data     extern E:\3.46\pic18-lt\cxx-framework\src\traditional\proc\p18f8723.asm
                  SPBRGH2   0x000f7d       data     extern E:\3.46\pic18-lt\cxx-framework\src\traditional\proc\p18f8723.asm
              BAUDCONbits   0x000f7e       data     extern E:\3.46\pic18-lt\cxx-framework\src\traditional\proc\p18f8723.asm
             BAUDCON1bits   0x000f7e       data     extern E:\3.46\pic18-lt\cxx-framework\src\traditional\proc\p18f8723.asm
                 BAUDCON1   0x000f7e       data     extern E:\3.46\pic18-lt\cxx-framework\src\traditional\proc\p18f8723.asm
                  BAUDCON   0x000f7e       data     extern E:\3.46\pic18-lt\cxx-framework\src\traditional\proc\p18f8723.asm
                  SPBRGH1   0x000f7f       data     extern E:\3.46\pic18-lt\cxx-framework\src\traditional\proc\p18f8723.asm
                   SPBRGH   0x000f7f       data     extern E:\3.46\pic18-lt\cxx-framework\src\traditional\proc\p18f8723.asm
                PORTAbits   0x000f80       data     extern E:\3.46\pic18-lt\cxx-framework\src\traditional\proc\p18f8723.asm
                    PORTA   0x000f80       data     extern E:\3.46\pic18-lt\cxx-framework\src\traditional\proc\p18f8723.asm
                PORTBbits   0x000f81       data     extern E:\3.46\pic18-lt\cxx-framework\src\traditional\proc\p18f8723.asm
                    PORTB   0x000f81       data     extern E:\3.46\pic18-lt\cxx-framework\src\traditional\proc\p18f8723.asm
                PORTCbits   0x000f82       data     extern E:\3.46\pic18-lt\cxx-framework\src\traditional\proc\p18f8723.asm
                    PORTC   0x000f82       data     extern E:\3.46\pic18-lt\cxx-framework\src\traditional\proc\p18f8723.asm
                PORTDbits   0x000f83       data     extern E:\3.46\pic18-lt\cxx-framework\src\traditional\proc\p18f8723.asm
                    PORTD   0x000f83       data     extern E:\3.46\pic18-lt\cxx-framework\src\traditional\proc\p18f8723.asm
                    PORTE   0x000f84       data     extern E:\3.46\pic18-lt\cxx-framework\src\traditional\proc\p18f8723.asm
                PORTEbits   0x000f84       data     extern E:\3.46\pic18-lt\cxx-framework\src\traditional\proc\p18f8723.asm
                    PORTF   0x000f85       data     extern E:\3.46\pic18-lt\cxx-framework\src\traditional\proc\p18f8723.asm
                PORTFbits   0x000f85       data     extern E:\3.46\pic18-lt\cxx-framework\src\traditional\proc\p18f8723.asm
                    PORTG   0x000f86       data     extern E:\3.46\pic18-lt\cxx-framework\src\traditional\proc\p18f8723.asm
                PORTGbits   0x000f86       data     extern E:\3.46\pic18-lt\cxx-framework\src\traditional\proc\p18f8723.asm
                PORTHbits   0x000f87       data     extern E:\3.46\pic18-lt\cxx-framework\src\traditional\proc\p18f8723.asm
                    PORTH   0x000f87       data     extern E:\3.46\pic18-lt\cxx-framework\src\traditional\proc\p18f8723.asm
                PORTJbits   0x000f88       data     extern E:\3.46\pic18-lt\cxx-framework\src\traditional\proc\p18f8723.asm
                    PORTJ   0x000f88       data     extern E:\3.46\pic18-lt\cxx-framework\src\traditional\proc\p18f8723.asm
                     LATA   0x000f89       data     extern E:\3.46\pic18-lt\cxx-framework\src\traditional\proc\p18f8723.asm
                 LATAbits   0x000f89       data     extern E:\3.46\pic18-lt\cxx-framework\src\traditional\proc\p18f8723.asm
                     LATB   0x000f8a       data     extern E:\3.46\pic18-lt\cxx-framework\src\traditional\proc\p18f8723.asm
                 LATBbits   0x000f8a       data     extern E:\3.46\pic18-lt\cxx-framework\src\traditional\proc\p18f8723.asm
                 LATCbits   0x000f8b       data     extern E:\3.46\pic18-lt\cxx-framework\src\traditional\proc\p18f8723.asm
                     LATC   0x000f8b       data     extern E:\3.46\pic18-lt\cxx-framework\src\traditional\proc\p18f8723.asm
                     LATD   0x000f8c       data     extern E:\3.46\pic18-lt\cxx-framework\src\traditional\proc\p18f8723.asm
                 LATDbits   0x000f8c       data     extern E:\3.46\pic18-lt\cxx-framework\src\traditional\proc\p18f8723.asm
                 LATEbits   0x000f8d       data     extern E:\3.46\pic18-lt\cxx-framework\src\traditional\proc\p18f8723.asm
                     LATE   0x000f8d       data     extern E:\3.46\pic18-lt\cxx-framework\src\traditional\proc\p18f8723.asm
                     LATF   0x000f8e       data     extern E:\3.46\pic18-lt\cxx-framework\src\traditional\proc\p18f8723.asm
                 LATFbits   0x000f8e       data     extern E:\3.46\pic18-lt\cxx-framework\src\traditional\proc\p18f8723.asm
                     LATG   0x000f8f       data     extern E:\3.46\pic18-lt\cxx-framework\src\traditional\proc\p18f8723.asm
                 LATGbits   0x000f8f       data     extern E:\3.46\pic18-lt\cxx-framework\src\traditional\proc\p18f8723.asm
                     LATH   0x000f90       data     extern E:\3.46\pic18-lt\cxx-framework\src\traditional\proc\p18f8723.asm
                 LATHbits   0x000f90       data     extern E:\3.46\pic18-lt\cxx-framework\src\traditional\proc\p18f8723.asm
                     LATJ   0x000f91       data     extern E:\3.46\pic18-lt\cxx-framework\src\traditional\proc\p18f8723.asm
                 LATJbits   0x000f91       data     extern E:\3.46\pic18-lt\cxx-framework\src\traditional\proc\p18f8723.asm
                    TRISA   0x000f92       data     extern E:\3.46\pic18-lt\cxx-framework\src\traditional\proc\p18f8723.asm
                TRISAbits   0x000f92       data     extern E:\3.46\pic18-lt\cxx-framework\src\traditional\proc\p18f8723.asm
                     DDRA   0x000f92       data     extern E:\3.46\pic18-lt\cxx-framework\src\traditional\proc\p18f8723.asm
                 DDRAbits   0x000f92       data     extern E:\3.46\pic18-lt\cxx-framework\src\traditional\proc\p18f8723.asm
                    TRISB   0x000f93       data     extern E:\3.46\pic18-lt\cxx-framework\src\traditional\proc\p18f8723.asm
                TRISBbits   0x000f93       data     extern E:\3.46\pic18-lt\cxx-framework\src\traditional\proc\p18f8723.asm
                 DDRBbits   0x000f93       data     extern E:\3.46\pic18-lt\cxx-framework\src\traditional\proc\p18f8723.asm
                     DDRB   0x000f93       data     extern E:\3.46\pic18-lt\cxx-framework\src\traditional\proc\p18f8723.asm
                TRISCbits   0x000f94       data     extern E:\3.46\pic18-lt\cxx-framework\src\traditional\proc\p18f8723.asm
                    TRISC   0x000f94       data     extern E:\3.46\pic18-lt\cxx-framework\src\traditional\proc\p18f8723.asm
                     DDRC   0x000f94       data     extern E:\3.46\pic18-lt\cxx-framework\src\traditional\proc\p18f8723.asm
                 DDRCbits   0x000f94       data     extern E:\3.46\pic18-lt\cxx-framework\src\traditional\proc\p18f8723.asm
                    TRISD   0x000f95       data     extern E:\3.46\pic18-lt\cxx-framework\src\traditional\proc\p18f8723.asm
                TRISDbits   0x000f95       data     extern E:\3.46\pic18-lt\cxx-framework\src\traditional\proc\p18f8723.asm
                     DDRD   0x000f95       data     extern E:\3.46\pic18-lt\cxx-framework\src\traditional\proc\p18f8723.asm
                 DDRDbits   0x000f95       data     extern E:\3.46\pic18-lt\cxx-framework\src\traditional\proc\p18f8723.asm
                 DDREbits   0x000f96       data     extern E:\3.46\pic18-lt\cxx-framework\src\traditional\proc\p18f8723.asm
                     DDRE   0x000f96       data     extern E:\3.46\pic18-lt\cxx-framework\src\traditional\proc\p18f8723.asm
                    TRISE   0x000f96       data     extern E:\3.46\pic18-lt\cxx-framework\src\traditional\proc\p18f8723.asm
                TRISEbits   0x000f96       data     extern E:\3.46\pic18-lt\cxx-framework\src\traditional\proc\p18f8723.asm
                 DDRFbits   0x000f97       data     extern E:\3.46\pic18-lt\cxx-framework\src\traditional\proc\p18f8723.asm
                TRISFbits   0x000f97       data     extern E:\3.46\pic18-lt\cxx-framework\src\traditional\proc\p18f8723.asm
                    TRISF   0x000f97       data     extern E:\3.46\pic18-lt\cxx-framework\src\traditional\proc\p18f8723.asm
                     DDRF   0x000f97       data     extern E:\3.46\pic18-lt\cxx-framework\src\traditional\proc\p18f8723.asm
                     DDRG   0x000f98       data     extern E:\3.46\pic18-lt\cxx-framework\src\traditional\proc\p18f8723.asm
                 DDRGbits   0x000f98       data     extern E:\3.46\pic18-lt\cxx-framework\src\traditional\proc\p18f8723.asm
                    TRISG   0x000f98       data     extern E:\3.46\pic18-lt\cxx-framework\src\traditional\proc\p18f8723.asm
                TRISGbits   0x000f98       data     extern E:\3.46\pic18-lt\cxx-framework\src\traditional\proc\p18f8723.asm
                 DDRHbits   0x000f99       data     extern E:\3.46\pic18-lt\cxx-framework\src\traditional\proc\p18f8723.asm
                     DDRH   0x000f99       data     extern E:\3.46\pic18-lt\cxx-framework\src\traditional\proc\p18f8723.asm
                TRISHbits   0x000f99       data     extern E:\3.46\pic18-lt\cxx-framework\src\traditional\proc\p18f8723.asm
                    TRISH   0x000f99       data     extern E:\3.46\pic18-lt\cxx-framework\src\traditional\proc\p18f8723.asm
                     DDRJ   0x000f9a       data     extern E:\3.46\pic18-lt\cxx-framework\src\traditional\proc\p18f8723.asm
                TRISJbits   0x000f9a       data     extern E:\3.46\pic18-lt\cxx-framework\src\traditional\proc\p18f8723.asm
                    TRISJ   0x000f9a       data     extern E:\3.46\pic18-lt\cxx-framework\src\traditional\proc\p18f8723.asm
                 DDRJbits   0x000f9a       data     extern E:\3.46\pic18-lt\cxx-framework\src\traditional\proc\p18f8723.asm
              OSCTUNEbits   0x000f9b       data     extern E:\3.46\pic18-lt\cxx-framework\src\traditional\proc\p18f8723.asm
                  OSCTUNE   0x000f9b       data     extern E:\3.46\pic18-lt\cxx-framework\src\traditional\proc\p18f8723.asm
                   MEMCON   0x000f9c       data     extern E:\3.46\pic18-lt\cxx-framework\src\traditional\proc\p18f8723.asm
               MEMCONbits   0x000f9c       data     extern E:\3.46\pic18-lt\cxx-framework\src\traditional\proc\p18f8723.asm
                 PIE1bits   0x000f9d       data     extern E:\3.46\pic18-lt\cxx-framework\src\traditional\proc\p18f8723.asm
                     PIE1   0x000f9d       data     extern E:\3.46\pic18-lt\cxx-framework\src\traditional\proc\p18f8723.asm
                     PIR1   0x000f9e       data     extern E:\3.46\pic18-lt\cxx-framework\src\traditional\proc\p18f8723.asm
                 PIR1bits   0x000f9e       data     extern E:\3.46\pic18-lt\cxx-framework\src\traditional\proc\p18f8723.asm
                     IPR1   0x000f9f       data     extern E:\3.46\pic18-lt\cxx-framework\src\traditional\proc\p18f8723.asm
                 IPR1bits   0x000f9f       data     extern E:\3.46\pic18-lt\cxx-framework\src\traditional\proc\p18f8723.asm
                 PIE2bits   0x000fa0       data     extern E:\3.46\pic18-lt\cxx-framework\src\traditional\proc\p18f8723.asm
                     PIE2   0x000fa0       data     extern E:\3.46\pic18-lt\cxx-framework\src\traditional\proc\p18f8723.asm
                     PIR2   0x000fa1       data     extern E:\3.46\pic18-lt\cxx-framework\src\traditional\proc\p18f8723.asm
                 PIR2bits   0x000fa1       data     extern E:\3.46\pic18-lt\cxx-framework\src\traditional\proc\p18f8723.asm
                     IPR2   0x000fa2       data     extern E:\3.46\pic18-lt\cxx-framework\src\traditional\proc\p18f8723.asm
                 IPR2bits   0x000fa2       data     extern E:\3.46\pic18-lt\cxx-framework\src\traditional\proc\p18f8723.asm
                     PIE3   0x000fa3       data     extern E:\3.46\pic18-lt\cxx-framework\src\traditional\proc\p18f8723.asm
                 PIE3bits   0x000fa3       data     extern E:\3.46\pic18-lt\cxx-framework\src\traditional\proc\p18f8723.asm
                     PIR3   0x000fa4       data     extern E:\3.46\pic18-lt\cxx-framework\src\traditional\proc\p18f8723.asm
                 PIR3bits   0x000fa4       data     extern E:\3.46\pic18-lt\cxx-framework\src\traditional\proc\p18f8723.asm
                     IPR3   0x000fa5       data     extern E:\3.46\pic18-lt\cxx-framework\src\traditional\proc\p18f8723.asm
                 IPR3bits   0x000fa5       data     extern E:\3.46\pic18-lt\cxx-framework\src\traditional\proc\p18f8723.asm
               EECON1bits   0x000fa6       data     extern E:\3.46\pic18-lt\cxx-framework\src\traditional\proc\p18f8723.asm
                   EECON1   0x000fa6       data     extern E:\3.46\pic18-lt\cxx-framework\src\traditional\proc\p18f8723.asm
                   EECON2   0x000fa7       data     extern E:\3.46\pic18-lt\cxx-framework\src\traditional\proc\p18f8723.asm
                   EEDATA   0x000fa8       data     extern E:\3.46\pic18-lt\cxx-framework\src\traditional\proc\p18f8723.asm
                    EEADR   0x000fa9       data     extern E:\3.46\pic18-lt\cxx-framework\src\traditional\proc\p18f8723.asm
                   EEADRH   0x000faa       data     extern E:\3.46\pic18-lt\cxx-framework\src\traditional\proc\p18f8723.asm
                RCSTAbits   0x000fab       data     extern E:\3.46\pic18-lt\cxx-framework\src\traditional\proc\p18f8723.asm
               RCSTA1bits   0x000fab       data     extern E:\3.46\pic18-lt\cxx-framework\src\traditional\proc\p18f8723.asm
                   RCSTA1   0x000fab       data     extern E:\3.46\pic18-lt\cxx-framework\src\traditional\proc\p18f8723.asm
                    RCSTA   0x000fab       data     extern E:\3.46\pic18-lt\cxx-framework\src\traditional\proc\p18f8723.asm
                   TXSTA1   0x000fac       data     extern E:\3.46\pic18-lt\cxx-framework\src\traditional\proc\p18f8723.asm
                    TXSTA   0x000fac       data     extern E:\3.46\pic18-lt\cxx-framework\src\traditional\proc\p18f8723.asm
               TXSTA1bits   0x000fac       data     extern E:\3.46\pic18-lt\cxx-framework\src\traditional\proc\p18f8723.asm
                TXSTAbits   0x000fac       data     extern E:\3.46\pic18-lt\cxx-framework\src\traditional\proc\p18f8723.asm
                    TXREG   0x000fad       data     extern E:\3.46\pic18-lt\cxx-framework\src\traditional\proc\p18f8723.asm
                   TXREG1   0x000fad       data     extern E:\3.46\pic18-lt\cxx-framework\src\traditional\proc\p18f8723.asm
                   RCREG1   0x000fae       data     extern E:\3.46\pic18-lt\cxx-framework\src\traditional\proc\p18f8723.asm
                    RCREG   0x000fae       data     extern E:\3.46\pic18-lt\cxx-framework\src\traditional\proc\p18f8723.asm
                   SPBRG1   0x000faf       data     extern E:\3.46\pic18-lt\cxx-framework\src\traditional\proc\p18f8723.asm
                    SPBRG   0x000faf       data     extern E:\3.46\pic18-lt\cxx-framework\src\traditional\proc\p18f8723.asm
                   PSPCON   0x000fb0       data     extern E:\3.46\pic18-lt\cxx-framework\src\traditional\proc\p18f8723.asm
               PSPCONbits   0x000fb0       data     extern E:\3.46\pic18-lt\cxx-framework\src\traditional\proc\p18f8723.asm
                    T3CON   0x000fb1       data     extern E:\3.46\pic18-lt\cxx-framework\src\traditional\proc\p18f8723.asm
                T3CONbits   0x000fb1       data     extern E:\3.46\pic18-lt\cxx-framework\src\traditional\proc\p18f8723.asm
                    TMR3L   0x000fb2       data     extern E:\3.46\pic18-lt\cxx-framework\src\traditional\proc\p18f8723.asm
                    TMR3H   0x000fb3       data     extern E:\3.46\pic18-lt\cxx-framework\src\traditional\proc\p18f8723.asm
                    CMCON   0x000fb4       data     extern E:\3.46\pic18-lt\cxx-framework\src\traditional\proc\p18f8723.asm
                CMCONbits   0x000fb4       data     extern E:\3.46\pic18-lt\cxx-framework\src\traditional\proc\p18f8723.asm
               CVRCONbits   0x000fb5       data     extern E:\3.46\pic18-lt\cxx-framework\src\traditional\proc\p18f8723.asm
                   CVRCON   0x000fb5       data     extern E:\3.46\pic18-lt\cxx-framework\src\traditional\proc\p18f8723.asm
              ECCP1ASbits   0x000fb6       data     extern E:\3.46\pic18-lt\cxx-framework\src\traditional\proc\p18f8723.asm
                  ECCP1AS   0x000fb6       data     extern E:\3.46\pic18-lt\cxx-framework\src\traditional\proc\p18f8723.asm
                 ECCP3CON   0x000fb7       data     extern E:\3.46\pic18-lt\cxx-framework\src\traditional\proc\p18f8723.asm
             ECCP3CONbits   0x000fb7       data     extern E:\3.46\pic18-lt\cxx-framework\src\traditional\proc\p18f8723.asm
              CCP3CONbits   0x000fb7       data     extern E:\3.46\pic18-lt\cxx-framework\src\traditional\proc\p18f8723.asm
                  CCP3CON   0x000fb7       data     extern E:\3.46\pic18-lt\cxx-framework\src\traditional\proc\p18f8723.asm
                   CCPR3L   0x000fb8       data     extern E:\3.46\pic18-lt\cxx-framework\src\traditional\proc\p18f8723.asm
                    CCPR3   0x000fb8       data     extern E:\3.46\pic18-lt\cxx-framework\src\traditional\proc\p18f8723.asm
                   CCPR3H   0x000fb9       data     extern E:\3.46\pic18-lt\cxx-framework\src\traditional\proc\p18f8723.asm
                  CCP2CON   0x000fba       data     extern E:\3.46\pic18-lt\cxx-framework\src\traditional\proc\p18f8723.asm
              CCP2CONbits   0x000fba       data     extern E:\3.46\pic18-lt\cxx-framework\src\traditional\proc\p18f8723.asm
                 ECCP2CON   0x000fba       data     extern E:\3.46\pic18-lt\cxx-framework\src\traditional\proc\p18f8723.asm
             ECCP2CONbits   0x000fba       data     extern E:\3.46\pic18-lt\cxx-framework\src\traditional\proc\p18f8723.asm
                   CCPR2L   0x000fbb       data     extern E:\3.46\pic18-lt\cxx-framework\src\traditional\proc\p18f8723.asm
                    CCPR2   0x000fbb       data     extern E:\3.46\pic18-lt\cxx-framework\src\traditional\proc\p18f8723.asm
                   CCPR2H   0x000fbc       data     extern E:\3.46\pic18-lt\cxx-framework\src\traditional\proc\p18f8723.asm
              CCP1CONbits   0x000fbd       data     extern E:\3.46\pic18-lt\cxx-framework\src\traditional\proc\p18f8723.asm
                  CCP1CON   0x000fbd       data     extern E:\3.46\pic18-lt\cxx-framework\src\traditional\proc\p18f8723.asm
                 ECCP1CON   0x000fbd       data     extern E:\3.46\pic18-lt\cxx-framework\src\traditional\proc\p18f8723.asm
             ECCP1CONbits   0x000fbd       data     extern E:\3.46\pic18-lt\cxx-framework\src\traditional\proc\p18f8723.asm
                   CCPR1L   0x000fbe       data     extern E:\3.46\pic18-lt\cxx-framework\src\traditional\proc\p18f8723.asm
                    CCPR1   0x000fbe       data     extern E:\3.46\pic18-lt\cxx-framework\src\traditional\proc\p18f8723.asm
                   CCPR1H   0x000fbf       data     extern E:\3.46\pic18-lt\cxx-framework\src\traditional\proc\p18f8723.asm
               ADCON2bits   0x000fc0       data     extern E:\3.46\pic18-lt\cxx-framework\src\traditional\proc\p18f8723.asm
                   ADCON2   0x000fc0       data     extern E:\3.46\pic18-lt\cxx-framework\src\traditional\proc\p18f8723.asm
               ADCON1bits   0x000fc1       data     extern E:\3.46\pic18-lt\cxx-framework\src\traditional\proc\p18f8723.asm
                   ADCON1   0x000fc1       data     extern E:\3.46\pic18-lt\cxx-framework\src\traditional\proc\p18f8723.asm
               ADCON0bits   0x000fc2       data     extern E:\3.46\pic18-lt\cxx-framework\src\traditional\proc\p18f8723.asm
                   ADCON0   0x000fc2       data     extern E:\3.46\pic18-lt\cxx-framework\src\traditional\proc\p18f8723.asm
                   ADRESL   0x000fc3       data     extern E:\3.46\pic18-lt\cxx-framework\src\traditional\proc\p18f8723.asm
                    ADRES   0x000fc3       data     extern E:\3.46\pic18-lt\cxx-framework\src\traditional\proc\p18f8723.asm
                   ADRESH   0x000fc4       data     extern E:\3.46\pic18-lt\cxx-framework\src\traditional\proc\p18f8723.asm
              SSPCON2bits   0x000fc5       data     extern E:\3.46\pic18-lt\cxx-framework\src\traditional\proc\p18f8723.asm
                  SSPCON2   0x000fc5       data     extern E:\3.46\pic18-lt\cxx-framework\src\traditional\proc\p18f8723.asm
             SSP1CON2bits   0x000fc5       data     extern E:\3.46\pic18-lt\cxx-framework\src\traditional\proc\p18f8723.asm
                 SSP1CON2   0x000fc5       data     extern E:\3.46\pic18-lt\cxx-framework\src\traditional\proc\p18f8723.asm
              SSPCON1bits   0x000fc6       data     extern E:\3.46\pic18-lt\cxx-framework\src\traditional\proc\p18f8723.asm
                  SSPCON1   0x000fc6       data     extern E:\3.46\pic18-lt\cxx-framework\src\traditional\proc\p18f8723.asm
                 SSP1CON1   0x000fc6       data     extern E:\3.46\pic18-lt\cxx-framework\src\traditional\proc\p18f8723.asm
             SSP1CON1bits   0x000fc6       data     extern E:\3.46\pic18-lt\cxx-framework\src\traditional\proc\p18f8723.asm
                 SSP1STAT   0x000fc7       data     extern E:\3.46\pic18-lt\cxx-framework\src\traditional\proc\p18f8723.asm
             SSP1STATbits   0x000fc7       data     extern E:\3.46\pic18-lt\cxx-framework\src\traditional\proc\p18f8723.asm
                  SSPSTAT   0x000fc7       data     extern E:\3.46\pic18-lt\cxx-framework\src\traditional\proc\p18f8723.asm
              SSPSTATbits   0x000fc7       data     extern E:\3.46\pic18-lt\cxx-framework\src\traditional\proc\p18f8723.asm
                  SSP1ADD   0x000fc8       data     extern E:\3.46\pic18-lt\cxx-framework\src\traditional\proc\p18f8723.asm
                   SSPADD   0x000fc8       data     extern E:\3.46\pic18-lt\cxx-framework\src\traditional\proc\p18f8723.asm
                  SSP1BUF   0x000fc9       data     extern E:\3.46\pic18-lt\cxx-framework\src\traditional\proc\p18f8723.asm
                   SSPBUF   0x000fc9       data     extern E:\3.46\pic18-lt\cxx-framework\src\traditional\proc\p18f8723.asm
                T2CONbits   0x000fca       data     extern E:\3.46\pic18-lt\cxx-framework\src\traditional\proc\p18f8723.asm
                    T2CON   0x000fca       data     extern E:\3.46\pic18-lt\cxx-framework\src\traditional\proc\p18f8723.asm
                      PR2   0x000fcb       data     extern E:\3.46\pic18-lt\cxx-framework\src\traditional\proc\p18f8723.asm
                     TMR2   0x000fcc       data     extern E:\3.46\pic18-lt\cxx-framework\src\traditional\proc\p18f8723.asm
                    T1CON   0x000fcd       data     extern E:\3.46\pic18-lt\cxx-framework\src\traditional\proc\p18f8723.asm
                T1CONbits   0x000fcd       data     extern E:\3.46\pic18-lt\cxx-framework\src\traditional\proc\p18f8723.asm
                    TMR1L   0x000fce       data     extern E:\3.46\pic18-lt\cxx-framework\src\traditional\proc\p18f8723.asm
                    TMR1H   0x000fcf       data     extern E:\3.46\pic18-lt\cxx-framework\src\traditional\proc\p18f8723.asm
                     RCON   0x000fd0       data     extern E:\3.46\pic18-lt\cxx-framework\src\traditional\proc\p18f8723.asm
                 RCONbits   0x000fd0       data     extern E:\3.46\pic18-lt\cxx-framework\src\traditional\proc\p18f8723.asm
                   WDTCON   0x000fd1       data     extern E:\3.46\pic18-lt\cxx-framework\src\traditional\proc\p18f8723.asm
               WDTCONbits   0x000fd1       data     extern E:\3.46\pic18-lt\cxx-framework\src\traditional\proc\p18f8723.asm
                   LVDCON   0x000fd2       data     extern E:\3.46\pic18-lt\cxx-framework\src\traditional\proc\p18f8723.asm
               LVDCONbits   0x000fd2       data     extern E:\3.46\pic18-lt\cxx-framework\src\traditional\proc\p18f8723.asm
              HLVDCONbits   0x000fd2       data     extern E:\3.46\pic18-lt\cxx-framework\src\traditional\proc\p18f8723.asm
                  HLVDCON   0x000fd2       data     extern E:\3.46\pic18-lt\cxx-framework\src\traditional\proc\p18f8723.asm
                   OSCCON   0x000fd3       data     extern E:\3.46\pic18-lt\cxx-framework\src\traditional\proc\p18f8723.asm
               OSCCONbits   0x000fd3       data     extern E:\3.46\pic18-lt\cxx-framework\src\traditional\proc\p18f8723.asm
                T0CONbits   0x000fd5       data     extern E:\3.46\pic18-lt\cxx-framework\src\traditional\proc\p18f8723.asm
                    T0CON   0x000fd5       data     extern E:\3.46\pic18-lt\cxx-framework\src\traditional\proc\p18f8723.asm
                    TMR0L   0x000fd6       data     extern E:\3.46\pic18-lt\cxx-framework\src\traditional\proc\p18f8723.asm
                    TMR0H   0x000fd7       data     extern E:\3.46\pic18-lt\cxx-framework\src\traditional\proc\p18f8723.asm
               STATUSbits   0x000fd8       data     extern E:\3.46\pic18-lt\cxx-framework\src\traditional\proc\p18f8723.asm
                   STATUS   0x000fd8       data     extern E:\3.46\pic18-lt\cxx-framework\src\traditional\proc\p18f8723.asm
                    FSR2L   0x000fd9       data     extern E:\3.46\pic18-lt\cxx-framework\src\traditional\proc\p18f8723.asm
                     FSR2   0x000fd9       data     extern E:\3.46\pic18-lt\cxx-framework\src\traditional\proc\p18f8723.asm
                    FSR2H   0x000fda       data     extern E:\3.46\pic18-lt\cxx-framework\src\traditional\proc\p18f8723.asm
                   PLUSW2   0x000fdb       data     extern E:\3.46\pic18-lt\cxx-framework\src\traditional\proc\p18f8723.asm
                  PREINC2   0x000fdc       data     extern E:\3.46\pic18-lt\cxx-framework\src\traditional\proc\p18f8723.asm
                 POSTDEC2   0x000fdd       data     extern E:\3.46\pic18-lt\cxx-framework\src\traditional\proc\p18f8723.asm
                 POSTINC2   0x000fde       data     extern E:\3.46\pic18-lt\cxx-framework\src\traditional\proc\p18f8723.asm
                    INDF2   0x000fdf       data     extern E:\3.46\pic18-lt\cxx-framework\src\traditional\proc\p18f8723.asm
                      BSR   0x000fe0       data     extern E:\3.46\pic18-lt\cxx-framework\src\traditional\proc\p18f8723.asm
                    FSR1L   0x000fe1       data     extern E:\3.46\pic18-lt\cxx-framework\src\traditional\proc\p18f8723.asm
                     FSR1   0x000fe1       data     extern E:\3.46\pic18-lt\cxx-framework\src\traditional\proc\p18f8723.asm
                    FSR1H   0x000fe2       data     extern E:\3.46\pic18-lt\cxx-framework\src\traditional\proc\p18f8723.asm
                   PLUSW1   0x000fe3       data     extern E:\3.46\pic18-lt\cxx-framework\src\traditional\proc\p18f8723.asm
                  PREINC1   0x000fe4       data     extern E:\3.46\pic18-lt\cxx-framework\src\traditional\proc\p18f8723.asm
                 POSTDEC1   0x000fe5       data     extern E:\3.46\pic18-lt\cxx-framework\src\traditional\proc\p18f8723.asm
                 POSTINC1   0x000fe6       data     extern E:\3.46\pic18-lt\cxx-framework\src\traditional\proc\p18f8723.asm
                    INDF1   0x000fe7       data     extern E:\3.46\pic18-lt\cxx-framework\src\traditional\proc\p18f8723.asm
                     WREG   0x000fe8       data     extern E:\3.46\pic18-lt\cxx-framework\src\traditional\proc\p18f8723.asm
                     FSR0   0x000fe9       data     extern E:\3.46\pic18-lt\cxx-framework\src\traditional\proc\p18f8723.asm
                    FSR0L   0x000fe9       data     extern E:\3.46\pic18-lt\cxx-framework\src\traditional\proc\p18f8723.asm
                    FSR0H   0x000fea       data     extern E:\3.46\pic18-lt\cxx-framework\src\traditional\proc\p18f8723.asm
                   PLUSW0   0x000feb       data     extern E:\3.46\pic18-lt\cxx-framework\src\traditional\proc\p18f8723.asm
                  PREINC0   0x000fec       data     extern E:\3.46\pic18-lt\cxx-framework\src\traditional\proc\p18f8723.asm
                 POSTDEC0   0x000fed       data     extern E:\3.46\pic18-lt\cxx-framework\src\traditional\proc\p18f8723.asm
                 POSTINC0   0x000fee       data     extern E:\3.46\pic18-lt\cxx-framework\src\traditional\proc\p18f8723.asm
                    INDF0   0x000fef       data     extern E:\3.46\pic18-lt\cxx-framework\src\traditional\proc\p18f8723.asm
                  INTCON3   0x000ff0       data     extern E:\3.46\pic18-lt\cxx-framework\src\traditional\proc\p18f8723.asm
              INTCON3bits   0x000ff0       data     extern E:\3.46\pic18-lt\cxx-framework\src\traditional\proc\p18f8723.asm
                  INTCON2   0x000ff1       data     extern E:\3.46\pic18-lt\cxx-framework\src\traditional\proc\p18f8723.asm
              INTCON2bits   0x000ff1       data     extern E:\3.46\pic18-lt\cxx-framework\src\traditional\proc\p18f8723.asm
               INTCONbits   0x000ff2       data     extern E:\3.46\pic18-lt\cxx-framework\src\traditional\proc\p18f8723.asm
                   INTCON   0x000ff2       data     extern E:\3.46\pic18-lt\cxx-framework\src\traditional\proc\p18f8723.asm
                     PROD   0x000ff3       data     extern E:\3.46\pic18-lt\cxx-framework\src\traditional\proc\p18f8723.asm
                    PRODL   0x000ff3       data     extern E:\3.46\pic18-lt\cxx-framework\src\traditional\proc\p18f8723.asm
                    PRODH   0x000ff4       data     extern E:\3.46\pic18-lt\cxx-framework\src\traditional\proc\p18f8723.asm
                   TABLAT   0x000ff5       data     extern E:\3.46\pic18-lt\cxx-framework\src\traditional\proc\p18f8723.asm
                  TBLPTRL   0x000ff6       data     extern E:\3.46\pic18-lt\cxx-framework\src\traditional\proc\p18f8723.asm
                   TBLPTR   0x000ff6       data     extern E:\3.46\pic18-lt\cxx-framework\src\traditional\proc\p18f8723.asm
                  TBLPTRH   0x000ff7       data     extern E:\3.46\pic18-lt\cxx-framework\src\traditional\proc\p18f8723.asm
                  TBLPTRU   0x000ff8       data     extern E:\3.46\pic18-lt\cxx-framework\src\traditional\proc\p18f8723.asm
                      PCL   0x000ff9       data     extern E:\3.46\pic18-lt\cxx-framework\src\traditional\proc\p18f8723.asm
                       PC   0x000ff9       data     extern E:\3.46\pic18-lt\cxx-framework\src\traditional\proc\p18f8723.asm
                   PCLATH   0x000ffa       data     extern E:\3.46\pic18-lt\cxx-framework\src\traditional\proc\p18f8723.asm
                   PCLATU   0x000ffb       data     extern E:\3.46\pic18-lt\cxx-framework\src\traditional\proc\p18f8723.asm
                   STKPTR   0x000ffc       data     extern E:\3.46\pic18-lt\cxx-framework\src\traditional\proc\p18f8723.asm
               STKPTRbits   0x000ffc       data     extern E:\3.46\pic18-lt\cxx-framework\src\traditional\proc\p18f8723.asm
                     TOSL   0x000ffd       data     extern E:\3.46\pic18-lt\cxx-framework\src\traditional\proc\p18f8723.asm
                      TOS   0x000ffd       data     extern E:\3.46\pic18-lt\cxx-framework\src\traditional\proc\p18f8723.asm
                     TOSH   0x000ffe       data     extern E:\3.46\pic18-lt\cxx-framework\src\traditional\proc\p18f8723.asm
                     TOSU   0x000fff       data     extern E:\3.46\pic18-lt\cxx-framework\src\traditional\proc\p18f8723.asm


